:020000040000FA
:0400000007EF00F016
:100008007482CCED45F0ECEF4BF080C0D9FF81C095
:10001800DAFF000EDE6E000EDD6E82C00CF0A7EC7B
:1000280049F00CC0BCF00DC0BDF00001BDAF02D05E
:100038000B0E1200D890BC35D96EBD35DA6E820E23
:10004800D926010EDA22DECFD6F0DDCFD7F0D65191
:10005800D711D8A402D00C0E120080C0D9FF81C0DD
:10006800DAFFD6C0DEFFD7C0DDFFD6C0D9FFD7C0C4
:10007800DAFFDF50D8B415D020EE01F0D651D926DA
:10008800D751DA22DF5003EC5AF00001C86FC8B12B
:1000980008D08351D8A4C8A502D00A0E1200000EB9
:1000A8001200D6C0D9FFD7C0DAFF000EDF6E20EEEF
:1000B80001F0D651D926D751DA22BCC0DFFF20EE95
:1000C80001F0D651D926D751DA22DF5017EC41F08A
:1000D8000001C86FC8A102D0030E12008351D8B422
:1000E80002D0C8B5DAD7000ECF6F000ED06F000E61
:1000F800D16F000ED26FD6C045F0D7C046F0000EC3
:10010800476E000E486E000E496E000E4A6EA7EC50
:1001180038F00001D56FD505D8A4E6D0000ED46F0D
:10012800000ED36FD45105E1040ED35DD8B098D03A
:1001380001D096D0D3C084F0D4C085F0843B853BF1
:10014800F00E851784510F0B8513F00E8417D6C057
:1001580086F0D7C087F08451862785518723EC0E17
:100168008625C96F010E8721CA6F20EE04F0C95198
:10017800D926CA51DA22DF50D8A408D0000EAE6FB3
:10018800000EAF6F000EB06F000E58D020EE09F0D1
:10019800C951D926CA51DA22DF50846F8451866F3B
:1001A800856B20EE0AF0C951D926CA51DA22DF50F0
:1001B800876F87C088F0896B8A6B8B6B89C08BF0DF
:1001C80088C08AF0896B886B20EE0BF0C951D9265C
:1001D800CA51DA22DF508C6F8CC08DF08E6B8F6B1A
:1001E800906B8DC090F08F6B8E6B8D6B88518D11DD
:1001F800916F89518E11926F8A518F11936F8B5124
:100208009011946F85519111956F86519211966F47
:10021800000E9311976F000E9411986F20EE08F05E
:10022800C951D926CA51DA22DF50996F99519511CF
:10023800AE6F9651AF6F9751B06F9851B16FD35160
:10024800040DF3509E0FD96EDA6AAEC0DEFFAFC060
:10025800DEFFB0C0DEFFB1C0DEFFD34BD42B62D7C8
:10026800000ED46F000ED36FD351D411D8B403D07D
:10027800D307D8A0D407D351040DF3509E0FD96EDD
:10028800DA6ADECFCFF0DECFD0F0DECFD1F0DECF2E
:10029800D2F0CF51D011D111D211D8A405D0000E6F
:1002A800B36F020EB26F13D0D6C045F0D7C046F078
:1002B800CFC047F0D0C048F0D1C049F0D2C04AF012
:1002C800A7EC38F00001846F8451B26FB36BB2C0F1
:1002D800D5F0D551D8B408D0D34BD42BD45104E1A0
:1002E800040ED35DD8A0C7D7030ED519D8A402D061
:1002F800010E1200D551D8B402D00D0E120020EE16
:100308003AF0D651D926D751DA22DF50846F84517A
:10031800866F856B20EE39F0D651D926D751DA226F
:10032800DF50876F87518513000E8613020E8619DA
:100338008511D8A4E2D720EE45F0D651D926D75159
:10034800DA22DF50846F8451866F856B20EE44F08B
:10035800D651D926D751DA22DF50876F87518513B6
:10036800000E861385C0CBF086C0CCF0CD6BCE6B6B
:10037800CB51CC11CD11CE11D8A459D020EE53F0C9
:10038800D651D926D751DA22DF50846F8451866F2F
:10039800856B20EE54F0D651D926D751DA22DF509A
:1003A800876F87C088F0896B8A6B8B6B89C08BF0ED
:1003B80088C08AF0896B886B20EE55F0D651D92613
:1003C800D751DA22DF508C6F8CC08DF08E6B8F6B1B
:1003D800906B8DC090F08F6B8E6B8D6B88518D11EB
:1003E800916F89518E11926F8A518F11936F8B5132
:1003F8009011946F85519111956F86519211966F56
:10040800000E9311976F000E9411986F20EE52F022
:10041800D651D926D751DA22DF50996F99519511C3
:10042800CB6F9651CC6F9751CD6F9851CE6F20EE10
:1004380016F0D651D926D751DA22CBC0DEFFCCC070
:10044800DEFFCDC0DEFFCEC0DEFF20EE3EF0D6518F
:10045800D926D751DA2210EE03F0D651E126D7512A
:10046800E222DFCFE7FF20EE03F0D651D926D7519D
:10047800DA22DE04D8B40AD020EE03F0D651D92609
:10048800D751DA22020EDE18D8A437D7CBC00CF029
:10049800CCC00DF0CDC00EF0CEC00FF020EE03F0B2
:1004A800D651D926D751DA22DF50846F8451106E85
:1004B800116A126A136AACEC55F00CC0CBF00DC08F
:1004C800CCF00EC0CDF00FC0CEF0000120EE3BF016
:1004D800D651D926D751DA2210EE02F0D651E126AC
:1004E800D751E222DFCFE7FF20EE02F0D651D9261E
:1004F800D751DA22DF50D8B400D720EE02F0D65117
:10050800D926D751DA22DF50846F20EE02F0D65177
:10051800D926D751DA22DF50856F85058415000961
:10052800D8A4EBD620EE40F0D651D926D751DA22FE
:10053800DF50846F8451866F856B20EE3FF0D65173
:10054800D926D751DA22DF50876F87518513000EDD
:10055800861320EE08F0D651D926D751DA2285C065
:10056800DEFF86C0DDFF20EE08F0D651D926D75130
:10057800DA22DF50846F0F0E8417D8A4BED620EE7F
:1005880042F0D651D926D751DA22DF50846F8451F0
:10059800866F856B20EE41F0D651D926D751DA22E5
:1005A800DF50876F87518513000E861385C0C0F012
:1005B80086C0C1F0C26BC36BC051C111C211C31157
:1005C800D8A459D020EE4FF0D651D926D751DA22E7
:1005D800DF50846F8451866F856B20EE50F0D651C2
:1005E800D926D751DA22DF50876F87C088F0896B08
:1005F8008A6B8B6B89C08BF088C08AF0896B886B9B
:1006080020EE51F0D651D926D751DA22DF508C6F1F
:100618008CC08DF08E6B8F6B906B8DC090F08F6B54
:100628008E6B8D6B88518D11916F89518E11926FE0
:100638008A518F11936F8B519011946F855191113D
:10064800956F86519211966F000E9311976F000E59
:100658009411986F20EE4EF0D651D926D751DA2250
:10066800DF50996F99519511C06F9651C16F97518D
:10067800C26F9851C36F20EE3CF0D651D926D7519E
:10068800DA22DF50846F20EE3DF0D651D926D751BB
:10069800DA22DF50856F8451BE6F85C0BFF0BE512E
:1006A800BF11D8B42AD620EE08F0D651D926D75192
:1006B800DA22DECF84F0DDCF85F0040E866FD89085
:1006C80085338433862FFBD7BE518425876FBF516E
:1006D8008521886F896BD8B0892B8A6BCB51872588
:1006E800B86FCC518821B96FCD518921BA6FCE51DD
:1006F8008A21BB6FB851C05DB951C159BA51C259AD
:10070800BB51C359D8A0F9D5B851C05D0C6EB951C9
:10071800C1590D6EBA51C2590E6EBB51C3590F6EF5
:1007280020EE02F0D651D926D751DA22DF50846F55
:100738008451106E116A126A136A9AEC53F00CC055
:10074800C4F00DC0C5F00EC0C6F00FC0C7F0000160
:10075800C451C511C611C711D8B4CFD5010ED56F74
:10076800C751C61106E1F60EC45D0F0EC559D8A0D3
:1007780002D0020ED56FC751C61106E1F60EC45D50
:10078800FF0EC559D8A002D0030ED56F020EC4259E
:10079800846F000EC521856F000EC621866F000E7E
:1007A800C721876F20EE12F0D651D926D751DA2209
:1007B80084C0DEFF85C0DEFF86C0DEFF87C0DEFFA7
:1007C80020EE1AF0D651D926D751DA22CFC0DEFF53
:1007D800D0C0DEFFD1C0DEFFD2C0DEFFBE51CF25C4
:1007E800846FBF51D021856F000ED121866F000E16
:1007F800D221876F20EE1EF0D651D926D751DA22A2
:1008080084C0DEFF85C0DEFF86C0DEFF87C0DEFF56
:10081800B851CF25846FB951D021856FBA51D121F4
:10082800866FBB51D221876F20EE26F0D651D9268C
:10083800D751DA2284C0DEFF85C0DEFF86C0DEFF26
:1008480087C0DEFF030ED519D8A490D020EE08F09B
:10085800D651D926D751DA22DE50DE10D8A44DD58C
:1008680020EE5BF0D651D926D751DA22DF50846FBB
:100878008451866F856B20EE5CF0D651D926D7510E
:10088800DA22DF50876F87C088F0896B8A6B8B6BA1
:1008980089C08BF088C08AF0896B886B20EE5DF088
:1008A800D651D926D751DA22DF508C6F8CC08DF003
:1008B8008E6B8F6B906B8DC090F08F6B8E6B8D6B8A
:1008C80088518D11916F89518E11926F8A518F11B4
:1008D800936F8B519011946F85519111956F86513B
:1008E8009211966F000E9311976F000E9411986FE6
:1008F80020EE5AF0D651D926D751DA22DF50996F17
:10090800995195119A6F96519B6F97519C6F985179
:100918009D6F20EE22F0D651D926D751DA229AC0FF
:10092800DEFF9BC0DEFF9CC0DEFF9DC0DEFF20EE29
:1009380012F0D651D926D751DA22DECF84F0DECF95
:1009480085F0DECF86F0DECF87F0020ED8908437B0
:10095800853786378737E82EF9D784C0B4F085C045
:10096800B5F086C0B6F087C0B7F091D020EE08F099
:10097800D651D926D751DA22DE50DE10D8B4BDD4EC
:1009880020EE1EF0D651D926D751DA22DECF84F0D8
:10099800DECF85F0DECF86F0DECF87F0CB51842521
:1009A800886FCC518521896FCD5186218A6FCE51B0
:1009B80087218B6F20EE22F0D651D926D751DA2223
:1009C80088C0DEFF89C0DEFF8AC0DEFF8BC0DEFF85
:1009D800020ED519D8B444D020EE12F0D651D9263B
:1009E800D751DA22DECF84F0DECF85F0DECF86F075
:1009F800DECF87F0010E8415886F000E8515896F8C
:100A0800000E86158A6F000E87158B6F20EE12F088
:100A1800D651D926D751DA22DECF0CF0DECF0DF031
:100A2800DECF0EF0DECF0FF0030E106E000E116E4B
:100A3800000E126E000E136EACEC55F0D8900F320B
:100A48000E320D320C32000188510C24B46F8951DA
:100A58000D20B56F8A510E20B66F8B510F2016D01E
:100A680020EE12F0D651D926D751DA22DECF84F003
:100A7800DECF85F0DECF86F0DECF87F0D8908435E4
:100A8800B46F8535B56F8635B66F8735B76FFF0E8E
:100A9800B425846F010EB521856F000EB621866FCF
:100AA800000EB721876F0A0E05D0D890873386339A
:100AB80085338433E82EF9D720EE16F0D651D9269F
:100AC800D751DA228451DE5C8551DE588651DE58D2
:100AD8008751DE58D8A011D420EE0EF0D651D92671
:100AE800D751DA22FF0EDE6EFF0EDE6EFF0EDE6ECF
:100AF800FF0EDD6EDD52DD5210EE0AF0D651E12612
:100B0800D751E222DECFE6FFDECFE6FFDECFE6FFFB
:100B1800DECFE6FF20EE05F0D651D926D751DA22EE
:100B2800800EDF6E030ED519D8A4F1D120EE5FF048
:100B3800D651D926D751DA22DF50846F8451866F77
:100B4800856B20EE5EF0D651D926D751DA22DF50D8
:100B5800876F87518513000E861385058611D8A4E3
:100B6800D6D1D6C03AF0D7C03BF0010ECF253C6EA7
:100B7800000ED0213D6E000ED1213E6E000ED22116
:100B88003F6E78EC50F00009D8A4C1D1000120EEE6
:100B980005F0D651D926D751DA22000EDF6E22EEA3
:100BA8002DF0D651D926D751DA22DF50846F8451DF
:100BB800866F856B22EE2CF0D651D926D751DA22D2
:100BC800DF50876F87518513000E8613550E8519E0
:100BD80003E1AA0E8619D8A49AD120EE2FF0D65197
:100BE800D926D751DA22DF50846F8451866F856BFE
:100BF80020EE30F0D651D926D751DA22DF50876F50
:100C080087C088F0896B8A6B8B6B89C08BF088C032
:100C18008AF0896B886B20EE31F0D651D926D751EE
:100C2800DA22DF508C6F8CC08DF08E6B8F6B906BDF
:100C38008DC090F08F6B8E6B8D6B88518D11916F7D
:100C480089518E11926F8A518F11936F8B51901128
:100C5800946F85519111956F86519211966F000E80
:100C68009311976F000E9411986F20EE2EF0D651C5
:100C7800D926D751DA22DF50996F995195119A6F79
:100C880096519B6F97519C6F98519D6F520E9A1970
:100C980009E1520E9B1906E1610E9C1903E1410E10
:100CA8009D19D8A434D122EE13F0D651D926D751A4
:100CB800DA22DF50846F8451866F856B22EE14F040
:100CC800D651D926D751DA22DF50876F87C088F0EE
:100CD800896B8A6B8B6B89C08BF088C08AF0896BB3
:100CE800886B22EE15F0D651D926D751DA22DF507B
:100CF8008C6F8CC08DF08E6B8F6B906B8DC090F06D
:100D08008F6B8E6B8D6B88518D11916F89518E1100
:100D1800926F8A518F11936F8B519011946F8551F7
:100D28009111956F86519211966F000E9311976FDE
:100D3800000E9411986F22EE12F0D651D926D75191
:100D4800DA22DF50996F995195119A6F96519B6FDE
:100D580097519C6F98519D6F720E9A1909E1720E06
:100D68009B1906E1410E9C1903E1610E9D19D8A457
:100D7800CED022EE17F0D651D926D751DA22DF503D
:100D8800846F8451866F856B22EE18F0D651D92670
:100D9800D751DA22DF50876F87C088F0896B8A6B5A
:100DA8008B6B89C08BF088C08AF0896B886B22EEC8
:100DB80019F0D651D926D751DA22DF508C6F8CC062
:100DC8008DF08E6B8F6B906B8DC090F08F6B8E6BF0
:100DD8008D6B88518D11916F89518E11926F8A5147
:100DE8008F11936F8B519011946F85519111956F5D
:100DF80086519211966F000E9311976F000E941101
:100E0800986F22EE16F0D651D926D751DA22DF5044
:100E1800996F995195119A6F96519B6F97519C6F45
:100E280098519D6F20EE0EF0D651D926D751DA226F
:100E38009AC0DEFF9BC0DEFF9CC0DEFF9DC0DEFFC8
:100E480022EE1BF0D651D926D751DA22DF50846F13
:100E58008451866F856B22EE1CF0D651D926D75166
:100E6800DA22DF50876F87C088F0896B8A6B8B6BBB
:100E780089C08BF088C08AF0896B886B22EE1DF0E0
:100E8800D651D926D751DA22DF508C6F8CC08DF01D
:100E98008E6B8F6B906B8DC090F08F6B8E6B8D6BA4
:100EA80088518D11916F89518E11926F8A518F11CE
:100EB800936F8B519011946F85519111956F865155
:100EC8009211966F000E9311976F000E9411986F00
:100ED80022EE1AF0D651D926D751DA22DF50996F6F
:100EE800995195119A6F96519B6F97519C6F985194
:100EF8009D6F20EE0AF0D651D926D751DA229AC032
:100F0800DEFF9BC0DEFF9CC0DEFF9DC0DEFFD6C0BB
:100F1800D9FFD7C0DAFFD5C0DFFF0101804B812B95
:100F2800000120EE06F0D651D926D751DA2280C129
:100F3800DEFF81C1DDFF53EF00F0000E0101A66F57
:100F4800000E906F070E966E010EE16F000EA86FEF
:100F58000F0EC16E926893689468948E92909292E4
:100F68008982020E726E86EC58F092948984929867
:100F78008998929E899E95689368810E0001806F7A
:100F8800F60E816FCD0E826FFF0E836FD70E846FC2
:100F9800FE0E856F310E866FFF0E876FC9EC59F014
:100FA8009DEC59F017D08A0E0001806FFE0E816FFC
:100FB80082CF82F0836BC9EC59F0150E0101DB6F0B
:100FC8004B0EDA6FBE0EE82EFED7DA2FFCD7DB2FDA
:100FD800FAD700F082B2E7D7FCEC58F0A66F270EDC
:100FE8000001806FFD0E816FA6C182F0836BC9EC92
:100FF80059F00400150E0101DB6F4B0EDA6FBE0EBF
:10100800E82EFED7DA2FFCD7DB2FFAD700F0F286CE
:10101800F180F288F19CF28ED3EC52F08992899497
:101028008980040042EC32F0A9EC43F05BEC59F003
:101038008F51D8B4E4D05A0E0001806FFD0E816F35
:10104800C9EC59F0CCEC4FF049C0E9F34AC0EAF3D7
:101058004BC0EBF34CC0ECF3000E0301F76F000E2E
:10106800F66FD90E0001806FFF0E816FE90E030144
:10107800F625D96E030EF721DA6EDF500101DA6F1B
:10108800DA510001826F836BC9EC59F00301F64B0A
:10109800F72BF7BFE6D7F75104E1040EF65DD8A0A9
:1010A800E0D75A0E0001806FFC0E816FC9EC59F031
:1010B800A80E0001806FFA0E816FC9EC59F022EE7C
:1010C80004F000EED8F01F0EDBCFEBFFE806FCE2E1
:1010D800D10E0001F86FFF0EF96F08EC35F0D8C09B
:1010E80058F1D9C059F1DAC05AF1DBC05BF10101FE
:1010F800585159115A115B11D8B481D08E0E000184
:10110800806FFA0E816F58C182F059C183F05AC1BD
:1011180084F05BC185F0C9EC59F0040E0001B16F91
:10112800020EB26F58C1DBF159C1DCF15AC1DDF1D1
:101138000101DA6B000EDA250001B36F010E01011F
:10114800DB210001B46F000E0101DC210001B56F45
:10115800000E0101DD210001B66F9FEC12F0040EB4
:101168008C6F020E8D6F340E8E6F0B0E8F6F000E0C
:10117800916F080E906FF30E926F030E936FA4ECAD
:1011880015F0000E0301F96F000EF86FF9BF06D0D5
:10119800F9511DE1080EF85DD8B019D0D50E00013F
:1011A800806FFF0E816F340E0301F825D96E0B0E88
:1011B800F921DA6EDF500101DA6FDA510001826F2E
:1011C800836BC9EC59F00301F84BF92BDFD734CB0B
:1011D800DAF10101DA510301E16FE26BE36BE46BD1
:1011E800520E0001806FFE0E816FE1C382F0E2C3F0
:1011F80083F0E3C384F0E4C385F0C9EC59F001013E
:10120800A8AF13D0946889928982150E0101DB6F0B
:101218004B0EDA6FBE0EE82EFED7DA2FFCD7DB2F87
:10122800FAD700F025EC40F0EED7E151D8B40CD055
:101238007A0E0001806FFD0E816FC9EC59F0020E25
:101248000101956F220E0BD06A0E0001806FFD0E12
:10125800816FC9EC59F0010E0101956F040E946F6E
:10126800000E0301F06F000EEF6F000EFD6F899EF8
:10127800000EFC6F010EFB6FFCBF08D0FC5105E1AE
:10128800040EFB5DD8B0E0D101D0DED1FBC30CF079
:10129800FCC30DF0000E0F6E0F0E0E6E23EC59F00E
:1012A800240E0C24126E0E0E0D20136EFBEC56F05D
:1012B800135004E1030E125CD8A04ED0FBC30CF00F
:1012C800FCC30DF0000E0F6E0F0E0E6E23EC59F0DE
:1012D800240E0C240301E76F0E0E0D20E86FDA0EC2
:1012E8000001806FFD0E816FE7C382F0E8C383F0D1
:1012F800C9EC59F0FBC3DAF1FCC3DBF1050ED89059
:101308000101DA37DB37E82EFAD7040EDA250001B7
:10131800D86F020E0101DB210001D96FFBC30CF06D
:10132800FCC30DF0000E0F6E0F0E0E6E23EC59F07D
:10133800240E0C240001DA6F0E0E0D20DB6F030E55
:10134800DC6F6FEC18F00101DC6FDC510301F16F09
:10135800F26BF1511FEC55F00301FB4BFC2B8CD7C2
:101368008450070B0101906F928A80AA03D0905194
:10137800080F906F9151D8B452D0A6519019D8B493
:101388004ED0898E000E0301EE6F000EED6F90C1F6
:10139800E5F3E66B680E0101DA6FE40EE82EFED77E
:1013A800DA2FFCD700F0FCEC58F0906F80AA03D03D
:1013B8009051080F906F9051DA6FDB6B0301E55184
:1013C8000101DA1909E10301E6510101DB19D8A489
:1013D80003D00301ED4BEE2B0301EEBFD8D7EE513E
:1013E80004E1650EED5DD8A0D2D790C1A6F1150E27
:1013F8000101DB6F4B0EDA6FBE0EE82EFED7DA2F37
:10140800FCD7DB2FFAD700F0490E0001806FFC0EE5
:10141800816FA6C182F0836BC9EC59F035D181A8E0
:10142800939419EC5AF00C500D10D8B40DD1FDC39B
:10143800F5F3FA0E0C6E030E0D6EFDEC51F0030180
:10144800FD6F3A0E0001806FFF0E816FFDC382F0C1
:10145800836B80A004D00101DA6BDA2B02D0010182
:10146800DA6BDA510001846F856BC9EC59F003011E
:10147800FAA94BD0600EFD19D8A447D05F0EF51914
:10148800D8A443D07B0E0001806FF90E816FFDC395
:1014980082F0836BF5C384F0856B81A204D00101CF
:1014A800DA6BDA2B02D00101DA6BDA510001866FB0
:1014B800876B81A404D00101DB6BDB2B02D0010117
:1014C800DB6BDB510001886F896BC9EC59F07250F6
:1014D8000209726E2BEE34F095C1DFFF2BEE35F06A
:1014E80094C1DFFF8984000E4A6E020E496E44ECF7
:1014F80036F089947250FD0B726E000E716E10EC0E
:1015080059F0000E0301FD6F9FD00101E151D8B4DD
:101518004AD00301FA51100B0001AC6F000EAD6FF9
:101528000301FD515FEC2FF0ACC0FEF3ADC0FFF33B
:10153800080E0301FE19FF11D8B400F0070E0301CD
:10154800FE19FF11D8B459EC53F00301FE05FF1141
:10155800D8B4B5EC51F0020E0301FE19FF11D8B44E
:101568001EEC3EF0030E0301FE19FF11D8A406D0AD
:101578004CEC2AF0EFC0EFF3F0C0F0F3050E0301D6
:10158800FE19FF11D8A406D078EC37F0FAC0EFF3B3
:10159800FBC0F0F3090E0301FE19FF11D8A454D0C3
:1015A8000BEC5AF051D00301FA51100B496E000EA2
:1015B8004A6EFD5112EC24F049C0FEF34AC0FFF315
:1015C800070E0301FE19FF11D8B449EC59F0020EB9
:1015D8000301FE19FF11D8B4BBEC54F00301FE055A
:1015E800FF11D8B403EC42F0030E0301FE19FF11FA
:1015F800D8B427EC47F0040E0301FE19FF11D8B444
:1016080093EC56F0050E0301FE19FF11D8B41CEC3B
:1016180045F0060E0301FE19FF11D8B4BDEC57F0D2
:10162800080E0301FE19FF11D8B4FFEC3BF0090EB8
:101638000301FE19FF11D8B42FEC5AF00A0EFE1957
:10164800FF11D8B46CEC4CF082B21ED0050E030129
:10165800EF19F011D8B418D083D68A0E0001806F24
:10166800FE0E816F82CF82F0836BC9EC59F0150EA4
:101678000101DB6F4B0EDA6FBE0EE82EFED7DA2FB4
:10168800FCD7DB2FFAD700F082B2E7D7150E01019D
:10169800DB6F4B0EDA6FBE0EE82EFED7DA2FFCD7C3
:1016A800DB2FFAD700F0000E03EC5AF001018D6F22
:1016B8005D0E0001806FFC0E816F8DC182F0836B1F
:1016C800C9EC59F0150E0101DB6F4B0EDA6FBE0E37
:1016D800E82EFED7DA2FFCD7DB2FFAD700F0899453
:1016E8008992000E0001D86F000ED96F5C0EDA6F78
:1016F800FC0EDB6F000EDC6F24EC50F092D4666EAB
:10170800000E656E17D36650D8A419D00001FC519D
:10171800D8B415D0E10E806FFB0E816FCFCF82F069
:10172800836BCECF84F0856BC9EC59F0000E656EE3
:10173800000E0101736F0A0E62D089906DD3020EFC
:101748006618D8A417D00001FC51D8B413D06E0E77
:10175800806FFB0E816FCFCF82F0836BCECF84F08A
:10176800856BC9EC59F0000E656E000E0101736FB0
:10177800140E45D01F0E666444D0300E666041D00A
:101788000001FC51D8B43DD06650E00F6E6EB60E25
:10179800806FF90E816FCFCF82F0836BCECF84F04C
:1017A800856B6EC086F0876BC9EC59F0000E656ECC
:1017B8006E50200D0E0EF324D96E020EF420DA6E50
:1017C800DE50DE10DE10DE10D8B403D0030E6E64D7
:1017D80048D0010E6D6E6E50140D130EF324D96EA1
:1017E800010EF420DA6E6E50140D130EF324E16E20
:1017F800010EF420E26EE7500409DF6E32D0726FFA
:101808009CD73F0E666432D0500E66602FD0000120
:10181800FC51D8B42BD06E50140D000EF324D96EA1
:10182800010EF420DA6E6650C00FDF6E010E806F75
:10183800F90E816FCFCF82F0836BCECF84F0856BAA
:101848006E50140D000EF324D96E010EF420DA6EDA
:10185800DF50496E4950866F876BC9EC59F0000E0E
:10186800656E000E0101736F000EC9D7340E66183D
:10187800D8A417D00001FC51D8B413D00C0E806F37
:10188800FC0E816FCFCF82F0836BCECF84F0856B57
:10189800C9EC59F0000E0101736F000E726F000E53
:1018A80047D2350E6618D8A417D00001FC51D8B419
:1018B80013D05A0E806FFA0E816FCFCF82F0836BF0
:1018C800CECF84F0856BC9EC59F0000E656E0D0E15
:1018D8000101736FAC0E93D7370E6618D8A409D0E0
:1018E8000001FC51D8B405D00E0E0101736F750EBE
:1018F8000AD20D0E6618D8A41AD00001FC51D8B42B
:1019080016D0000E656E020E0101736FBC0E726F69
:101918008990250E0001806FFA0E816FCFCF82F07B
:10192800836BCECF84F0856BC9EC59F075D2100E5D
:101938006618D8A409D00001FC51D8B405D0030E0C
:101948000101736FE90EDFD1180E6618D8A409D00B
:101958000001FC51D8B405D0070E0101736F090EC0
:10196800D2D13E0E6618D8A409D00001FC51D8B4D3
:1019780005D00F0E0101736F3D0EC5D1D30E0001C6
:10198800806FF90E816FCFCF82F0836BCECF84F05A
:10199800856B66C086F0876BC9EC59F03DD26E50F6
:1019A800140D010EF324D96E010EF420DA6E66C010
:1019B800DFFF030E0101736FEA0EA5D16E50140DFF
:1019C800020EF324D96E010EF420DA6E66C0DFFF32
:1019D800030E0101736FEB0E96D16E50140D030EBA
:1019E800F324D96E010EF420DA6E66C0DFFF030E11
:1019F8000101736FEC0E87D16E50140D040EF324A1
:101A0800D96E010EF420DA6E66C0DFFF030E010105
:101A1800736FED0E78D16E50140D050EF324D96E48
:101A2800010EF420DA6E66C0DFFF030E0101736F4A
:101A3800EE0E69D16E50140D060EF324D96E010E08
:101A4800F420DA6E66C0DFFF6E50140D060EF32424
:101A5800D96E010EF420DA6EDF50496E49C04AF0A3
:101A68004B6A4C6A4D6A4CC04DF04BC04CF04AC0B2
:101A78004BF04A6A6E50140D050EF324D96E010E10
:101A8800F420DA6EDF504E6E4EC04FF0506A516A45
:101A9800526A50C052F04FC051F0506A4F6A6E50AF
:101AA800140D040EF324D96E010EF420DA6EDF5003
:101AB800536E53C054F0556A566A576A54C057F06B
:101AC800566A556A546A6E50140D030EF324D96E83
:101AD800010EF420DA6EDF50586E58505424596EB7
:101AE800000E55205A6E000E56205B6E000E5720D1
:101AF8005C6E4F5059245D6E50505A205E6E5150A6
:101B08005B205F6E52505C20606E4A505D24616EAF
:101B18004B505E20626E4C505F20636E4D506020CB
:101B2800646E6E50140D070EF324D96E010EF42066
:101B3800DA6E61C0DEFF62C0DEFF63C0DEFF64C034
:101B4800DEFF1E0E0001806FF80E816FCFCF82F08E
:101B5800836BCECF84F0856B6E50140D070EF32483
:101B6800D96E010EF420DA6EDECF86F0DECF87F074
:101B7800DECF88F0DECF89F0C9EC59F0000E010104
:101B8800736F000EC0D06E50140D120EF324D96E70
:101B9800010EF420DA6E66C0DFFF070E0101736FD5
:101BA8000A0EB1D06E50140D110EF324D96E010E29
:101BB800F420DA6E66C0DFFF070E0101736F0B0EAB
:101BC800A2D06E50140D100EF324D96E010EF4201D
:101BD800DA6E66C0DFFF070E0101736F0C0E93D03B
:101BE8006E50140D0F0EF324D96E010EF420DA6E28
:101BF80066C0DFFFC10E0001806FF80E816FCFCF86
:101C080082F0836BCECF84F0856B6E50140D0F0E6F
:101C1800F324D96E010EF420DA6EDECF86F0DECF23
:101C280087F0DECF88F0DECF89F0C9EC59F0A6D76F
:101C380066C050F10F0E0101736F3E0E64D066C08E
:101C480051F10F0E0101736F3F0E5DD066C052F166
:101C58000F0E0101736F400E56D066C053F10F0E80
:101C68000101736F410E4FD066C054F10F0E010190
:101C7800736F420E48D066C055F10F0E0101736FA5
:101C8800430E41D066C056F10F0E0101736F440E2A
:101C98003AD066C057F1160E0001806FF60E816FBC
:101CA800CFCF82F0836BCECF84F0856B50C186F0A6
:101CB800876B51C188F0896B52C18AF08B6B53C115
:101CC8008CF08D6B54C18EF08F6B55C190F0916B79
:101CD80056C192F0936B57C194F0956BC9EC59F0CB
:101CE8004DD70C0E0001806FFC0E816FCFCF82F0B4
:101CF800836BCECF84F0856BC9EC59F03FD70E0EBD
:101D08000101736F760E726F87D00A0E0001806F23
:101D1800FA0E816FCFCF82F0836BCECF84F0856BC4
:101D2800C9EC59F0000E0101736F000E726F090EB5
:101D3800656E03D572C149F073C14AF04A50000A72
:101D4800D8B416D0030AD8B418D0040AD8B429D005
:101D58000A0AD8B434D0030AD8B437D0010AD8B4A0
:101D68003CD0130AD8B453D03B0AD8B453D054D07B
:101D78004950000AD8B4C7D44FD04950E90AD8B45A
:101D88000ED6030AD8B41AD6010AD8B426D6070A3A
:101D9800D8B432D6010AD8B43ED6030AD8B44AD643
:101DA8003BD04950090AD8B4EED6030AD8B4FAD6BB
:101DB800010AD8B406D7070AD8B412D72DD049508B
:101DC800480AD8B48ED7E40A27D04950750AD8B43F
:101DD80096D7030AD8B499D71FD049503D0AD8B42A
:101DE80027D7030AD8B42BD7010AD8B42FD77F0A2C
:101DF800D8B433D7010AD8B437D7030AD8B43BD7F5
:101E0800010AD8B43FD7070AD8B443D705D04950F8
:101E18002A0A02D049500F0A65501200B3C0C5F013
:101E2800B4C0C6F0B751D96EDA6A000EDE6E000E85
:101E3800DD6EB1C00DF0B2C00EF06BEC51F00001D8
:101E4800C46FC451D8B402D0C451120020EE05F0BA
:101E5800B151D926B251DA22DF50D8B408D020EED9
:101E680005F0B151D926B251DA22DF50120020EE26
:101E780004F0B151D926B251DA22DFB202D0070EEE
:101E8800120020EE06F0B151D926B251DA2210EE36
:101E980006F0B151E126B251E222E6CFBCF0E6CF1E
:101EA800BDF0E6CFBEF0E6CFBFF0B551BC25C06FA0
:101EB800B651BD21C16F000EBE21C26F000EBF21F9
:101EC800C36FDE50C05DDE50C159DE50C259DE50CE
:101ED800C359D8B0F8D2000EB66F000EB56FF3D262
:101EE80020EE06F0B151D926B251DA22FF0EDE14E7
:101EF800B86F010EDE14B96F000EDE14BA6F000E53
:101F0800DE14BB6FB851B911BA11BB11D8A443D2B2
:101F180020EE06F0B151D926B251DA22DECFB8F060
:101F2800DECFB9F0DECFBAF0DECFBBF00A0E05D0B7
:101F3800D890BB33BA33B933B833E82EF9D7B1C028
:101F4800D9FFB2C0DAFF10EE02F0DE50E126DD5014
:101F5800E222E750BC6FBC05B815C76FC751D8A4BB
:101F6800A4D020EE06F0B151D926B251DA22DE50C3
:101F7800DE10DE10DE10D8A427D020EE0EF0B1510E
:101F8800D926B251DA22DECFCEF0DECFCFF0DECFC7
:101F9800D0F0DECFD1F0CE51CF11D011D111D8A4CD
:101FA80033D0B1C0D9FFB2C0DAFFDECF9EF0DDCFAB
:101FB8009FF0000EA06F000EA16F000EA26F000E22
:101FC800A36FE3EC2DF018D0B1C0D9FFB2C0DAFF8F
:101FD800DECF9EF0DDCF9FF020EE12F0B151D92672
:101FE800B251DA22DECFA0F0DECFA1F0DECFA2F030
:101FF800DECFA3F0E3EC2DF09EC0CEF09FC0CFF073
:10200800A0C0D0F0A1C0D1F0CE51CF11D011D111C4
:10201800D8B45DD2CE05CF11D011D111D8A40AD031
:1020280020EE05F0B151D926B251DA22020EDF6E48
:10203800020E1200CE2911E1CF290FE1D0290DE1BE
:10204800D129D8A40AD020EE05F0B151D926B25131
:10205800DA22010EDF6E010E120020EE12F0B151ED
:10206800D926B251DA22CEC0DEFFCFC0DEFFD0C003
:10207800DEFFD1C0DEFF20EE0EF0B151D926B251FD
:10208800DA22DE50DE10DE10DE10D8A40ED020EEEC
:102098000EF0B151D926B251DA22CEC0DEFFCFC040
:1020A800DEFFD0C0DEFFD1C0DEFF20EE16F0B1515A
:1020B800D926B251DA22B1C0E1FFB2C0E2FF00EE88
:1020C8002AF0E650E926E550EA22DE50EE1817E13C
:1020D800DE50EE1814E1DE50EE1811E1DE50EE1875
:1020E800D8A40DD0B1C0D9FFB2C0DAFFDECF25F039
:1020F800DDCF26F07BEC46F00009D8A48BD1B1C027
:10210800D9FFB2C0DAFFDECF18F0DDCF19F0000139
:1021180020EE12F0B151D926B251DA22DECF1AF0F0
:10212800DECF1BF0DECF1CF0DECF1DF06FEC4FF0E2
:1021380018C0CAF019C0CBF01AC0CCF01BC0CDF043
:102148000001CA51CB11CC11CD11D8B469D7C751F0
:10215800CA27000ECB23CC23CD23B5C0B8F0B6C018
:10216800B9F0090EBA6FD890B933B833BA2FFBD784
:10217800B8C0C8F0B9C0C9F0C851C911D8B4C7D0DF
:10218800C751C825B86F000EC921B96FB1C0D9FFB2
:10219800B2C0DAFF10EE02F0DE50E126DD50E22296
:1021A800E750BA6FBB6BB851BA5DB951BB59D8B0DB
:1021B80012D0B1C0D9FFB2C0DAFF10EE02F0DE5083
:1021C800E126DD50E222E750B86FC751B85DC86F0D
:1021D800C96BD8A0C907C5C01BF0C6C01CF0CAC0CF
:1021E8001DF0CBC01EF0CCC01FF0CDC020F0C8C081
:1021F80021F0C9C022F0B1C0D9FFB2C0DAFF10EE99
:1022080001F0DE50E126DD50E222E75065EC4BF0AC
:102218000009D8A4FFD00001C851B86FC951B96FDF
:10222800BA6BBB6BB1C0D9FFB2C0DAFF10EE2AF0AF
:10223800DE50E126DD50E222E6CFBCF0E6CFBDF06D
:10224800E6CFBEF0E6CFBFF0CA51BC5DC06FCB5140
:10225800BD59C16FCC51BE59C26FCD51BF59C36F63
:10226800B851C05DB951C159BA51C259BB51C359CE
:10227800D8B03ED0B1C0D9FFB2C0DAFFDECFB8F0D7
:10228800DDCFB9F02E0EB8250C6E000EB9210D6EFB
:10229800B1C0D9FFB2C0DAFF10EE2AF0DE50E12655
:1022A800DD50E222E6CFBAF0E5CFBBF0CA51BA5F03
:1022B800CB51BB5B090ED890BA37BB37E82EFBD79A
:1022C800BA51C5250E6EBB51C6210F6E020E116E96
:1022D800000E106E5FEC57F0B1C0D9FFB2C0DAFF44
:1022E80010EE04F0DE50E126DD50E222000EE76E2B
:1022F800C8C0B8F0C9C0B9F0090ED890B837B93716
:10230800E82EFBD7B8C0D2F0B9C0D3F0C0D020EEC9
:102318000AF0B151D926B251DA2210EE06F0B151C5
:10232800E126B251E222DE50E65CDE50E658DE508D
:10233800E658DE50E658D8A01FD0B1C0D9FFB2C0C9
:10234800DAFFDECF25F0DDCF26F07BEC46F0000982
:10235800D8A460D0B1C0D9FFB2C0DAFF10EE2AF01D
:10236800DE50E126DD50E222CAC0E6FFCBC0E6FF20
:10237800CCC0E6FFCDC0E6FF000120EE16F0B1515B
:10238800D926B251DA22CAC0DEFFCBC0DEFFCCC0EC
:10239800DEFFCDC0DEFFFF0EB86F010EB96F20EE75
:1023A80006F0B151D926B251DA22DECFBAF0DDCF2C
:1023B800BBF0B851BA17B951BB17BA510008D26F60
:1023C800BB51D8A0E82A0208D36FD251B55DD351CA
:1023D800B659D8B004D0B5C0D2F0B6C0D3F0B1C0A9
:1023E800D9FFB2C0DAFFDECF3AF0DDCF3BF020EE06
:1023F80016F0B151D926B251DA22DECF3CF0DECF49
:102408003DF0DECF3EF0DECF3FF078EC50F0000933
:10241800D8B402D0000117D6FF0E0001B86F010E24
:10242800B96F20EE06F0B151D926B251DA22DECFCB
:10243800BAF0DDCFBBF0B851BA17B951BB17B1C06C
:10244800D9FFB2C0DAFFDECFBCF0DDCFBDF0BA51A4
:10245800BC27BB51BD232E0EBC250C6E000EBD2122
:102468000D6EC5C00EF0C6C00FF0D2C010F0D3C0BC
:1024780011F05FEC57F0B1C0D9FFB2C0DAFF10EE2F
:1024880004F0DE50E126DD50E222010EE76ED25163
:10249800C527D351C62320EE06F0B151D926B25133
:1024A800DA22D251DE26D351DE22000EDE22DE22CF
:1024B800B751D96EDA6AD251DE26D351DD22D25114
:1024C800B55FD351B65BB551B611D8A409D520EE86
:1024D80006F0B151D926B251DA2210EE0AF0B15104
:1024E800E126B251E222DE50E65CDE50E658DE50CC
:1024F800E658DE50E658D8B014D020EE06F0B151B8
:10250800D926B251DA2210EE0AF0B151E126B251C1
:10251800E222DECFE6FFDECFE6FFDECFE6FFDECF4C
:10252800E6FF20EE04F0B151D926B251DA22000EAE
:10253800DB8A000E1200B1C00DF0B2C00EF06BECD9
:1025480051F00001CB6FCB51D8B402D0CB5112005F
:1025580020EE05F0B151D926B251DA22DF50D8B4B5
:1025680008D020EE05F0B151D926B251DA22DF5059
:10257800120020EE0AF0B151D926B251DA22B35135
:10258800DE5CB451DE58B551DE58B651DE58D8B0CD
:1025980016D020EE04F0B151D926B251DA22DFB2BA
:1025A8000ED020EE0AF0B151D926B251DA22DECF90
:1025B800B3F0DECFB4F0DECFB5F0DECFB6F020EE6C
:1025C80006F0B151D926B251DA22DECFC7F0DECFFC
:1025D800C8F0DECFC9F0DECFCAF0000ECC6F000E17
:1025E800CD6F000ECE6F000ECF6F20EE06F0B1510A
:1025F800D926B251DA22CCC0DEFFCDC0DEFFCEC074
:10260800DEFFCFC0DEFFB351B411B511B611D8B497
:102618002BD2B1C0D9FFB2C0DAFF10EE02F0DE5003
:10262800E126DD50E222E750B76FB7C0B8F0B96BCA
:10263800BA6BBB6B090ED890B837B937BA37BB3706
:10264800E82EF9D7B8C0D0F0B9C0D1F0BAC0D2F0EE
:10265800BBC0D3F0C751C811C911CA11D8B497D09B
:10266800FF0EB3250C6EFF0EB4210D6EFF0EB521C3
:102678000E6EFF0EB6210F6ED0C010F0D1C011F053
:10268800D2C012F0D3C013F09AEC53F00CC0B7F0DC
:102698000DC0B8F00EC0B9F00FC0BAF0FF0E0001BF
:1026A800C7250C6EFF0EC8210D6EFF0EC9210E6ED8
:1026B800FF0ECA210F6ED0C010F0D1C011F0D2C0E9
:1026C80012F0D3C013F09AEC53F00C500001B75D30
:1026D8000D50B8590E50B9590F50BA59D8A057D003
:1026E800FF0ED025B76FFF0ED121B86FFF0ED22194
:1026F800B96FFF0ED321BA6FB71DBB6FB81DBC6F82
:10270800B91DBD6FBA1DBE6FFF0EC725BF6FFF0E87
:10271800C821C06FFF0EC921C16FFF0ECA21C26F49
:10272800BB51BF15C36FBC51C015C46FBD51C11596
:10273800C56FBE51C215C66F20EE06F0B151D9263D
:10274800B251DA22C3C0DEFFC4C0DEFFC5C0DEFF5F
:10275800C6C0DEFF20EE06F0B151D926B251DA220A
:10276800DE50B35FDE50B45BDE50B55BDD50B65B68
:1027780020EE12F0B151D926B251DA22DECFD4F0D0
:10278800DECFD5F0DECFD6F0DECFD7F06DD020EE9D
:102798000EF0B151D926B251DA22DECFD4F0DECF15
:1027A800D5F0DECFD6F0DECFD7F0D451D511D61183
:1027B800D711D8A44BD0B1C0D9FFB2C0DAFFDECF51
:1027C8009EF0DDCF9FF0000EA06F000EA16F000EEF
:1027D800A26F000EA36FE3EC2DF09EC0D4F09FC053
:1027E800D5F0A0C0D6F0A1C0D7F0D405D511D61128
:1027F800D711D8A40AD020EE05F0B151D926B2518C
:10280800DA22020EDF6E020E1200D42911E1D52958
:102818000FE1D6290DE1D729D8A40AD020EE05F07A
:10282800B151D926B251DA22010EDF6E010E120023
:1028380020EE0EF0B151D926B251DA22D4C0DEFF13
:10284800D5C0DEFFD6C0DEFFD7C0DEFF20EE12F017
:10285800B151D926B251DA22D4C0DEFFD5C0DEFF8D
:10286800D6C0DEFFD7C0DEFFD451D511D611D7119F
:10287800D8A496D0F9D020EE04F0B151D926B2519F
:10288800DA22DFA229D0B1C0D9FFB2C0DAFFDECF89
:102898009EF0DDCF9FF0D4C0A0F0D5C0A1F0D6C087
:1028A800A2F0D7C0A3F0E3EC2DF09EC0D4F09FC0F7
:1028B800D5F0A0C0D6F0A1C0D7F0D451D511D6110B
:1028C800D711D8A423D0D0C0B3F0D1C0B4F0D2C0AF
:1028D800B5F0D3C0B6F06ED0B1C0D9FFB2C0DAFF40
:1028E800DECF45F0DDCF46F0D4C047F0D5C048F084
:1028F800D6C049F0D7C04AF0E3EC21F045C0D4F087
:1029080046C0D5F047C0D6F048C0D7F00001D4295A
:1029180007E1D52905E1D62903E1D729D8B47ED71F
:10292800D751D611D51104E1020ED45DD8A063D7D2
:10293800B1C0D9FFB2C0DAFF10EE12F0DE50E126C6
:10294800DD50E222E650D45DE650D559E650D6591E
:10295800E650D759D8B04FD720EE12F0B151D9264A
:10296800B251DA22D4C0DEFFD5C0DEFFD6C0DEFF0A
:10297800D7C0DEFF20EE06F0B151D926B251DA22D7
:10298800D051DE26D151DE22D251DE22D351DE22B1
:10299800D051B35FD151B45BD251B55BD351B65B63
:1029A800B351D05DB451D159B551D259B651D3595B
:1029B800D8A061D720EE06F0B151D926B251DA225B
:1029C800B351DE26B451DE22B551DE22B651DE22E5
:1029D800FF0EB315B76F010EB415B86F000EB5151D
:1029E800B96F000EB615BA6FB751B811B911BA114F
:1029F800D8B43AD0B1C0D9FFB2C0DAFFDECF18F0F0
:102A0800DDCF19F0D4C01AF0D5C01BF0D6C01CF029
:102A1800D7C01DF06FEC4FF018C0CCF019C0CDF046
:102A28001AC0CEF01BC0CFF00001CC51CD11CE1191
:102A3800CF11D8B4E0D6B3C0B7F0B4C0B8F0B5C0C1
:102A4800B9F0B6C0BAF00A0E05D0D890BA33B93387
:102A5800B833B733E82EF9D7B751CC27B851CD23BF
:102A6800B951CE23BA51CF2320EE06F0B151D92661
:102A7800B251DA22FF0EDE14B76F010EDE14B86F02
:102A8800000EDE14B96F000EDE14BA6FB751B8111C
:102A9800B911BA11D8B421D020EE16F0B151D92607
:102AA800B251DA22CC51DE180AE1CD51DE1807E125
:102AB800CE51DE1804E1CF51DE18D8B40ED020EE86
:102AC80016F0B151D926B251DA22CCC0DEFFCDC002
:102AD800DEFFCEC0DEFFCFC0DEFF20EE06F0B15134
:102AE800D926B251DA2210EE0AF0B151E126B251DC
:102AF800E222DE50E65CDE50E658DE50E658DE5054
:102B0800E658D8B023D520EE06F0B151D926B251F7
:102B1800DA2210EE0AF0B151E126B251E222DECFFC
:102B2800E6FFDECFE6FFDECFE6FFDECFE6FF20EEF4
:102B380004F0B151D926B251DA22000EDB8A06D54B
:102B48008EC0A9F08FC0AAF092C0D9FF93C0DAFF57
:102B5800000EDE6E000EDD6E8CC00DF08DC00EF026
:102B68006BEC51F00001A46FA451D8B402D0A45169
:102B7800120020EE05F08C51D9268D51DA22DF5053
:102B8800D8B408D020EE05F08C51D9268D51DA2220
:102B9800DF50120020EE04F08C51D9268D51DA2234
:102BA800DFB002D0070E120020EE06F08C51D926B5
:102BB8008D51DA22DECF94F0DECF95F0DECF96F09D
:102BC800DECF97F020EE0AF08C51D9268D51DA220B
:102BD800DECF98F0DECF99F0DECF9AF0DECF9BF013
:102BE8009451985DA06F95519959A16F96519A5932
:102BF800A26F97519B59A36F9051946F9151956F04
:102C0800966B976B9451A05D9551A1599651A25915
:102C18009751A359D8B059D2A0C090F0A1C091F053
:102C280054D220EE06F08C51D9268D51DA22FF0EAF
:102C3800DE14946F010EDE14956F000EDE14966F8D
:102C4800000EDE14976F9451951196119711D8A420
:102C5800AFD120EE06F08C51D9268D51DA22DECF85
:102C680094F0DECF95F0DECF96F0DECF97F00A0E27
:102C780005D0D8909733963395339433E82EF9D707
:102C88008CC0D9FF8DC0DAFF10EE02F0DE50E126CD
:102C9800DD50E222E750986F98059415AB6FAB5161
:102CA800D8A46FD020EE06F08C51D9268D51DA22A7
:102CB800DE50DE10DE10DE10D8A40FD020EE0EF0AD
:102CC8008C51D9268D51DA22DECFA5F0DECFA6F0C1
:102CD800DECFA7F0DECFA8F020D08CC0D9FF8DC002
:102CE800DAFFDECF45F0DDCF46F020EE12F08C5152
:102CF800D9268D51DA22DECF47F0DECF48F0DECF7D
:102D080049F0DECF4AF0E3EC21F045C0A5F046C01B
:102D1800A6F047C0A7F048C0A8F00001A851A71125
:102D2800A6110EE1020EA55DD8B00AD020EE05F07E
:102D38008C51D9268D51DA22020EDF6E020E120056
:102D4800A52911E1A6290FE1A7290DE1A829D8A4F1
:102D58000AD020EE05F08C51D9268D51DA22010EC9
:102D6800DF6E010E120020EE12F08C51D9268D5123
:102D7800DA22A5C0DEFFA6C0DEFFA7C0DEFFA8C01E
:102D8800DEFF8CC0D9FF8DC0DAFFDECF18F0DDCFB3
:102D980019F020EE12F08C51D9268D51DA22DECFAF
:102DA8001AF0DECF1BF0DECF1CF0DECF1DF06FEC8B
:102DB8004FF018C0ACF019C0ADF01AC0AEF01BC08F
:102DC800AFF00001AC51AD11AE11AF11D8B4AED710
:102DD800AB51AC27000EAD23AE23AF2390C094F0C7
:102DE80091C095F0090E966FD89095339433962F2D
:102DF800FBD794C0B0F095C0B1F0B051B111D8B4C0
:102E0800C9D0AB51B025946F000EB121956F8CC01D
:102E1800D9FF8DC0DAFF10EE02F0DE50E126DD505A
:102E2800E222E750966F976B9451965D95519759AA
:102E3800D8B012D08CC0D9FF8DC0DAFF10EE02F0E6
:102E4800DE50E126DD50E222E750946FAB51945DED
:102E5800B06FB16BD8A0B107A9C01BF0AAC01CF015
:102E6800ACC01DF0ADC01EF0AEC01FF0AFC020F06A
:102E7800B0C021F0B1C022F08CC0D9FF8DC0DAFFFC
:102E880010EE01F0DE50E126DD50E222E750A8EC1A
:102E98004EF00009D8A4CBD08CC0D9FF8DC0DAFF82
:102EA80010EE04F0DE50E126DD50E222E750D8B4FF
:102EB80061D00001B051946FB151956F966B976BCB
:102EC8008CC0D9FF8DC0DAFF10EE2AF0DE50E12663
:102ED800DD50E222E6CF98F0E6CF99F0E6CF9AF0FF
:102EE800E6CF9BF0AC51985D9C6FAD5199599D6FA1
:102EF800AE519A599E6FAF519B599F6F94519C5DEB
:102F080095519D5996519E5997519F59D8B032D095
:102F18008CC0D9FF8DC0DAFF10EE2AF0DE50E12612
:102F2800DD50E222E6CF94F0E5CF95F0AC51945F06
:102F3800AD51955B090ED89094379537E82EFBD79D
:102F48009451A9250C6E9551AA210D6E8CC0D9FFFC
:102F58008DC0DAFFDECF96F0DDCF97F02E0E9625E6
:102F68000E6E000E97210F6E020E116E000E106E7F
:102F78005FEC57F0B0C094F0B1C095F0090ED8904E
:102F8800000194379537E82EFAD794C0B2F095C06F
:102F9800B3F07ED020EE16F08C51D9268D51DA226E
:102FA800ACC0DEFFADC0DEFFAEC0DEFFAFC0DEFFEF
:102FB800FF0E946F010E956F20EE06F08C51D92606
:102FC8008D51DA22DECF96F0DDCF97F09451961727
:102FD8009551971796510008B26F9751D8A0E82AD3
:102FE8000208B36FB251905DB3519159D8B004D073
:102FF80090C0B2F091C0B3F08CC0D9FF8DC0DAFF99
:10300800DECF3AF0DDCF3BF020EE16F08C51D9261A
:103018008D51DA22DECF3CF0DECF3DF0DECF3EF040
:10302800DECF3FF078EC50F00009D8B402D00001B0
:1030380090D6A9C00CF0AAC00DF0FF0E0001946F45
:10304800010E956F20EE06F08C51D9268D51DA22AB
:10305800DECF96F0DDCF97F09451961795519717DC
:103068008CC0D9FF8DC0DAFFDECF98F0DDCF99F0A4
:1030780096519827975199232E0E98250E6E000E7B
:1030880099210F6EB2C010F0B3C011F05FEC57F089
:10309800B251A927B351AA2320EE06F08C51D926A4
:1030A8008D51DA22B251DE26B351DE22000EDE2225
:1030B800DE2292C0D9FF93C0DAFFB251DE26B351A7
:1030C800DD22B251905FB351915B90519111D8A418
:1030D800A8D5000E1200D851D911D8A402D0090ED3
:1030E8001200D8C0D9FFD9C0DAFF000EDE6E000E7C
:1030F800DD6E82C1C0F183C1C1F11F0EDC17C00EA5
:10310800806F010E816FDA0E826FDC51FE0B836FC8
:1031180009EC00F00101BD6FBD51D8A45BD2A90E26
:10312800D46F010ED56FC00E0001CA6F010ECB6FB0
:10313800DAC0CCF0DBC0CDF0E6EC42F00101BD6FA7
:10314800D2C1BEF1D3C1BFF1BD51D8A406D0BE5182
:10315800BF11D8A402D0060EBD6FDCC0DDF01C0E76
:103168000001DD17D8B426D10101BD51D8B414D05F
:10317800040EBD19D8A409D0C00E0001CE6F010EEF
:10318800CF6F40EC4EF00101BD6F0001DC87D2C16A
:10319800BEF1D3C1BFF114D020EE0BF0BE51D92639
:1031A800BF51DA22DF500001DD6F110EDD17D8B4F0
:1031B80002D0070E03D0DCA503D0080E0101BD6FB5
:1031C8000101BD51D8A412D10001DCA70FD1000E16
:1031D8000101B96F000EBA6F210EBB6F460EBC6FAE
:1031E80020EE0EF0BE51D926BF51DA22000EDF6E56
:1031F80020EE0FF0BE51D926BF51DA22BAC1DFFF47
:1032080020EE10F0BE51D926BF51DA22BBC1DFFF34
:1032180020EE11F0BE51D926BF51DA22BCC1DFFF22
:1032280020EE16F0BE51D926BF51DA22000EDF6E0D
:1032380020EE17F0BE51D926BF51DA22BAC1DFFFFE
:1032480020EE18F0BE51D926BF51DA22BBC1DFFFEC
:1032580020EE19F0BE51D926BF51DA22BCC1DFFFDA
:1032680020EE0BF0BE51D926BF51DA22000EDF6ED8
:1032780020EE1CF0BE51D926BF51DA22000EDF6EB7
:1032880020EE1DF0BE51D926BF51DA22000EDF6EA6
:1032980020EE1EF0BE51D926BF51DA22000EDF6E95
:1032A80020EE1FF0BE51D926BF51DA22000EDF6E84
:1032B800C0C10CF0C1C10DF0BEC10EF0BFC10FF00E
:1032C8000DEC4FF00CC0B5F10DC0B6F10EC0B7F162
:1032D8000FC0B8F1BEC10CF0BFC10DF0000E0E6EEC
:1032E800000E0F6E000E106E000E116E1DEC57F0E2
:1032F800010120EE04F0C051D926C151DA22010E95
:10330800DF6EB551B611B711B811D8B46FD020EE31
:103318002AF0C051D926C151DA22DECFB9F1DECF69
:10332800BAF1DECFBBF1DECFBCF1C0C19EF0C1C1A6
:103338009FF0B5C1A0F0B6C1A1F0B7C1A2F0B8C165
:10334800A3F0CDEC47F00101BD6FBD51D8A44ED01C
:10335800FF0EB5250001DD6FFF0E0101B62100014A
:10336800DE6FFF0E0101B7210001DF6FFF0E0101C3
:10337800B8210001E06F010120EE0AF0C051D92602
:10338800C151DA22DDC0DEFFDEC0DEFFDFC0DEFFB6
:10339800E0C0DEFFC0C13AF0C1C13BF0B9C13CF0AA
:1033A800BAC13DF0BBC13EF0BCC13FF078EC50F073
:1033B80001011BD00101BD51D8A418D020EE0BF09B
:1033C800BE51D926BF51DA22DFA802D0040E0DD093
:1033D8000001DCA30BD0010120EE0BF0BE51D92671
:1033E800BF51DA22DFA002D0070EBD6F0101BD5127
:1033F800D8A423D00001DCB7DC8B010120EE2AF031
:10340800C051D926C151DA22000110EE1AF0D85164
:10341800E126D951E222DECFE6FFDECFE6FFDECF9E
:10342800E6FFDECFE6FF20EE1EF0D851D926D951AF
:10343800DA22BEC1DEFFBFC1DDFF0101BD51D8A444
:10344800C9D0000120EE04F0D851D926D951DA228A
:10345800DCC0DFFF20EE05F0D851D926D951DA2299
:10346800000EDF6EC0C10CF0C1C10DF0BEC10EF080
:10347800BFC10FF00DEC4FF0000120EE0EF0D85157
:10348800D926D951DA220CC0DEFF0DC0DEFF0EC0EE
:10349800DEFF0FC0DEFF010120EE1DF0BE51D92670
:1034A800BF51DA22DF500001DD6FDD51DF6FDE6BC7
:1034B800010120EE1EF0BE51D926BF51DA22DF509D
:1034C8000001E06FE0C0E1F0E26BE36BE46BE2C0A7
:1034D800E4F0E1C0E3F0E26BE16B010120EE1FF0E4
:1034E800BE51D926BF51DA22DF500001E56FE5C091
:1034F800E6F0E76BE86BE96BE6C0E9F0E86BE76BD1
:10350800E66BE151E611EA6FE251E711EB6FE35127
:10351800E811EC6FE451E911ED6FDE51EA11EE6F3D
:10352800DF51EB11EF6F000EEC11F06F000EED1193
:10353800F16F010120EE1CF0BE51D926BF51DA22ED
:10354800DF500001F26FF251EE11F36FEF51F46F9B
:10355800F051F56FF151F66F20EE0AF0D851D926E7
:10356800D951DA22F3C0DEFFF4C0DEFFF5C0DEFF7A
:10357800F6C0DEFF20EE06F0D851D926D951DA225E
:10358800DE6ADE6ADE6ADD6A20EE16F0D851D926D8
:10359800D951DA22DE6ADE6ADE6ADD6AD8C0D9FF6E
:1035A800D9C0DAFFC0C1DEFFC1C1DDFFD8C0D9FF75
:1035B800D9C0DAFF10EE06F0DE50E126DD50E22237
:1035C80020EE02F0D851D926D951DA22E6CFDEFF13
:1035D800E5CFDDFF0101BD5112004A5049104810E6
:1035E80004E1020E475CD8A010D020EE12F045503E
:1035F800D9264650DA22DE50475CDE504858DE5065
:103608004958DE504A58D8A03FD2020E556E52D2C1
:1036180047C053F048C054F0D8905430816F5330AD
:10362800806F805153268151542245C03AF046C0DC
:103638003BF020EE1EF04550D9264650DA22DECF68
:1036480080F0DECF81F0DECF82F0DECF83F053C092
:1036580084F054C085F0090E866FD8908533843382
:10366800862FFBD7845180253C6E855181213D6E84
:10367800000E82213E6E000E83213F6E78EC50F0E2
:10368800556E5550D8A416D2FF0E0001806F010E5A
:10369800816F53C082F054C083F0805182178151EA
:1036A800831745C084F046C085F082518427835132
:1036B80085232E0E8425566E000E8521576E534A9B
:1036C800542A47B004D04BC04FF0506A1AD04B5020
:1036D800806F816B803B813BF00E811780510F0B0F
:1036E8008113F00E801756C0D9FF57C0DAFFDF509C
:1036F8000F0B826F836B805182114F6E8151831142
:10370800506E56C0D9FF57C0DAFF4FC0DFFF20EE1A
:1037180004F04550D9264650DA22010EDF6E45C026
:103728003AF046C03BF020EE1EF04550D9264650F0
:10373800DA22DECF80F0DECF81F0DECF82F0DECF7E
:1037480083F053C084F054C085F0090E866FD8907A
:1037580085338433862FFBD7845180253C6E855171
:1037680081213D6E000E82213E6E000E83213F6E48
:1037780078EC50F0556E5550D8A49CD1FF0E00013E
:10378800806F010E816F53C082F054C083F0805166
:1037980082178151831745C084F046C085F0825155
:1037A8008427835185232E0E8425566E000E85218D
:1037B800576E47B00ED04CC080F00F0E801756C021
:1037C800D9FF57C0DAFFDF50F00B8011816F8151AC
:1037D80012D04BC080F04CC081F04DC082F04EC07A
:1037E80083F0050E05D0D89083338233813380333C
:1037F800E82EF9D78051516E526A56C0D9FF57C08A
:10380800DAFF51C0DFFF37D145C03AF046C03BF080
:1038180020EE1EF04550D9264650DA22DECF80F041
:10382800DECF81F0DECF82F0DECF83F04850846FA8
:103838004950856F4A50866F876B805184253C6E4E
:10384800815185213D6E825186213E6E83518721AB
:103858003F6E78EC50F0556E5550D8A42BD1FF0E22
:103868000001806F010E816F47C082F048C083F06D
:10387800D89082378337805182178151831745C08A
:1038880084F046C085F082518427835185232E0E0B
:103898008425566E000E8521576E56C0D9FF57C035
:1038A800DAFF4BC0DFFF20EE01F05650D926575003
:1038B800DA224CC0DFFFDFD045C03AF046C03BF00B
:1038C80020EE1EF04550D9264650DA22DECF80F091
:1038D800DECF81F0DECF82F0DECF83F047C084F008
:1038E80048C085F049C086F04AC087F0080E05D068
:1038F800D8908733863385338433E82EF9D78051BF
:1039080084253C6E815185213D6E825186213E6E13
:10391800835187213F6E78EC50F0556E5550D8A4EE
:10392800C9D0FF0E0001806F010E816F47C082F081
:1039380048C083F0D89082378337D890823783374E
:10394800805182178151831745C084F046C085F0A5
:1039580082518427835185232E0E8425566E000EAE
:103968008521576E20EE01F05650D9265750DA229D
:10397800DF50806F8051826F816B20EE02F05650CD
:10398800D9265750DA22DF50836F83C084F0856BC5
:10399800866B876B85C087F084C086F0856B846BE7
:1039A80020EE03F05650D9265750DA22DF50886FA0
:1039B80088C089F08A6B8B6B8C6B89C08CF08B6BA1
:1039C8008A6B896B845189118D6F85518A118E6F2D
:1039D80086518B118F6F87518C11906F81518D118A
:1039E800916F82518E11926F000E8F11936F000E9E
:1039F8009011946F56C0D9FF57C0DAFFDF50956F0A
:103A080095519111966F9251976F9351986F945168
:103A1800996F000E96159A6F000E97159B6F000E02
:103A280098159C6FF00E99159D6F9A514B129B51EA
:103A38004C129C514D129D514E1256C0D9FF57C081
:103A4800DAFF4BC0DFFF20EE01F05650D926575061
:103A5800DA224CC0DFFF20EE02F05650D92657502C
:103A6800DA224DC0DFFF20EE03F05650D92657501A
:103A7800DA224EC0DFFF20EE04F04550D92646502A
:103A8800DA22010EDF6E16D045C0D9FF46C0DAFF34
:103A9800DF50806F816B8151000AD8A4B6D5805160
:103AA800010AD8B4B5D5030AD8B4AED6010AD8B439
:103AB80003D7ABD5555012002B6E1CC042F01DC069
:103AC80043F02B50D8B402D0040E1200010E406E01
:103AD80073A013D2030E1200ACEC59F00009D8B44D
:103AE8002DD2000E08D2000E156E000E166E000EB6
:103AF800176E000E186E090E3EEC57F00009D8A498
:103B08001DD22C0E0C6E0D6A000E0F6E100E0E6E6E
:103B1800EDEC54F00009D8B411D22C44E846030B5C
:103B2800E806D8A44ED033C01EF03F0E1E161EC0A5
:103B38001FF0206A216A226A20C022F01FC021F0EB
:103B4800206A1F6A3450246E236A3550256E266A0F
:103B5800235025262450262225501F24276E265020
:103B68002020286E000E2120296E000E22202A6EA9
:103B7800010E27243C6E000E28203D6E000E2920E1
:103B88003E6E000E2A203F6E3CC01EF03DC01FF066
:103B98003EC020F03FC021F00A0ED8901E361F36D6
:103BA80020362136E82EF9D71CC0D9FF1DC0DAFF10
:103BB8001EC0DEFF1FC0DEFF20C0DEFF21C0DEFF0B
:103BC80090D71E6A36AE01D01E2A010E1E1631C0CD
:103BD8001FF00F0E1F163550030B020DF3501F2454
:103BE8001E24020F416E3250030B1E6E1F6A0A0E0E
:103BF800D8901E361F36E82EFBD73350206E216A28
:103C0800D89020362136D890203621363444E846DC
:103C1800030B226E236A20502226215023221E5095
:103C280022261F502322010E2226000E232222C004
:103C38003CF023C03DF03E6A3F6A41C01EF0F70EDB
:103C48001E263CC01FF03DC020F03EC021F03FC002
:103C580022F01E2A05D0D8901F362036213622366B
:103C68001E2EF9D73AD06FA445D0000E156E000E5F
:103C7800166E000E176E000E186E8D0E3EEC57F085
:103C88000009D8A45BD112EC5AF02C0E0C6E0D6A08
:103C9800000E0F6E100E0E6EEDEC54F00009D8B445
:103CA8004DD1300E416E03D012EC5AF0410641500E
:103CB800D8A4FAD736C01EF01E3A0F0E1E16100EE4
:103CC8001F6E206A216A226A1E2A05D0D8901F36E4
:103CD8002036213622361E2EF9D71CC0D9FF1DC02A
:103CE800DAFF1FC0DEFF20C0DEFF21C0DEFF22C0DA
:103CF800DEFFF7D6000E156E000E166E000E176E5C
:103D0800000E186E090E3EEC57F00009D8A416D123
:103D18002C0E0C6E0D6A000E0F6E100E0E6EEDEC72
:103D280054F00009D8B40AD16FA22AD039C01EF0C5
:103D3800060E1F6ED8901E321F2EFCD7FF0E1E26B1
:103D480036503F0B206E216AD89020362136226AE1
:103D580037AE01D0222A010E221622502026000E4C
:103D68002122010E2026000E21221E2A03D0D890DF
:103D7800203621361E2EFBD72050236E215034D0FA
:103D880036C01EF0D8901E32D8901E321F0E1E1656
:103D9800010E1E240C6E0D6A000E0D223750030B07
:103DA8001F6E206AD8901F362036D8901F362036CE
:103DB800D8901F36203637C021F0050E226ED890D5
:103DC8002132222EFCD7070E211621501F26000E65
:103DD8002022010E1F240E6E000E20200F6E23ECF1
:103DE80059F00C50236E0D50246E256A266A1CC0AB
:103DF800D9FF1DC0DAFF23C0DEFF24C0DEFF25C0C7
:103E0800DEFF26C0DEFF6DD642C0D9FF43C0DAFF11
:103E18006FC0DFFF66D6000E156E000E166E000E20
:103E2800176E000E186E090E3EEC57F00009D8A464
:103E380085D042C00CF043C00DF0000E0F6E100E7E
:103E48000E6EEDEC54F00009D8A44BD677D0000ED6
:103E5800156E000E166E000E176E000E186E0A0E06
:103E68003EEC57F00009D8A469D042C00CF043C01A
:103E78000DF0000E0F6E100E0E6EEDEC54F0E3D741
:103E8800000E156E000E166E000E176E000E186EE0
:103E98003A0E3EEC57F00009D8A450D0040E416EFB
:103EA8000AD012EC5AF042C0D9FF43C0DAFFDF6EE5
:103EB800424A432A41064150D8B413D6F2D7000EDD
:103EC800156E000E166E000E176E000E186E8D0E13
:103ED8003EEC57F00009D8A431D012EC5AF042C099
:103EE8000CF043C00DF0000E0F6E400E0E6EEDECA0
:103EF80054F0A9D7040E406E21D01B501E6E1F6AC5
:103F08001F50000AD8A4F6D71E50000AD8B4E4D52A
:103F1800010AD8B4E8D5020AD8B4A5D6090AD8B493
:103F280073D7010AD8B477D7070AD8B490D7010A4B
:103F3800D8B4A6D7030AD8B4C2D7DCD71EEC5AF037
:103F48004050120019C0F6FF1AC0F7FF000EF86EB5
:103F58000F0EF76403D00800F55005D0F6CFE9FF3F
:103F6800F7CFEAFFEF50476E194A1A2A4750D8B4DC
:103F78001200250E4718D8B404D04750DEEC59F08B
:103F8800E1D7000E436E000E426E19C0F6FF1AC04C
:103F9800F7FF000EF86E0F0EF76403D00800F55017
:103FA80005D0F6CFE9FFF7CFEAFFEF50476E194A81
:103FB8001A2A300E4718D8A419D0000E436E010EE5
:103FC800426E19C0F6FF1AC0F7FF000EF86E0F0E0A
:103FD800F76403D00800F55005D0F6CFE9FFF7CF16
:103FE800EAFFEF50476E194A1A2A08D02D0E4718D3
:103FF800D8A404D0000E436E020EE2D7000E3B6E2A
:10400800000E3A6E28D03AC00CF03BC00DF0000EFE
:104018000F6E0A0E0E6E23EC59F047500C26000E58
:104028000D22D00E0C243A6EFF0E0D203B6E19C0E7
:10403800F6FF1AC0F7FF000EF86E0F0EF76403D0F4
:104048000800F55005D0F6CFE9FFF7CFEAFFEF50AB
:10405800476E194A1A2A2F0E476403D0390E47644F
:10406800D2D76C0E4718D8B404D04C0E4718D8A431
:1040780015D0428419C0F6FF1AC0F7FF000EF86E7B
:104088000F0EF76403D00800F55005D0F6CFE9FF0E
:10409800F7CFEAFFEF50476E194A1A2A4750D8B4AB
:1040A800120047C046F0600E46647AD0200E465E85
:1040B80077D01B50D96EDA6A020EDF26DF5CD96E24
:1040C800DA6ADECF36F0DECF37F0000E3D6E000E36
:1040D8003C6E02D03C4A3D2A3C5036241C6E3D5072
:1040E80037201D6E1CC0F6FF1DC0F7FF000EF86ECE
:1040F8000F0EF76403D00800F55005D0F6CFE9FF9E
:10410800F7CFEAFFEF500009D8B404D0E3D7200E68
:10411800DEEC59F042B20CD03C501C6E3D501D6E86
:104128003C4A3D2A3A501C5C3B501D58D8A0EFD75A
:1041380036C00DF037C00EF0D7EC55F003D0200E86
:10414800DEEC59F03C501C6E3D501D6E3C4A3D2A39
:104158003A501C5C3B501D58D8B0F4D6F0D71B50D1
:10416800D96EDA6ADF50DF2ADF2AD96EDA6ADF50C1
:10417800DEEC59F0E7D6000E396E020E0BD0000EB9
:10418800396E080E07D0000E396E0A0E03D0000EE5
:10419800396E100E386E22D04750DEEC59F0D2D668
:1041A80046501C6E1D6A1D50000AD8A4F5D71C5035
:1041B800420AD8B4E0D7010AD8B4D1D7070AD8B48C
:1041C800E2D70B0AD8B4DBD71C0AD8B472D7060AD0
:1041D800D8B4D9D70D0AD8B4DAD7DED742B431D09B
:1041E800440E4618D8B413D01B50D96EDA6ADF5083
:1041F800DF2ADF2AD96EDA6ADECF1CF0DDCF1DF0A8
:104208001CC02EF01DC02FF0306A316A11D01B502F
:10421800D96EDA6ADF50DF2ADF2AD96EDA6ADECF92
:104228002EF0DDCF2FF0000E2FBEFF0E306E316E58
:104238002EC03EF02FC03FF030C040F031C041F0FA
:1042480010D01B50D96EDA6A040EDF26DF5CD96EF7
:10425800DA6ADECF3EF0DECF3FF0DECF40F0DECFD1
:1042680041F0440E4618D8B441AE0AD03E6C3F1E09
:10427800D8B03F2A401ED8B0402A000E4156428688
:10428800000E456E000E446E3EC00CF03FC00DF0AF
:1042980040C00EF041C00FF038C010F039C011F026
:1042A800126A136A88EC54F00C50466E3EC00CF04B
:1042B8003FC00DF040C00EF041C00FF038C010F004
:1042C80039C011F0126A136A9AEC53F00CC03EF030
:1042D8000DC03FF00EC040F00FC041F0090E46641B
:1042E8000ED0780E4718D8B404D0000E336E070EDF
:1042F80003D0000E336E270E326E325046264450DD
:104308001E0FD96EDA6A4650300FDF6E444A452ACE
:104318003E503F1040104110D8B406D0455004E13B
:10432800100E445CD8A0B0D742A608D044501E0F47
:10433800D96EDA6A2D0EDF6E444A452A44C03CF035
:1043480045C03DF042B004D0000E356E200E03D0BB
:10435800000E356E300E346E34C046F003D0465031
:10436800DEEC59F042B20CD03C501C6E3D501D6E34
:104378003C4A3D2A3A501C5C3B501D58D8A0EFD708
:104388004406D8A0450644501E0FD96EDA6ADF509D
:10439800DEEC59F044504510D8B404D0F1D7200EC3
:1043A800DEEC59F03C501C6E3D501D6E3C4A3D2AD7
:1043B8003A501C5C3B501D58D8B0C4D5F0D74A5071
:1043C8004910481004E1020E475CD8A010D020EE36
:1043D80012F04550D9264650DA22DE50475CDE50AE
:1043E8004858DE504958DE504A58D8A009D0010E26
:1043F8000001846F000E856F000E866F000EEDD1F0
:1044080000018469856986698769E9D147C088F0B0
:1044180048C089F0D89089314C6E88314B6E4B502A
:1044280088274C50892345C03AF046C03BF020EE1F
:104438001EF04550D9264650DA22DECF4BF0DECFAB
:104448004CF0DECF4DF0DECF4EF088C04FF089C083
:1044580050F0090E516ED89050324F32512EFBD782
:104468004F504B243C6E50504C203D6E000E4D205A
:104478003E6E000E4E203F6E78EC50F00009D8A436
:10448800C4D1FF0E4B6E010E4C6E88C04DF089C032
:104498004EF04B504D164C504E1645C04FF046C08E
:1044A80050F04D504F264E5050222E0E4F24D96EAC
:1044B800000E5020DA6EDF50516E51500001826FAD
:1044C800836B884B892B45C03AF046C03BF020EE01
:1044D8001EF04550D9264650DA22DECF4BF0DECF0B
:1044E8004CF0DECF4DF0DECF4EF088C04FF089C0E3
:1044F80050F0090E516ED89050324F32512EFBD7E2
:104508004F504B243C6E50504C203D6E000E4D20B9
:104518003E6E000E4E203F6E78EC50F00009D8A495
:1045280074D1FF0E4B6E010E4C6E88C04DF089C0E1
:104538004EF04B504D164C504E1645C04FF046C0ED
:1045480050F04D504F264E5050222E0E4F24D96E0B
:10455800000E5020DA6EDF50516E5150536E526A81
:104568005250000182135350831347B007D0FF0EF7
:104578008215806F0F0E8315816F0FD082C04BF0AC
:1045880083C04CF0040E4D6ED8904C324B324D2EF9
:10459800FBD74BC080F04CC081F080C084F081C054
:1045A80085F061D045C03AF046C03BF020EE1EF0E1
:1045B8004550D9264650DA22DECF4BF0DECF4CF0FC
:1045C800DECF4DF0DECF4EF048504F6E4950506E62
:1045D8004A50516E526A4B504F243C6E4C505020FA
:1045E8003D6E4D5051203E6E4E5052203F6E78EC3D
:1045F80050F00009D8A409D1FF0E4B6E010E4C6E85
:1046080047C04DF048C04EF0D8904D364E364B500E
:104618004D164C504E1645C04FF046C050F04D5008
:104628004F264E5050222E0E4F2400018A6F000E46
:1046380050208B6F20EE01F08A51D9268B51DA2257
:10464800DF504B6E4B504D6E4C6A8AC0D9FF8BC001
:10465800DAFFDF504E6E4E504C12000E4D124CC019
:1046680084F04DC085F0866B876BCFD045C03AF09B
:1046780046C03BF020EE1EF04550D9264650DA22BF
:10468800DECF4BF0DECF4CF0DECF4DF0DECF4EF07C
:1046980047C04FF048C050F049C051F04AC052F0EE
:1046A800080E05D0D8905232513250324F32E82E8F
:1046B800F9D74B504F243C6E4C5050203D6E4D5016
:1046C80051203E6E4E5052203F6E78EC50F000095B
:1046D800D8A49BD0FF0E4B6E010E4C6E47C04DF018
:1046E80048C04EF0D8904D364E36D8904D364E369E
:1046F8004B504D164C504E1645C04FF046C050F02A
:104708004D504F264E5050222E0E4F2400018A6FD6
:10471800000E50208B6F20EE01F08A51D9268B5164
:10472800DA22DF504B6E4B504D6E4C6A20EE02F091
:104738008A51D9268B51DA22DF504E6E4EC04FF087
:10474800506A516A526A50C052F04FC051F0506AD4
:104758004F6A20EE03F08A51D9268B51DA22DF50B6
:10476800536E53C054F0556A566A576A54C057F08E
:10477800566A556A546A4F505410586E5050551026
:10478800596E515056105A6E525057105B6E4C501D
:1047980058105C6E4D5059105D6E000E5A105E6ECA
:1047A800000E5B105F6E8AC0D9FF8BC0DAFFDF5046
:1047B800606E60505C10616E5D50626E5E50636E3C
:1047C8005F50646EFF0E6114846FFF0E6214856F74
:1047D800FF0E6314866F0F0E6414876F16D045C0E2
:1047E800D9FF46C0DAFFDF504B6E4C6A4C50000AC6
:1047F800D8A4FDD54B50010AD8B408D6030AD8B4BA
:10480800D1D6010AD8B432D7F2D584C045F085C0D4
:1048180046F086C047F087C048F012004E6E4A50F6
:10482800D8A45BEC59F0000E4D6E550E0001806F58
:10483800FF0E816F4EC082F0836B89A003D04B6A54
:104848004B2A01D04B6A4B500001846F856BC9EC31
:1048580059F04950D8B4A6D14E507F0B4E6E040E75
:104868004E18D8B404D0140E4E18D8A40AD0000E8E
:104878000101856F000E846F000E4A6E070E496EA7
:1048880012003F0E4E18D8A40CD0000E706E000E09
:104898000101856F000E846F000E4A6E000E496E8E
:1048A80012005F0E4E18D8A40CD0000E0101A46FA0
:1048B800000E856F000E846F000E4A6E000E496E62
:1048C80012003F0E4E6407D05F0E4E6004D0400EBB
:1048D8004E18D8A4EAD7400E4E18D8A40ED0010E10
:1048E8000101A46F000E706E000E856F000E846FBC
:1048F800000E4A6E000E496E1200200E4E18D8A403
:1049080051D1010E706E000E0101856F000E846F8B
:10491800000E4A6E000E496E1200600E4E18D8A4A2
:104928000DD00101A451D8B409D0A251D8B402D0F5
:10493800080E01D0030E4D6E000E28D0600E4E18E2
:10494800D8A40BD07050D8B408D00101A251D8B463
:1049580002D0090EF0D7050EEED7680E4E18D8A46F
:104968000AD07050D8B407D01A0E0101856F900E86
:1049780005D189807CD1680E4E18D8A40BD00101CE
:10498800A451D8B407D0020E4D6E5CD0856F000ECE
:10499800846F6DD16A0E4E18D8A408D07050D8B460
:1049A80005D01A0E0101856FF40EE8D06C0E4E1872
:1049B800D8A408D07050D8B405D01A0E0101856F5C
:1049C8002C0EDCD0700E4E18D8A40AD00101A451C8
:1049D800D8B406D0040E4D6E000E856F000ECED0F2
:1049E800700E4E18D8A443D17050D8B440D11B0EC5
:1049F8000101856F620EC2D0020E4E18D8A405D0F0
:104A08001A0E0101856F920E846F050E4E18D8A4F8
:104A180005D01A0E0101856FAE0E846F070E4E1871
:104A2800D8A405D01A0E0101856FB80E846F030E45
:104A38004E18D8B403D04E28D8A407D08980000EC9
:104A48004D6E8990000E0101A1D7160E4E18D8A4FC
:104A58000ED11A0E0101856FA40E9AD7050E4E18B5
:104A6800D8A405D11A0E0101856FF50E91D71A0E3B
:104A78000101856F9B0E8CD74EC069F01A0E01019B
:104A8800856F9C0E85D74EC06AF01A0E0101856F9E
:104A98009D0E7ED74EC06BF01A0E0101856F9E0EDB
:104AA80077D74EC06CF0000E0101856F000E846F41
:104AB800010E6AD01A0E0101856FB90E5FD01A0E69
:104AC8000101856FBA0E64D71A0E0101856FBB0EFE
:104AD8005FD7000E0101856F000E846FBE0E0001C6
:104AE800806FFE0E816FC9EC59F040D0000E0101B5
:104AF800856F000E846F060E47D0000E0101A26F6D
:104B08001A0E856FF70E846F020EE8EC59F02ED05E
:104B18001A0E0101856FF70E3BD78990270E010108
:104B2800856F0F0E846F030EE8EC59F0A0D0180EB5
:104B38004E18D8A49CD01A0E0101856F2D0E28D7C7
:104B48001A0E0101856F2E0E23D71A0E0101856FEB
:104B58002F0E1ED71A0E0101856F300E19D7000EC1
:104B68000101856F000E846F0A0E4D6E89907FD00B
:104B7800040E4D6E270E0101856F0F0E846FF9D656
:104B88008980000E010109D04D6E71D08990010E07
:104B98000101A26F080E4D6E000E856F000E846F26
:104BA800000EF2D784C14BF085C14CF04C50000A7E
:104BB800D8B40AD01A0AD8B40CD0010AD8B44DD047
:104BC8003C0AD8B452D053D04B50000AD8B4A5D61A
:104BD8004ED04B502C0AD8B4AAD7010AD8B4B0D7B3
:104BE800030AD8B4B2D7010AD8B4B4D71F0AD8B4C4
:104BF800B6D7A00AD8B400D7020AD8B438D7090A59
:104C0800D8B43AD7070AD8B43ED7010AD8B442D79D
:104C1800030AD8B446D73A0AD8B468D70A0AD8B427
:104C2800B5D7160AD8B446D7010AD8B448D7030A64
:104C3800D8B44AD7010AD8B44CD7790AD8B4A3D67D
:104C4800360AD8B40BD7010AD8B457D7030AD8B450
:104C58005FD7010AD8B461D70AD04B50580AD8B4E4
:104C680087D73A0AD8B48CD702D04B500F0A4DC018
:104C780049F04A6A1200040E8C6F020E8D6F340ED2
:104C88008E6F0B0E8F6F020E916F000E906FE50EF8
:104C9800926F936BA4EC15F0FD6F9A0E806FFD0E6A
:104CA800816FE5C082F0E6C083F0C9EC59F0000ED0
:104CB8000001E86F000EE76F000EE26F000EE16F73
:104CC800000EEA6F000EE96FE951C30FD96EDA6A78
:104CD800000EDF6EE951D20FD96EDA6A000EDF6E70
:104CE800E94BEA2BEABFF0D7EA5104E10F0EE95D80
:104CF800D8A0EAD7000EEC6F000EEB6F45D1340E4A
:104D0800EB25D96E0B0EEC21DA6E0D0EDE18D8A449
:104D1800F9D0800E806F030E816FE30E826FFE0E56
:104D2800836FC30E846F856BD20E866F876BC9EC59
:104D380059F0930E0C6EFF0E0D6EC30E0E6E1CEC2A
:104D480051F00C500D10D8A407D0D20E136E40ECC1
:104D58004AF013500101E16F8D0E0C6EFF0E0D6EBF
:104D6800C30E0E6E1CEC51F00C500D10D8A407D0D9
:104D7800D20E136E40EC4AF013500101A86F6B0E6F
:104D88000C6EFF0E0D6EC30E0E6E1CEC51F00C5027
:104D98000D10D8A407D0D20E136E40EC4AF0135071
:104DA8000101916FD10E0C6EFF0E0D6EC30E0E6ECB
:104DB8001CEC51F00C500D10D8A407D0D20E136E75
:104DC80040EC4AF0135001018F6F000E0001EE6FA6
:104DD800000EED6FB40E5F6E606A720E616EFF0EAC
:104DE800626EEDC063F0EEC064F0B6EC56F0B40E3F
:104DF8000C6E0D6AC30E0E6E1CEC51F00C500D10AB
:104E0800D8A418D0EDC00CF0EEC00DF0000E0F6E57
:104E18000F0E0E6E23EC59F0340E0C24126E0D0E8C
:104E28000D20136ED20E146E000E166E0F0E156E38
:104E38007FEC55F00001ED4BEE2BEEBFCBD7EE51DA
:104E480004E1100EED5DD8A0C5D7000EEE6F010E7F
:104E5800ED6FB40E5F6E606A790E616EFF0E626E62
:104E6800EDC063F0EEC064F0B6EC56F0B40E0C6E14
:104E78000D6AC30E0E6E1CEC51F00C500D10D8A428
:104E880018D0EDC00CF0EEC00DF0000E0F6E0F0E36
:104E98000E6E23EC59F0240E0C24126E0E0E0D200B
:104EA800136ED20E146E000E166E0F0E156E7FEC7A
:104EB80055F00001ED4BEE2BEEBFCBD7EE5104E1E0
:104EC800040EED5DD8A0C5D7000EEA6F000EE96F9D
:104ED800E951C30FD96EDA6A000EDF6EE951D20FBD
:104EE800D96EDA6A000EDF6EE94BEA2BEABFF0D71B
:104EF800EA5104E10F0EE95DD8A0EAD7000EE26F8F
:104F0800000E17D0340EEB25D96E0B0EEC21DA6E9D
:104F18000A0EDE18D8B436D0340EEB25D96E0B0E37
:104F2800EC21DA6E200EDE18D8A409D0000EE26F4C
:104F3800010EE16F000EE86F000EE76F23D0E1511C
:104F4800E211D8B409D0340EEB25D96E0B0EEC2142
:104F5800DA6EE751D20F08D0340EEB25D96E0B0E5E
:104F6800EC21DA6EE751C30FE16EE26ADFCFE7FFAB
:104F7800E8BF06D0E85106E10F0EE75DD8B002D0D1
:104F8800E74BE82BEB4BEC2BE551EB5DE651EC598D
:104F9800D8A0B5D68A0E806FFD0E816F91C182F0C0
:104FA800836BC9EC59F0F80E0001806FFD0E816F1C
:104FB800E1C182F0836BC9EC59F0E90E0001806F02
:104FC800FD0E816FA8C182F0836BC9EC59F0000E09
:104FD8000001EE6F000EED6FEDC00CF0EEC00DF0AD
:104FE800000E0F6E0F0E0E6E23EC59F0340E0C24CB
:104FF8000001E36F0D0E0D20E46F050E806FFD0EAE
:10500800816FEDC082F0EEC083F0E3C084F0E4C0AD
:1050180085F0C9EC59F00001ED4BEE2BEEBFDCD763
:10502800EE5104E1100EED5DD8A0D6D7000EEC6F5E
:10503800010EEB6FEBC00CF0ECC00DF0000E0F6E24
:105048000F0E0E6E23EC59F0240E0C240001E36FB2
:105058000E0E0D20E46F160E806FFD0E816FEBC0F3
:1050680082F0ECC083F0E3C084F0E4C085F0C9ECC2
:1050780059F00001EB4BEC2BECBFDCD7EC5104E111
:10508800040EEB5DD8A0D6D75A0E806FFC0E816F48
:10509800C9EC59F0120020EE04F0B151D926B251F2
:1050A800DA22DECFB5F0DDCFB6F0010EB525BE6F42
:1050B800000EB621BF6FBE51BF11D8B40CD020EE80
:1050C8000EF0B151D926B251DA22DE50DE10DE10D0
:1050D800DE10D8A402D0040E1200BEC0B5F00F0E28
:1050E800B517D8A4A3D120EE0EF0B151D926B251EC
:1050F800DA22DE2A000EDE22DE22DE2220EE0AF08E
:10510800B151D926B251DA22DE50DE10DE10DE109F
:10511800D8A411D0B1C0D9FFB2C0DAFF10EE08F0A0
:10512800DE50E126DD50E222E650BE5DE650BF5972
:10513800D8B0D1D77BD1BEC0B5F0BFC0B6F0040E91
:10514800B76FD890B633B533B72FFBD7FF0EB86F0C
:10515800FF0EB96FB1C0D9FFB2C0DAFF10EE02F08E
:10516800DE50E126DD50E222E750BA6FBB6BB85142
:10517800BA27B951BB23B551BA17B651BB17BA51A3
:10518800BB11D8A453D1B1C0D9FFB2C0DAFFDECF6A
:1051980045F0DDCF46F020EE0AF0B151D926B251E4
:1051A800DA22DECF47F0DECF48F0DECF49F0DECF9F
:1051B8004AF0E3EC21F045C0C0F046C0C1F047C05A
:1051C800C2F048C0C3F00001C351C211C11106E1C9
:1051D800020EC05DD8B002D0020E1200C02909E14B
:1051E800C12907E1C22905E1C329D8A402D0010ECB
:1051F8001200B1C0D9FFB2C0DAFF10EE12F0DE50D3
:10520800E126DD50E222E650C05DE650C159E65085
:10521800C259E650C359D8A0DAD0B351B411D8B4A2
:105228005AD7B1C0D9FFB2C0DAFFDECF9EF0DDCFCA
:105238009FF020EE0AF0B151D926B251DA22DECF22
:10524800A0F0DECFA1F0DECFA2F0DECFA3F0E3EC3A
:105258002DF09EC0C0F09FC0C1F0A0C0C2F0A1C098
:10526800C3F0C051C111C211C311D8A402D0070E96
:105278001200C005C111C211C311D8B4ADD7C029DD
:1052880007E1C12905E1C22903E1C329D8B4AFD791
:10529800B1C0D9FFB2C0DAFFDECF25F0DDCF26F0EE
:1052A8007BEC46F00009D8A4A2D7B1C0D9FFB2C0A0
:1052B800DAFFDECFB5F0DDCFB6F02E0E0001B52552
:1052C8000C6E000EB6210D6E000E0F6E000E0E6EE7
:1052D800020E116E000E106EE6EC58F0B1C0D9FF48
:1052E800B2C0DAFFDECF18F0DDCF19F0C0C01AF077
:1052F800C1C01BF0C2C01CF0C3C01DF06FEC4FF062
:10530800B1C0D9FFB2C0DAFF10EE2AF0DE50E126B4
:10531800DD50E22218C0E6FF19C0E6FF1AC0E6FF1A
:105328001BC0E6FF000E0001BD6F000EBC6F2BD046
:10533800B1C0D9FFB2C0DAFF10EE04F0DE50E126AA
:10534800DD50E222010EE76EB1C0D9FFB2C0DAFF2C
:10535800DECF25F0DDCF26F07BEC46F00009D8A49F
:1053680046D7B1C0D9FFB2C0DAFF10EE2AF0DE503E
:10537800E126DD50E222E62A000EE622E622E622B7
:105388000001BC4BBD2BB1C0D9FFB2C0DAFF10EE93
:1053980002F0DE50E126DD50E222E750B56FB66B31
:1053A800B551BC5DB651BD59D8A0C2D7B1C0D9FF5F
:1053B800B2C0DAFF10EE2AF0DE50E126DD50E2221C
:1053C800BC51E65EBD51E65A000EE65AE65A20EE9A
:1053D8000AF0B151D926B251DA22C0C0DEFFC1C0ED
:1053E800DEFFC2C0DEFFC3C0DEFFB1C0D9FFB2C05E
:1053F800DAFFDECF18F0DDCF19F0C0C01AF0C1C057
:105408001BF0C2C01CF0C3C01DF06FEC4FF00001D0
:1054180020EE0EF0B151D926B251DA2218C0DEFFC3
:1054280019C0DEFF1AC0DEFF1BC0DEFF20EE04F04D
:10543800B151D926B251DA22BEC0DEFFBFC0DDFFAE
:105448000F0EBE15B56F000EBF15B66F050ED890BE
:10545800B537B637E82EFBD7B1C0D9FFB2C0DAFFEF
:10546800DECFB7F0DDCFB8F0B551B727B651B823C6
:105478002E0EB727000EB82320EE12F0B151D92610
:10548800B251DA22B7C0DEFFB8C0DDFF000E12004D
:105498008980FD0E0001806FF70E816FCFCF82F0FB
:1054A800836BCECF84F0856B6E50140D070EF324FA
:1054B800D96E010EF420DA6EDECF86F0DECF87F0EB
:1054C800DECF88F0DECF89F06E50140D070EF3247E
:1054D800D96E010EF420DA6EDECF8AF0DECF8BF0C3
:1054E800DECF8CF0DECF8DF0C9EC59F024EC3FF024
:1054F800D8C0AFF1D9C0B0F10101AF51B011D8B4E3
:105508001AD06E50140D130EF324D96E010EF42028
:10551800DA6E6E50140D130EF324E16E010EF420B2
:10552800E26EE7500409DF6EDBEC57F0AFC1EFF035
:10553800B0C1F0F012006E50140D0F0EF324D96EA6
:10554800010EF420DA6EDECFF1F0DECFF2F0DECF1E
:10555800F3F0DECFF4F0F2C0F1F0F3C0F2F0F4C0F3
:10556800F3F00001F46BF1C0A9F1F2C0AAF16E509A
:10557800140D0F0EF324D96E010EF420DA6EDECF6F
:10558800F1F0DDCFF2F0F1510101B16FB26B725061
:10559800FD0B726E000EAE6F000EAD6F000EAC6F9D
:1055A800000EAB6FB1D0FF0EF16FFF0EF26FA9C105
:1055B800F3F0AAC1F4F0F151F327F251F4230101F9
:1055C800AB510001F3190EE10101AC510001F419CE
:1055D800D8A408D00101B151B211D8A403D0725097
:1055E8000209726E6E50200D040EF32400018C6FB8
:1055F800020EF4208D6F340E8E6F0B0E8F6F010E1E
:10560800916F000E906FB40E926F010E936FA4EC21
:1056180015F00101B36F730E0001806FF70E816FF3
:10562800CFCF82F0836BCECF84F0856BB3C186F089
:10563800876BB4C188F0B5C189F0C9EC59F0010194
:10564800B351D8A45ED7B4C149F0B5C14AF044EC0F
:1056580036F00101B451AD25AD6FB551AE21AE6F35
:105668006E50140D070EF324D96E010EF420DA6E75
:10567800000EDE240001F16F010EDE20F26F000E35
:10568800DE20F36F000EDE20F46F6E50140D070E4F
:10569800F324D96E010EF420DA6EF1C0DEFFF2C0F9
:1056A800DEFFF3C0DEFFF4C0DEFF990E806FF90E57
:1056B800816FCFCF82F0836BCECF84F0856B6E5035
:1056C800140D070EF324D96E010EF420DA6EDECF26
:1056D80086F0DECF87F0DECF88F0DECF89F06E501F
:1056E800140D070EF324D96E010EF420DA6EDECF06
:1056F8008AF0DECF8BF0DECF8CF0DECF8DF0C9ECF8
:1057080059F00101AB4BAC2BA951AB5DAC51800AF0
:105718000001F16F0101AA51800A0001F159D8A0D6
:1057280042D70101B2BF8BD0B25103E1B105D8A075
:1057380086D06E50200D040EF32400018C6F020EEB
:10574800F4208D6F340E8E6F0B0E8F6FB1C190F0F9
:10575800B2C191F0B40E926F010E936FA4EC15F0E4
:105768000101B36F400E0001806FFA0E816FB3C163
:1057780082F0836BB4C184F0B5C185F0C9EC59F0EF
:105788000101B351D8A4BDD672500209726EB1C1DD
:1057980049F0B2C14AF044EC36F00101B451AD25EC
:1057A800AD6FB551AE21AE6F6E50140D070EF324D8
:1057B800D96E010EF420DA6E000EDE240001F16FBE
:1057C800010EDE20F26F000EDE20F36F000EDE20E9
:1057D800F46F6E50140D070EF324D96E010EF420E9
:1057E800DA6EF1C0DEFFF2C0DEFFF3C0DEFFF4C008
:1057F800DEFF350E806FFC0E816F6E50140D070EA4
:10580800F324D96E010EF420DA6EDECF82F0DECFFB
:1058180083F0DECF84F0DECF85F06E50140D070ED6
:10582800F324D96E010EF420DA6EDECF86F0DECFD7
:1058380087F0DECF88F0DECF89F0C9EC59F07250DE
:10584800FD0B726E740E0001806FFA0E816FCFCF60
:1058580082F0836BCECF84F0856BADC186F0AEC18C
:1058680087F0C9EC59F0000E6D6E89906DC0EFF0AD
:105878000001F06B120044C025F045C026F07BEC17
:1058880046F04E6E4E50D8A498D144C0D9FF45C0BA
:10589800DAFF030EDE18D8A47CD120EE05F04450C0
:1058A800D9264550DA22DE04D8A473D12E0E44241A
:1058B8000C6E000E45200D6E000E0F6E000E0E6E63
:1058C800020E116E000E106EE6EC58F022EE2CF06F
:1058D8004450D9264550DA22550EDF6E22EE2DF0BF
:1058E8004450D9264550DA22AA0EDF6E20EE2EF05B
:1058F8004450D9264550DA22520EDF6E20EE2FF0A2
:105908004450D9264550DA22520EDF6E20EE30F090
:105918004450D9264550DA22610EDF6E20EE31F070
:105928004450D9264550DA22410EDF6E22EE12F09D
:105938004450D9264550DA22720EDF6E22EE13F05B
:105948004450D9264550DA22720EDF6E22EE14F04A
:105958004450D9264550DA22410EDF6E22EE15F06A
:105968004450D9264550DA22610EDF6E20EE0EF043
:105978004450D9264550DA2212EE16F04450E1265A
:105988004550E222DFCFE7FF22EE17F04450D92638
:105998004550DA2210EE0EF04450E1264550E2223E
:1059A800E6CF46F0E5CF47F047C046F0476A465095
:1059B800DF6E22EE18F04450D9264550DA2210EE58
:1059C8000EF04450E1264550E222E6CF46F0E6CFFD
:1059D80047F0E6CF48F0E6CF49F0110E05D0D89051
:1059E8004932483247324632E82EF9D74650DF6E00
:1059F80022EE19F04450D9264550DA2210EE0EF066
:105A08004450E1264550E222E6CF46F0E6CF47F083
:105A1800E6CF48F0E6CF49F0190E05D0D8904932C4
:105A2800483247324632E82EF9D74650DF6E20EE2C
:105A38000AF04450D9264550DA2212EE1AF04450A2
:105A4800E1264550E222DFCFE7FF22EE1BF044506B
:105A5800D9264550DA2210EE0AF04450E126455086
:105A6800E222E6CF46F0E5CF47F047C046F0476A66
:105A78004650DF6E22EE1CF04450D9264550DA22FB
:105A880010EE0AF04450E1264550E222E6CF46F0F7
:105A9800E6CF47F0E6CF48F0E6CF49F0110E05D043
:105AA800D8904932483247324632E82EF9D7465024
:105AB800DF6E22EE1DF04450D9264550DA2210EE52
:105AC8000AF04450E1264550E222E6CF46F0E6CF00
:105AD80047F0E6CF48F0E6CF49F0190E05D0D89048
:105AE8004932483247324632E82EF9D74650DF6EFF
:105AF80020EE1AF04450D9264550DA22DECF46F07F
:105B0800DECF47F0DECF48F0DECF49F0010E462465
:105B18004A6E000E47204B6E000E48204C6E000E59
:105B280049204D6E20EE2AF04450D9264550DA22FD
:105B38004AC0DEFF4BC0DEFF4CC0DEFF4DC0DEFFBB
:105B48002E0E44241B6E000E45201C6E20EE2AF0FB
:105B58004450D9264550DA22DECF1DF0DECF1EF0A4
:105B6800DECF1FF0DECF20F0000E226E010E216E78
:105B780020EE01F04450D9264550DA22DF5065EC7A
:105B88004BF020EE05F04450D9264550DA22000E9D
:105B9800DF6E000E1B6E000E1C6E000E1D6E20EEDA
:105BA80001F04450D9264550DA22DF5060EC1DF050
:105BB8000009D8B402D0010E4E6E4E501200A0510A
:105BC800A111A211A311D8A42DD020EE0AF09E5144
:105BD800D9269F51DA22DECFA5F0DECFA6F0DECFA0
:105BE800A7F0DECFA8F0A551A611A711A811D8B427
:105BF80010D020EE12F09E51D9269F51DA22DE50A5
:105C0800A55DDE50A659DE50A759DE50A859D8A088
:105C18005BD0010EA56F000EA66F000EA76F000ED9
:105C2800A86F52D09EC045F09FC046F0A0C047F074
:105C3800A1C048F0A2C049F0A3C04AF0E3EC21F0AB
:105C480045C0ADF046C0AEF047C0AFF048C0B0F0B8
:105C58000001B051AF11AE110DE1020EAD5DD8B02B
:105C680009D0010E9E6F000E9F6F000EA06F000EF0
:105C7800A16F1200AD2910E1AE290EE1AF290CE1A8
:105C8800B029D8A409D0ADC09EF0AEC09FF0AFC077
:105C9800A0F0B0C0A1F0120020EE12F09E51D9265B
:105CA8009F51DA22DE50AD5DDE50AE59DE50AF595D
:105CB800DE50B059D8A0E7D7A0C0A5F0A1C0A6F083
:105CC800A2C0A7F0A3C0A8F0A5C0A9F0A6C0AAF0DA
:105CD800A7C0ABF0A8C0ACF0010EA927000EAA23FC
:105CE800AB23AC2320EE12F09E51D9269F51DA2225
:105CF800DE50A95DDE50AA59DE50AB59DE50AC59D2
:105D0800D8A019D0020EA96F000EAA6F000EAB6FB3
:105D1800000EAC6FA851A711A6110DE1020EA55DEA
:105D2800D8B009D0000E9E6F000E9F6F000EA06FB6
:105D3800000EA16F12009EC045F09FC046F0A9C09A
:105D480047F0AAC048F0ABC049F0ACC04AF0E3EC59
:105D580021F045C0ADF046C0AEF047C0AFF048C036
:105D6800B0F00001AD51AE11AF11B011D8B41DD0D3
:105D7800AD2907E1AE2905E1AF2903E1B029D8B47F
:105D880082D7AD05AE11AF11B011D8B47CD7A551EB
:105D9800A919A2E1A651AA199FE1A751AB199CE143
:105DA800A851AC19D8B4BED797D79EC045F09FC0AC
:105DB80046F0A9C047F0AAC048F0ABC049F0ACC053
:105DC8004AF0FF0E4B6EFF0E4C6EFF0E4D6E0F0E1F
:105DD8004E6EF1EC1AF00001A46FA451D8A41ED0A5
:105DE800A051A111A211A311D8B418D09EC045F09A
:105DF8009FC046F0A0C047F0A1C048F0A2C049F03B
:105E0800A3C04AF0A9C04BF0AAC04CF0ABC04DF0FB
:105E1800ACC04EF0F1EC1AF00001A46FA451D8A464
:105E280031D020EE0AF09E51D9269F51DA22A9C01E
:105E3800DEFFAAC0DEFFABC0DEFFACC0DEFF20EE97
:105E48000EF09E51D9269F51DA22DE2807E1DE287E
:105E580005E1DE2803E1DE28D8B424D020EE0EF0D8
:105E68009E51D9269F51DA22DE06000EDE5ADE5AEE
:105E7800DE5A20EE05F09E51D9269F51DA22000EF7
:105E8800DB8010D0A405D8B409D0010EA96F000E8C
:105E9800AA6F000EAB6F000EAC6F04D0A969AA6997
:105EA800AB69AC69A9C09EF0AAC09FF0ABC0A0F0D6
:105EB800ACC0A1F012000001AF6F0001AD51D8A431
:105EC800A9EC43F0000E0001AE6FAC51D8B44AD132
:105ED800040EAF19D8B404D0140EAF19D8A40DD03D
:105EE800000E0101896F000E736F000E726F000EB5
:105EF8000001AD6F070EAC6F12003F0EAF19D8A4AA
:105F08000BD0000EFC6F000E0101896F000E00011E
:105F1800AD6F000EAC6F12005F0EAF19D8A40BD096
:105F2800000E01018A6F000E896F000E0001AD6F2F
:105F3800000EAC6F12003F0EAF6507D05F0EAF6169
:105F480004D0400EAF19D8A4EBD7400EAF19D8A48F
:105F58000BD0010E01018A6F000E896F000E00013F
:105F6800AD6F000EAC6F1200200EAF19D8A412D07E
:105F7800010EFC6F000E0101896F870E0001806F12
:105F8800FF0E816FC9EC59F0000E0001AD6F000ED5
:105F9800AC6F1200650EAF19D8A410D0FC51D8B45C
:105FA8000DD0000E0101736F000E726F010E896F24
:105FB800000E0001AD6F000EAC6F12006E0EAF192F
:105FC800D8A403D0020E0101896F700E0001AF1929
:105FD800D8A40AD001018A51D8B406D0000E736F34
:105FE800000E726F030E896F700E0001AF19D8A4EE
:105FF80011D0FC51D8B40ED08980000E0101736F06
:10600800000E726F040E896F000E0001AD6F000E56
:10601800AC6F1200720EAF19D8A4A4D0FC51D8B43A
:10602800A1D089801C0E0101736F2A0E726F050EB4
:10603800896F000E0001AD6F000EAC6F12000001F9
:10604800AF5183EC0BF00001AE6FA7D0898000013F
:10605800AF5119EC54F00001AE6F000E0101896FC9
:106068009CD089803F0E0001806FF90E816FCFCFE1
:1060780082F0836BCECF84F0856B6DC086F0876B22
:10608800C9EC59F0340E0C6E0B0E0D6E000E0F6E2F
:10609800000E0E6E010E116E000E106E0EEC49F021
:1060A80072500209726E2BEE34F06DC0DFFFF40EF1
:1060B8000001806FFC0E816F000E836F010E826FEE
:1060C800C9EC59F0340E0001A66F0B0EA76F000E35
:1060D800A96F010EA86F640EAA6FFF0EAB6FEAECF2
:1060E8003AF0000E4A6E010E496E44EC36F07250DA
:1060F800FD0B726E080EAFD78990000E0001AE6FCF
:10610800E10E806FF80E816FCFCF82F0836BCECF18
:1061180084F0856BAFC086F0876BC9EC59F03DD031
:10612800080E0001AF19D8A438D03F0E806FF80EC2
:10613800816FCFCF82F0836BCECF84F0856BAFC0F9
:1061480086F0876BC9EC59F08990000E0001AE6F9C
:10615800000E6D6E000E0101896F000E736F000E48
:10616800726F1BD001018951676E686A6850000A16
:10617800D8A413D06750000AD8B40FD0010AD8B4F5
:106188005ED7030AD8B462D7010AD8B46AD7070A17
:10619800D8B4B2D7010AD8B4C3D7AEC0ACF00001A6
:1061A800AD6B12001650D96EDA6ADECF23F0DDCF60
:1061B80024F002D0234A242A23C0F6FF24C0F7FF84
:1061C800000EF86E0F0EF76403D00800F55005D0E6
:1061D800F6CFE9FFF7CFEAFFEF502F0AD8B4EAD796
:1061E80023C0F6FF24C0F7FF000EF86E0F0EF76409
:1061F80003D00800F55005D0F6CFE9FFF7CFEAFF46
:10620800EF505C0AD8B4D6D720EE14F01450D92633
:106218001550DA22DECF25F0DDCF26F025C00CF0B0
:1062280026C00DF0000E0F6E200E0E6E000E116EC1
:106238000B0E106EE6EC58F0000E1F6E1FC027F014
:10624800286A27C01DF028C01EF0000E216E080E17
:10625800206E1D502324176E1E502420186E17C060
:10626800F6FF18C0F7FF000EF86E0F0EF76403D0A4
:106278000800F55005D0F6CFE9FFF7CFEAFFEF5059
:10628800296E1D4A1E2A200E2964AFD02F0E291808
:10629800D8B4ABD05C0E2918D8B4A7D02E0E2918C4
:1062A800D8B406D02050275C21502858D8A018D040
:1062B800080E20182110D8A404D02E0E2918D8B4FE
:1062C80002D0060E1200000E286E080E276E000E71
:1062D800216E0B0E206ED8901F36D8901F36B9D776
:1062E8007F0E296402D0030E1F12800E296403D08A
:1062F8009F0E296406D0DF0E29644ED0FD0E29605A
:106308004BD01D502324176E1E502420186E17C022
:10631800F6FF18C0F7FF000EF86E0F0EF76403D0F3
:106328000800F55005D0F6CFE9FFF7CFEAFFEF50A8
:10633800226E1D4A1E2A3F0E226403D07E0E22645E
:1063480006D07F0E2264BDD7FD0E2260BAD7FF0E9D
:10635800176EFF0E186E20C019F021C01AF01750E2
:10636800192618501A221950275C1A502858D8B0E4
:10637800A8D727502524D96E28502620DA6E29C0A0
:10638800DFFF274A282A27502524D96E285026209F
:10639800DA6E22C0DFFF26D0430E0C6EFE0E0D6EA5
:1063A80029C00EF00F6A4CEC56F00C500D10D8A412
:1063B80088D7400E296405D05B0E296002D01F8261
:1063C80009D0600E296406D07B0E296003D01F8097
:1063D800200E295E27502524D96E28502620DA6EF3
:1063E80029C0DFFF274A282A34D71D502324176ED7
:1063F8001E502420186E1650D96EDA6A17C0DEFFB8
:1064080018C0DDFF200E296404D0000E1C6E000E9B
:1064180003D0000E1C6E040E1B6E1BC029F0275003
:106428002810D8B44ED725C0D9FF26C0DAFFE50E0C
:10643800DE18D8A406D025C0D9FF26C0DAFF050E7D
:10644800DF6E080E20182110D8A404D0D8901F366B
:10645800D8901F361F50030BE806D8B429881F5060
:106468000C0B040AD8B4298620EE0BF02550D92647
:106478002650DA2229C0DFFF000E1200000E0101AB
:10648800D96F0A0ED86F000ED76F050ED66F4FD191
:10649800000E0101D96F140ED86F40D1710E0D6E28
:1064A800FC0E0E6ED7EC55F082B205D0000E01013D
:1064B800D96F1E0ED86F150E0001FA6F4B0EF96FCB
:1064C800BE0EE82EFED7F92FFCD7FA2FFAD700F028
:1064D80025D1CB0E0D6EFE0E0E6ED7EC55F0060EC6
:1064E8000001D86F090ED96F5C0EDA6FFC0EDB6FF6
:1064F800000EDC6F24EC50F0FD6FFD511FEC55F0E1
:10650800600E0001806FFE0E816F06C9F9F0F95127
:10651800826F836BC9EC59F00001FD51D8A4CBD729
:10652800000E0101D96F230EC5D7070E0D6EFE0EA2
:106538000E6ED7EC55F0040E0001D86F020ED96F1D
:10654800070EDA6FFF0EDB6F010EDC6F6FEC18F0D1
:106558000001FD6FFD511FEC55F00001FD51D8A45D
:106568000AD03FEC26F0040E5C6E020E5D6EF9EC6C
:1065780057F00001FD6FFD511FEC55F0000E0101B1
:10658800D96F280ED86F9151D8A40DD0000EA66FE0
:10659800340E5F6E0D0E606E970E616EFE0E626EAB
:1065A800B6EC56F00DD05D0E0001806FF90E816FCC
:1065B80091C182F0836BA6C184F0856BC9EC59F058
:1065C800160E0001806FFE0E816F0101A6510F0D9E
:1065D800340EF3240001826F0D0EF420836FC9EC92
:1065E80059F069D7850E806FFB0E816F0101A651A6
:1065F8000F0D340EF3240001826F0D0EF420836F0B
:10660800C9EC59F0040E0001D86F020ED96F0101D0
:10661800A6510F0D340EF3240001DA6F0D0EF4208D
:10662800DB6F030EDC6F6FEC18F00001FD6FFD519E
:10663800D8A405D0000E0101D96F3C0ED86F040E06
:106648000001FD19D8A437D7000E0101D96F320E09
:1066580031D7D00E806FFC0E816F0101A6510F0D4E
:10666800340EF3240001826F0D0EF420836FC9EC01
:1066780059F0040E0001D86F020ED96F0101A6511E
:106688000F0D340EF3240001DA6F0D0EF420DB6FCA
:10669800070EDC6F6FEC18F00001FD6FFD51D8A4F8
:1066A8000AD7000E0101D96F3C0E04D7990E806FEE
:1066B800FC0E816F0101A6510F0D340EF324000169
:1066C800826F0D0EF420836FC9EC59F0000E0001A3
:1066D800F86F010EF76F1200D8C1F9F0D9C1FAF0BE
:1066E8000001FA51000AD8A419D0F9510A0AD8B4FD
:1066F800CFD61E0AD8B4D2D60A0AD8B4EAD63D0AEA
:10670800D8B413D70B0AD8B46DD7050AD8B406D0B5
:106718001F0AD8B49ED70E0AD8B4C8D7140E0101E0
:10672800D819D911D8B403D0D607D8A0D707D7BF5E
:1067380005D0D751D1E1D605D8B0CED7000E00018B
:10674800F86F000EF76F120020EE04F06550D9269E
:106758006650DA2267C0DEFF68C0DDFF20EE06F073
:106768006550D9266650DA22DECF99F0DECF9AF04E
:10677800DECF9BF0DECF9CF099059A119B119C11FE
:10678800D8B414D065C0D9FF66C0DAFF10EE12F095
:10679800DE50E126DD50E222E650995DE6509A5936
:1067A800E6509B59E6509C59D8A002D0020E120020
:1067B80099519A119B119C11D8A422D065C0D9FF78
:1067C80066C0DAFFDECF8CF0DDCF8DF08CC0D9FF4C
:1067D8008DC0DAFF030EDE18D8A412D065C0D9FF29
:1067E80066C0DAFF10EE22F0DE50E126DD50E2222C
:1067F800E6CF99F0E6CF9AF0E6CF9BF0E6CF9CF093
:1068080099519A119B119C11D8A423D065C0D9FF26
:1068180066C0DAFF10EE08F0DE50E126DD50E22215
:10682800E650675CE6506858D8B0C0D765C0D9FF55
:1068380066C0DAFF10EE22F0DE50E126DD50E222DB
:10684800E6CF95F0E6CF96F0E6CF97F0E6CF98F052
:1068580079D065C0D9FF66C0DAFF10EE02F0DE50CD
:10686800E126DD50E222E7508C6F8C51100DF3CFFA
:1068780093F0F4CF94F046D065C0D9FF66C0DAFF34
:10688800DECF45F0DDCF46F099C047F09AC048F01A
:106898009BC049F09CC04AF0E3EC21F045C099F058
:1068A80046C09AF047C09BF048C09CF00001992967
:1068B80009E19A2907E19B2905E19C29D8A402D07E
:1068C800010E12009C519B119A1104E1020E995D70
:1068D800D8A06CD765C0D9FF66C0DAFF10EE12F0F9
:1068E800DE50E126DD50E222E650995DE6509A59E5
:1068F800E6509B59E6509C59D8B058D79351675EDB
:106908009451685A9351675C94516858D8B0B4D779
:1069180065C0D9FF66C0DAFFDECF18F0DDCF19F009
:1069280099C01AF09AC01BF09BC01CF09CC01DF0C7
:106938006FEC4FF018C095F019C096F01AC097F098
:106948001BC098F020EE0AF06550D9266650DA226E
:1069580099C0DEFF9AC0DEFF9BC0DEFF9CC0DEFF51
:1069680000019551961197119811D8B41FD767C097
:106978008CF068C08DF0040E8E6FD8908D338C33F8
:106988008E2FFBD78C5195258F6F8D519621906F47
:10699800000E9721916F000E9821926F20EE0EF055
:1069A8006550D9266650DA228FC0DEFF90C0DEFF20
:1069B80091C0DEFF92C0DEFF0F0E67148C6F000ED1
:1069C80068148D6F050ED8908C378D37E82EFBD75D
:1069D80065C0D9FF66C0DAFFDECF8EF0DDCF8FF05D
:1069E8008C518E278D518F232E0E8E27000E8F23CC
:1069F80020EE12F06550D9266650DA228EC0DEFFEE
:106A08008FC0DDFF000E1200340E0101C26F0B0EA5
:106A1800C36FF8C012F0F9C013F0FBEC56F0125037
:106A28000101B66FD80E0001B16FB26B000EB36FE3
:106A3800000EB46F000EB56F000EB66F9FEC12F02B
:106A48000101BF6FBF51D8B411D0DC0E0001806FB7
:106A5800FA0E816FC9EC59F0000E0001D86F000ED4
:106A6800D96F000EDA6F000EDB6F1200D80E00012E
:106A78008C6F8D6BC2C18EF0C3C18FF0010E916F08
:106A8800000E906FBD0E926F010E936FA4EC15F07F
:106A98000101BF6FBF51D8B408D0B30E0001806F99
:106AA800FB0E816FC9EC59F0D7D7C2C1D9FFC3C15A
:106AB800DAFF800EDE18D8B408D0380E0001806FD7
:106AC800FD0E816FC9EC59F0C7D720EE0AF0C2510C
:106AD800D926C351DA22DF50A96FA951AB6FAA6B2F
:106AE80020EE0BF0C251D926C351DA22DF50AC6F29
:106AF800AC51AA25BB6F000EAB21BC6F9C0E0001E8
:106B0800806FFB0E816FBBC182F0BCC183F0C9EC02
:106B180059F0D80E0001B16FB26B0101BB51AA6FD9
:106B2800A96BA9C1B3F0AAC1B4F00001B56BB66BEB
:106B38009FEC12F00101BF6FBF51D8A48DD7D80EBA
:106B480000018C6F8D6BC2C18EF0C3C18FF0010E36
:106B5800916F000E906FBD0E926F010E936FA4ECB3
:106B680015F00101BF6FBF51D8A476D7000EC16FD1
:106B7800000EC06FF8C00CF0F9C00DF0C0C1A9F14B
:106B8800C1C1AAF1050ED890A937AA37E82EFBD7BC
:106B9800A951C2250E6EAA51C3210F6EB6C110F0BD
:106BA800116ACBEC50F00C500D10D8A45DD0C0C1C8
:106BB800A9F1C1C1AAF1050ED890A937AA37E82EC4
:106BC800FBD7C2C1ABF1C3C1ACF1A951AB27AA51E4
:106BD800AC230E0EAB25D96E000EAC21DA6EDF5059
:106BE800AD6FAD51AF6FAE6BC0C1B0F1C1C1B1F106
:106BF800050ED890B037B137E82EFBD7C2C1B2F135
:106C0800C3C1B3F1B051B227B151B3230F0EB225AE
:106C1800D96E000EB321DA6EDF50B46FB56BAE518A
:106C2800B427AF51B523B4C1B7F1B5C1B8F1000E5F
:106C3800B8BFFF0EB96FBA6F250E0001806FFE0E48
:106C4800816FB7C182F0B8C183F0B9C184F0BAC10D
:106C580085F0C9EC59F0B7C1D8F0B8C1D9F0B9C1BD
:106C6800DAF0BAC1DBF01200C04BC12BC1BF82D72A
:106C7800C15105E10F0EC05DD8B0EED67BD7ECD67A
:106C8800000E0101996F000E7B6F000E7A6F9386DC
:106C9800938093829384938895688A908A928A9441
:106CA8008A98010E966F898E89B411D0E0A707D013
:106CB8002A0E0001806FF70E816FC9EC59F0000EA3
:106CC8000101966F000E4A6E000E496E1200F2988E
:106CD8001A0EE82EFED700D0F0D081A881BA1ED0B7
:106CE800B10E0001806FFE0E816F80A003D04B6A49
:106CF8004B2A01D04B6A4B500001826F836B89A0ED
:106D080003D04C6A4C2A01D04C6A4C500001846F65
:106D1800856B99C186F0876BC9EC59F081B806D0AC
:106D280095687AC149F07BC14AF0120081B80BD04E
:106D3800340E0001806FFE0E816FC9EC59F0630EAE
:106D48000101996FC1D0100E0101646F270E656FA4
:106D5800000E666F000E676F90D081B281A410D0CC
:106D68006407000E655B665B675B642906E165295D
:106D780004E1662902E16729D8A49FD0620E73D086
:106D8800010E71D081A899D0020E6DD0FF0E4B6E06
:106D9800FF0E4C6E49C04DF04AC04EF04B504D2688
:106DA8004C504E227A514D1806E17B514E18D8B4FA
:106DB80072A201D0939A340E7A25D96E0B0E7B21DC
:106DC800DA6EDF50FF0A8C6E7A4B7B2B000E956EC5
:106DD800030E21D0100E646F270E656F000E666FCC
:106DE800000E676F6AD081B20ED06407000E655B33
:106DF800665B675B642909E1652907E1662905E1A6
:106E08006729D8A402D0040E996F81A256D0040E27
:106E18002AD09390050E996FDDD7938481B40ED054
:106E28006407000E655B665B675B642909E1652999
:106E380007E1662905E16729D8A402D0060E996FF3
:106E480081A43BD0060E0FD0938A93809568495051
:106E58007A5D7B51800A4B6E4A50800A4B58D8A005
:106E68008FD7630E0101996F28D09F0E0001806FA4
:106E7800FF0E816FC9EC59F0F4D799514B6E4C6AEB
:106E88004C50000AD8A419D04B50000AD8B465D782
:106E9800010AD8B477D7030AD8B478D7010AD8B486
:106EA800A2D7070AD8B4B5D7010AD8B4B6D7030A07
:106EB800D8B4CAD7640AD8B4D8D7630E01019919CF
:106EC800D8B402D081BC09D7F292F288000E966F2E
:106ED8009380938293849388938A9568899E7AC1D4
:106EE80049F07BC14AF012008980000E6D6EB90E20
:106EF8000001806FF70E816FCFCF82F0836BCECF0A
:106F080084F0856B6E50140D070EF324D96E010EB4
:106F1800F420DA6EDECF86F0DECF87F0DECF88F0A1
:106F2800DECF89F06E50140D070EF324D96E010ED2
:106F3800F420DA6EDECF8AF0DECF8BF0DECF8CF075
:106F4800DECF8DF0C9EC59F024EC3FF0D8C0B1F198
:106F5800D9C0B2F10101B151B211D8B405D0B1C153
:106F6800FAF0B2C1FBF01200000EB36F000EB46F5E
:106F7800000EB56F000EB66F000EAF6F010EAE6F4C
:106F8800000EB96FBCD0000EB86F000EB76F1DD0E1
:106F980019EC5AF00C500D10D8B413D0B90E0C6E71
:106FA800010E0D6EFDEC51F00101AD6F000E712464
:106FB800D96EDA6A040EDA22ADC1DFFF712AB74B47
:106FC800B82B0101B9AB81AC05D0B8BFE1D7B80582
:106FD800D8A0DED7B7C1A9F1B8C1AAF1000EAABFDF
:106FE800FF0EAB6FAC6FB351A925B36FB451AA2193
:106FF800B46FB551AB21B56FB651AC21B66F6E50B9
:10700800140D0F0EF324D96E010EF420DA6EDE5043
:10701800B35DDE50B459DE50B559DE50B659D8A02C
:1070280004D0000EAF6F000EAE6FB9AB04D0000EE7
:10703800AF6F000EAE6F81BC04D0000EAF6F000EB4
:10704800AE6F7150D8B40ED00E0E0001806FFB0EDB
:10705800816FB1C182F0B2C183F071C084F0856BD9
:10706800C9EC59F00101B8BF03D0B805D8B01BD09E
:10707800000E71240C6E0D6A040E0D22FF0E712491
:10708800D96EDA6A030EDA22DF50A96FA9510E6EA3
:107098000F6A71500008106E000ED8A0E82A010887
:1070A800116E0EEC49F017EC53F0EF510101B06F7F
:1070B800B051D8B424D03E0E0001806FFB0E816F12
:1070C800B0C182F0836BC9EC59F0010E6D6E6E5041
:1070D800140D130EF324D96E010EF420DA6E6E50DF
:1070E800140D130EF324E16E010EF420E26EE75046
:1070F8000409DF6E6DC0FAF00001FB6B1200AE519F
:10710800AF11D8A440D7DE0E0001806FF60E816F54
:10711800CFCF82F0836BCECF84F0856BB3C186F07E
:10712800B4C187F0B5C188F0B6C189F0C9EC59F08F
:1071380082A402D0010E6D6E8990000E0001FB6FD3
:10714800000EFA6F120020EE04F04550D926465082
:10715800DA22000EDF6E20EE2AF04550D92646507E
:10716800DA22FF0EDE6EFF0EDE6EFF0EDE6EFF0E03
:10717800DD6E45C03AF046C03BF047C03CF048C021
:107188003DF049C03EF04AC03FF078EC50F00009AD
:10719800D8B402D0030E120022EE2DF04550D926A5
:1071A8004650DA22DF504B6E4B504D6E4C6A22EE41
:1071B8002CF04550D9264650DA22DF504E6E4E50FC
:1071C8004C12000E4D12550E4C1804E1AA0E4D1823
:1071D800D8B402D0020E120020EE65F04550D92630
:1071E8004650DA22DF504B6E4B504D6E4C6A20EE03
:1071F80066F04550D9264650DA22DF504E6E4EC012
:107208004FF0506A516A526A50C052F04FC051F064
:10721800506A4F6A20EE67F04550D9264650DA2268
:10722800DF50536E53C054F0556A566A576A54C0BB
:1072380057F0566A556A546A4F505410586E505059
:107248005510596E515056105A6E525057105B6E69
:107258004C5058105C6E4D5059105D6E000E5A100F
:107268005E6E000E5B105F6E20EE64F04550D9260E
:107278004650DA22DF50606E60505C10616E5D50DF
:10728800626E5E50636E5F50646EFF0E6114656ED1
:10729800FF0E6214666EFF0E6314676E000E6414B0
:1072A800686E460E65180AE1410E661807E1540E2D
:1072B80067186810D8A402D0000E120020EE81F0E2
:1072C8004550D9264650DA22DF504B6E4B504D6E52
:1072D8004C6A20EE82F04550D9264650DA22DF501B
:1072E8004E6E4EC04FF0506A516A526A50C052F00A
:1072F8004FC051F0506A4F6A20EE83F04550D926AE
:107308004650DA22DF50536E53C054F0556A566A1D
:10731800576A54C057F0566A556A546A4F50541009
:10732800586E50505510596E515056105A6E525052
:1073380057105B6E4C5058105C6E4D5059105D6E76
:10734800000E5A105E6E000E5B105F6E20EE80F02D
:107358004550D9264650DA22DF50606E60505C10E6
:10736800616E5D50626E5E50636E5F50646EFF0EBC
:107378006114656EFF0E6214666EFF0E6314676E0D
:10738800000E6414686E460E651808E1410E661812
:1073980005E1540E67186810D8B48ED7010E120094
:1073A8006DAF6E936DBF05D06D5108E16C05D8B017
:1073B80005D0000E3C6E010E3B6E04D06CC13BF054
:1073C8006DC13CF06AC13DF06BC13EF06EA904D0BE
:1073D800FE0E3D26FF0E3E2226C03FF027C040F09D
:1073E80028C041F029C042F02AC043F02BC044F025
:1073F8002CC045F02DC046F0000E486E1F0E476E9B
:10740800000E0201A36F93D04706D8A048060F0EBE
:107418003F14496E4A6A4ABE08D04A5004E10A0E2F
:10742800495CD8A002D0570E01D0300E4924496ECD
:10743800000E4A204A6EBF0E2F6EFF0E306E2E5081
:10744800316E326A2F50312630503222325006E1E6
:107458001A0E315CD8B002D0010E01D0000E376E82
:10746800386A37503810D8B427D09F0E2F6EFF0EC9
:10747800306E200E4910316E000E4A10326E2F50B9
:10748800312630503222325006E11A0E315CD8B023
:1074980002D0010E01D0000E396E3A6A39503A1006
:1074A800D8B40AD049C012F04AC013F027EC56F0FD
:1074B80012C049F013C04AF0840E4724D96E020E58
:1074C8004820DA6E49C0DFFF3B06D8A03C063D06DF
:1074D800D8A03E063FC02FF040C030F041C031F088
:1074E80042C032F043C033F044C034F045C035F0F8
:1074F80046C036F0050E09D0D890363235323432CF
:1075080033323232313230322F32E82EF5D72FC0B3
:107518003FF030C040F031C041F032C042F033C0DB
:1075280043F034C044F035C045F036C046F048BE9C
:1075380021D0485004E1020E475CD8A01BD03F5030
:107548004010411042104310441045104610D8A472
:107558005BD73CBE05D03C5002E13B04D8B054D7C1
:107568003EBE08D03E5003E13D04D8A003D001013F
:107578006EB34AD701016EA916D04706D8A04806AF
:10758800840E4724D96E020E4820DA6E2EC0DFFF23
:107598004706D8A04806840E4724D96E020E482014
:1075A800DA6E300EDF6E25C01BF0840E47241C6E89
:1075B800020E48201D6E3DC01EF03EC01FF08DEC2F
:1075C80052F01BC025F01CC026F01200A40E806FDC
:1075D800FE0E816FAAC082F0ABC083F0A6C084F013
:1075E800A7C085F0A8C086F0A9C087F0C9EC59F0FB
:1075F800000E506E000E4F6ED6D05A0E806FFC0EE5
:10760800816FC9EC59F0000E526E000E516E28D0F1
:107618004FC049F050C04AF0493A4A3AF00E4A166B
:1076280049500F0B4A12F00E4916A6C04BF0A7C0DE
:107638004CF049504B264A504C2251504B24D96E9D
:1076480052504C20DA6EDF504E6E990E806FFF0E4E
:10765800816F4EC082F0836BC9EC59F0514A522AAF
:1076680052BE06D0525020E1100E515CD8B01CD04A
:107678004FC049F050C04AF0493A4A3AF00E4A160B
:1076880049500F0B4A12F00E4916515049265250D4
:107698004A2249500001A85DA951800A4B6E4A5000
:1076A800800A4B58D8B0B4D7DD0E0001806FFF0EAA
:1076B800816FC9EC59F0000E526E000E516E4DD01C
:1076C8004FC049F050C04AF0493A4A3AF00E4A16BB
:1076D80049500F0B4A12F00E4916A6C04BF0A7C02E
:1076E8004CF049504B264A504C2251504B24D96EED
:1076F80052504C20DA6E200EDF6427D0F90E806FCE
:10770800FF0E816F4FC049F050C04AF0493A4A3ADB
:10771800F00E4A1649500F0B4A12F00E4916A6C031
:107728004BF0A7C04CF049504B264A504C225150C0
:107738004B24D96E52504C20DA6EDF504D6E4D50AE
:10774800826F836BC9EC59F006D0FC0E806FFF0E78
:10775800816FC9EC59F0514A522A52BE06D0525094
:1077680020E1100E515CD8B01CD04FC049F050C079
:107778004AF0493A4A3AF00E4A1649500F0B4A1253
:10778800F00E49165150492652504A2249500001DC
:10779800A85DA951800A4B6E4A50800A4B58D8B050
:1077A8008FD74F4A502A50BE06D050501CE1500E79
:1077B8004F5CD8B018D04FC049F050C04AF0493A91
:1077C8004A3AF00E4A1649500F0B4A12F00E491663
:1077D8000001A851495C4A50800A4B6EA951800AA1
:1077E8004B58D8A00AD75A0E0001806FFC0E816F43
:1077F800C9EC59F01200000E0001CC6F010ECB6FDE
:10780800040E806FF70E816F6AC082F0836B6BC0C5
:1078180084F0856B6CC086F0876B6BC0B4F0B56B79
:10782800B66BB76B040ED890B437B537B637B737E1
:10783800E82EF9D76AC0B8F0B96BBA6BBB6B040E07
:10784800D890B837B937BA37BB37E82EF9D7D890B8
:10785800B835BC6FB935BD6FBA35BE6FBB35BF6FB4
:10786800B451BC25C06FB551BD21C16FB651BE2101
:10787800C26FB751BF21C36F6C50C025886F000E0F
:10788800C121896F000EC2218A6F000EC3218B6F40
:10789800C9EC59F0000E0001C76F000EC86F000E4A
:1078A800C96F000ECA6F9FD0040E8C6F020E8D6FC9
:1078B800340E8E6F0B0E8F6F010E916F000E906F4E
:1078C800CF0E926F936BA4EC15F0C46F850E806F8A
:1078D800FC0E816FC4C082F0836BCFC084F0D0C02F
:1078E80085F0C9EC59F07250FD0B726ECFC049F0AB
:1078F800D0C04AF044EC36F049C0CDF04AC0CEF0D2
:107908000001CD51C725C76FCE51C821C86F000EE1
:10791800C921C96F000ECA21CA6F81AC69D0CF5185
:10792800CD1904E1D051CE19D8B40BD0EF0E806F29
:10793800FE0E816FCDC082F0CEC083F0C9EC59F045
:1079480057D010EC59F019EC5AF00C500D10D8B46F
:1079580011D0CA0E0001806FFD0E816F19EC5AF02C
:107968000CC082F00DC083F0C9EC59F0010E010182
:10797800A36F3ED0000E0001C66F050EC56F1FD065
:10798800680E0001B46FE40EE82EFED7B42FFCD7C2
:1079980000F019EC5AF00C500D10D8B410D0000EAD
:1079A8000001CC6F000ECB6FAA0E806FFD0E816FA9
:1079B800C5C082F0C6C083F0C9EC59F009D00001F7
:1079C800C507D8A0C607C529DBE1C629D8A4D8D7DA
:1079D80019EC5AF00C500D10D8B405D0000E000167
:1079E800CC6F000ECB6F0001CB51CC11D8A45CD763
:1079F800E20E0001806FFC0E816FC7C082F0C8C024
:107A080083F0C9C084F0CAC085F0C9EC59F0000EF3
:107A18000101A36F899012004FC00DF050C00EF005
:107A28006BEC51F0556E5550D8A402D120EE04F0FD
:107A38004F50D9265050DA22DFAAFAD04FC0D9FFCA
:107A480050C0DAFFDECF3AF0DDCF3BF020EE1AF07F
:107A58004F50D9265050DA22DECF3CF0DECF3DF031
:107A6800DECF3EF0DECF3FF078EC50F0556E55504B
:107A7800D8A4DED020EE1EF04F50D9265050DA227E
:107A8800DECF5AF0DDCF5BF020EE0BF05A50D9264E
:107A98005B50DA22000EDB8A20EE0AF04F50D9261E
:107AA8005050DA2210EE1CF05A50E1265B50E222C8
:107AB800DFCFE7FF20EE1DF05A50D9265B50DA22BF
:107AC80010EE0AF04F50E1265050E222E6CF51F076
:107AD800E5CF52F052C051F0526A5150DF6E20EE9D
:107AE8001EF05A50D9265B50DA2210EE0AF04F5099
:107AF800E1265050E222E6CF51F0E6CF52F0E6CF31
:107B080053F0E6CF54F0110E05D0D89054325332CA
:107B180052325132E82EF9D75150DF6E20EE1FF065
:107B28005A50D9265B50DA2210EE0AF04F50E1265F
:107B38005050E222E6CF51F0E6CF52F0E6CF53F0B4
:107B4800E6CF54F0190E05D0D89054325332523241
:107B58005132E82EF9D75150DF6E5AC00CF05BC095
:107B68000DF020EE0EF04F50D9265050DA22DECF1D
:107B78000EF0DECF0FF0DECF10F0DECF11F01DECEF
:107B880057F0000E566E000E576E210E586E460EB8
:107B9800596E20EE16F05A50D9265B50DA22000EA4
:107BA800DF6E20EE17F05A50D9265B50DA2257C004
:107BB800DFFF20EE18F05A50D9265B50DA2258C061
:107BC800DFFF20EE19F05A50D9265B50DA2259C04F
:107BD800DFFF20EE12F05A50D9265B50DA22000E51
:107BE800DF6E20EE13F05A50D9265B50DA22000ED1
:107BF800DF6E20EE04F04F50D9265050DA22DF0E07
:107C0800DF164FC0D9FF50C0DAFF10EE04F0DE5087
:107C1800E126DD50E222010EE76E4FC0D9FF50C0C9
:107C2800DAFFDECF44F0DDCF45F03FEC2CF0556EA7
:107C380055501200DB0E0001806FF70E816FCFCF19
:107C480082F0836BCECF84F0856B6EC086F0876B35
:107C5800C9EC59F072500209726E340E0C6E0B0E9C
:107C68000D6E000E0F6E000E0E6E010E116E000EE0
:107C7800106E0EEC49F02BEE34F06EC0DFFFFF0EF5
:107C8800E8CF35FB6E50140D130EF324D96E010E98
:107C9800F420DA6E0101DFA403D0010EE8CF38FB2F
:107CA8006E50140D130EF324D96E010EF420DA6E03
:107CB800DFA003D0020EE8CF3AFB6E50140D130E6E
:107CC800F324D96E010EF420DA6EDFA203D0020E7F
:107CD800E8CF3AFB82A403D0080EE8CF3AFB000EA7
:107CE800526E000E516EA10E0001806FF80E816F6A
:107CF800CFCF82F0836BCECF84F0856B51C086F0F6
:107D080052C087F0360E5124D96E0B0E5220DA6E0F
:107D1800DF504F6E4F50886F896BC9EC59F0500E89
:107D28005124D96E010E5220DA6EDF50FF0A506ED0
:107D3800360E5124D96E0B0E5220DA6E360E5124AF
:107D4800E16E0B0E5220E26EE7505014DF6E5D0EAE
:107D58000001806FFF0E816F360E5124D96E0B0E15
:107D68005220DA6EDF504F6E4F50826F836BC9EC32
:107D780059F0514A522A52BEB6D7525004E1070E62
:107D8800515CD8A0B0D76E50140D130EF324D96EE1
:107D9800010EF420DA6EDF506D6E6E50140D010E78
:107DA800F324D96E010EF420DA6EDF504F6E4FC007
:107DB8003FFB6E50140D020EF324D96E010EF42011
:107DC800DA6EDF504F6E4FC040FB6E50140D030E3D
:107DD800F324D96E010EF420DA6EDF504F6E4FC0D7
:107DE80041FB6E50140D040EF324D96E010EF420DD
:107DF800DA6EDF504F6E4FC042FB6E50140D050E09
:107E0800F324D96E010EF420DA6EDF504F6E4FC0A6
:107E180043FB6E50140D060EF324D96E010EF420A8
:107E2800DA6EDF504F6E4FC044FB000E4A6E140EE0
:107E3800496E44EC36F07250FD0B726E8990120058
:107E48006E50140D070EF324D96E010EF420DA6E6D
:107E5800DECFEBF0DECFECF0DECFEDF0DECFEEF0F4
:107E6800B10E0001806FF60E816FCFCF82F0836B69
:107E7800CECF84F0856BEBC086F0ECC087F0EDC008
:107E880088F0EEC089F0EBC08AF0ECC08BF0EDC052
:107E98008CF0EEC08DF0C9EC59F06E50140D070E41
:107EA800F324D96E010EF420DA6E6E50140D0B0E09
:107EB800F324E16E010EF420E26EDE50E65CDE5043
:107EC800E658DE50E658DE50E658D8B01CD0BE0E54
:107ED8000001806FFC0E816FC9EC59F0010E6D6EC8
:107EE8006E50140D130EF324D96E010EF420DA6EC1
:107EF8006E50140D130EF324E16E010EF420E26EA1
:107F0800E7500409DF6E6E50140D0F0EF324D96E7E
:107F1800010EF420DA6EDECFDAF0DECFDBF0DECF52
:107F2800DCF0DECFDDF06E50140D070EF324D96EB1
:107F3800010EF420DA6EDECFDEF0DECFDFF0DECF2A
:107F4800E0F0DECFE1F00001DA51DE25E26FDB512F
:107F5800DF21E36FDC51E021E46FDD51E121E56FC2
:107F68006E50140D0B0EF324D96E010EF420DA6E48
:107F7800E251DE5CE351DE58E451DE58E551DE584B
:107F8800D8B01BD0AC0E806FFC0E816FC9EC59F0D5
:107F9800010E6D6E6E50140D130EF324D96E010E82
:107FA800F420DA6E6E50140D130EF324E16E010EF8
:107FB800F420E26EE7500409DF6E000E6D6E6E501D
:107FC800200D040EF3240001B16F020EF420B26FED
:107FD800EBC0B3F0ECC0B4F0EDC0B5F0EEC0B6F055
:107FE8009FEC12F0EA6FEA51D8B426D0560E806F93
:107FF800FB0E816FEBC082F0ECC083F0EDC084F023
:10800800EEC085F0EAC086F0876BC9EC59F0010E26
:108018006D6E6E50140D130EF324D96E010EF420FC
:10802800DA6E6E50140D130EF324E16E010EF42077
:10803800E26EE7500409DF6E6DC0D8F00001D96B1D
:10804800120081A605D0E60E0001A66FFD0E04D031
:10805800AF0E0001A66FFF0EA76F81AA04D0E60E2F
:10806800A86FFD0E03D0AA0EA86FFF0EA96F81A8F6
:1080780004D0E60EAA6FFD0E03D0B40EAA6FFF0E51
:10808800AB6F81AE04D0E60EAC6FFD0E03D0B90E17
:10809800AC6FFF0EAD6F81AC04D0E60EAE6FFD0E77
:1080A80003D0A50EAE6FFF0EAF6F81A404D0E60E0D
:1080B800B06FFD0E03D0C30EB06FFF0EB16F81A27B
:1080C80004D0E60EB26FFD0E03D0C80EB26FFF0EDD
:1080D800B36F81A004D0E60EB46FFD0E03D0BE0EC0
:1080E800B46FFF0EB56F83AE04D0E60EB66FFD0E0B
:1080F80003D0F60EB66FFF0EB76F83AC04D0E60E52
:10810800B86FFD0E03D0F30EB86FFF0EB96F83AAD8
:1081180004D0E60EBA6FFD0E03D0F00EBA6FFF0E54
:10812800BB6F83A804D0E60EBC6FFD0E03D0ED0E26
:10813800BC6FFF0EBD6F83A604D0E60EBE6FFD0EAA
:1081480003D0EA0EBE6FFF0EBF6F83A404D0E60E05
:10815800C06FFD0E03D0E70EC06FFF0EC16F83A284
:1081680004D0E60EC26FFD0E03D0E40EC26FFF0E00
:10817800C36F83A004D0E60EC46FFD0E03D0E10EDA
:10818800C46FFF0EC56FCA0E806FF50E816F8350E6
:10819800FF0A496E4950826F836B81CF84F0856BEB
:1081A800C4C086F0C5C087F0C2C088F0C3C089F0DB
:1081B800C0C08AF0C1C08BF0BEC08CF0BFC08DF0CB
:1081C800BCC08EF0BDC08FF0BAC090F0BBC091F0BB
:1081D800B8C092F0B9C093F0B6C094F0B7C095F0AB
:1081E800B4C096F0B5C097F0B2C098F0B3C099F09B
:1081F800B0C09AF0B1C09BF0AEC09CF0AFC09DF08B
:10820800ACC09EF0ADC09FF0AAC0A0F0ABC0A1F07A
:10821800A8C0A2F0A9C0A3F0A6C0A4F0A7C0A5F06A
:10822800C9EC59F012001C6E1C50D8B402D0010ED3
:10823800120073A202D073501200000E8DEC59F098
:108248000A0E276E03D012EC5AF027062750D8A43E
:10825800FAD7000E246E000E156E000E166E000E74
:10826800176E000E186E000E3EEC57F0E806D8A404
:10827800BDD0AA0E156E010E166E000E176E000EFA
:10828800186E080E3EEC57F0E806D8A462D0000E2F
:10829800276E27501D0FD96EDA6A12EC5AF0DF6E7E
:1082A800272A030E2764F5D71F04D8A49FD0AA0E47
:1082B8002018D8A49BD0030E266EE80E256E19D080
:1082C800000E156E000E166E000E176E400E186E1C
:1082D800A90E3EEC57F00009D8B40FD00B0E1B6E58
:1082E800620EE82EFED71B2EFCD700D02506D8A09C
:1082F800260625502610D8A4E3D725502610D8B432
:1083080075D0000E156E000E166E000E176E000E5C
:10831800186E3A0E3EEC57F00009D8A467D0000E4C
:10832800276E27501D0FD96EDA6A12EC5AF0DF6EED
:10833800272A030E2764F5D71DBC04D0000E226E31
:10834800040E03D0000E226E0C0E216E21C024F004
:108358004DD0000E156E000E166E000E176E000E34
:10836800186EA90E3EEC57F01B6E020E1B6004D06F
:10837800020E246EA90E03D0010E246E010E236E88
:10838800030E266EE80E256E19D0000E156E000E2F
:10839800166E000E176E000E186E23503EEC57F046
:1083A8000009D8B40FD00B0E1B6E620EE82EFED754
:1083B8001B2EFCD700D02506D8A02606255026104F
:1083C800D8A4E3D725502610D8B40ED0000E156EC9
:1083D800020E166E000E176E000E186E100E3EEC92
:1083E80057F00009D8B402D0000E246E24C06FF0F4
:1083F8001EEC5AF02450D8B41ED773901CD76CC00A
:10840800D8F00001D96BDA6BDB6BDAC0DBF0D9C0CE
:10841800DAF0D8C0D9F0D86B6BC0DCF0DD6BDE6B5E
:10842800DF6BDEC0DFF0DDC0DEF0DCC0DDF0DC6B72
:10843800040ED890DC37DD37DE37DF37E82EF9D782
:108448006AC0E0F0E16BE26BE36B040ED890E037B2
:10845800E137E237E337E82EF9D7E2C0E3F0E1C0CD
:10846800E2F0E0C0E1F0E06BD890E035E46FE13590
:10847800E56FE235E66FE335E76FDC51E425E86F39
:10848800DD51E521E96FDE51E621EA6FDF51E72191
:10849800EB6FD851E825ED6FD951E921EE6FDA512C
:1084A800EA21EF6FDB51EB21F06F200E806FF90EA0
:1084B800816F69C082F0836B6AC084F0856B6BC082
:1084C80086F0876B6CC088F0896B6BC0D8F0D96B6D
:1084D800DA6BDB6B040ED890D837D937DA37DB374D
:1084E800E82EF9D76AC0DCF0DD6BDE6BDF6B040EBB
:1084F800D890DC37DD37DE37DF37E82EF9D7D8906C
:10850800DC35E06FDD35E16FDE35E26FDF35E36FD7
:10851800D851E025E46FD951E121E56FDA51E22124
:10852800E66FDB51E321E76F6C50E4258A6F000E9C
:10853800E5218B6F000EE6218C6F000EE7218D6F11
:10854800C9EC59F0CA0E0001806FFB0E816FEDC0B7
:1085580082F0EEC083F0EFC084F0F0C085F0EDC08B
:1085680086F0EEC087F0EFC088F0F0C089F0C9EC63
:1085780059F0040E0001B16F020EB26FEDC0B3F0F6
:10858800EEC0B4F0EFC0B5F0F0C0B6F09FEC12F05A
:10859800EC6FEC51D8B411D0560E806FFB0E816F82
:1085A800EDC082F0EEC083F0EFC084F0F0C085F03B
:1085B800ECC086F0876BC9EC59F0000E0101A36F7F
:1085C80089901200CCC0F6FFCDC0F7FF000EF86E00
:1085D8000F0EF76403D00800F55005D0F6CFE9FF79
:1085E800F7CFEAFFEF502F0AD8B414D0CCC0F6FF6B
:1085F800CDC0F7FF000EF86E0F0EF76403D0080029
:10860800F55005D0F6CFE9FFF7CFEAFFEF505C0A47
:10861800D8A403D00001CC4BCD2B000120EE06F0EE
:10862800CA51D926CB51DA22DE6ADE6ADE6ADD6AF1
:10863800CCC0F6FFCDC0F7FF000EF86E0F0EF76442
:1086480003D00800F55005D0F6CFE9FFF7CFEAFFD1
:10865800EF500001CE6F200ECE6116D0CAC065F073
:10866800CBC066F0000E686E000E676EA8EC33F0A3
:10867800D26F20EE12F0CA51D926CB51DA22000E61
:10868800DE6E000EDD6E5FD0CAC014F0CBC015F0F0
:10869800CC0E166ED6EC30F00001D26FD251D8A4B1
:1086A80052D0CAC0C4F0CBC0C5F061EC4DF0D26F57
:1086B80020EE14F0CA51D926CB51DA2210EE0BF075
:1086C800DE50E126DD50E222E750D16FD251D8B416
:1086D80008D0040ED219D8B4D1B535D0050ED26F52
:1086E80032D0D1B530D020EE12F0CA51D926CB51B4
:1086F800DA22DECFCFF0DDCFD0F020EE0BF0CF5175
:10870800D926D051DA22DFA8E9D7CAC0D9FFCBC011
:10871800DAFFDECF0CF0DDCF0DF0CFC00EF0D0C009
:108728000FF00DEC4FF0000120EE06F0CA51D926EB
:10873800CB51DA220CC0DEFF0DC0DEFF0EC0DEFF1B
:108748000FC0DEFFA1D7D2511200000E6E6E000ED0
:108758006E6E030E6E6401D0A2D06E50140D130E0F
:10876800F324D96E010EF420DA6E000EDF6E6E501F
:10877800140D000EF324D96E010EF420DA6E000EEB
:10878800DF6E6E50140D070EF324D96E010EF4201F
:10879800DA6EDE6ADE6ADE6ADD6AE3C249F04A6AD8
:1087A8004B6A4C6A4BC04CF04AC04BF049C04AF087
:1087B800496AE2C24DF04E6A4F6A506A4EC050F0A4
:1087C8004DC04FF04E6A4D6AE1C251F0526A536A89
:1087D800546A51C054F0536A526A516A0201E05116
:1087E8005124556E000E5220566E000E5320576EBF
:1087F800000E5420586E4D505524596E4E50562038
:108808005A6E4F5057205B6E505058205C6E49503E
:1088180059245D6E4A505A205E6E4B505B205F6E45
:108828004C505C20606E6E50140D0B0EF324D96E04
:10883800010EF420DA6E5DC0DEFF5EC0DEFF5FC0B1
:10884800DEFF60C0DEFF810E0001806FF80E816FD1
:108858006EC082F0836B6E50140D0B0EF324D96E2C
:10886800010EF420DA6EDECF84F0DECF85F0DECFA5
:1088780086F0DECF87F06E50140D0B0EF324D96E00
:10888800010EF420DA6EDECF88F0DECF89F0DECF7D
:108898008AF0DECF8BF0C9EC59F06E2A5AD7000E59
:1088A80001018A6F000E0001FC6F000E01019C6F30
:1088B800000E896F000E736F000E726F020E6D6EE0
:1088C800899012004C50D96EDA6ADECFF6FFDDCF00
:1088D800F7FF0800F550250AD8A494D04C50D96E5B
:1088E800DA6ADE2A000EDD22000E01016B6F000E2F
:1088F8006A6F6AC16EF16BC16FF16C696D694C503A
:10890800D96EDA6ADECFF6FFDDCFF7FF0800F55043
:10891800780AD8B40CD04C50D96EDA6ADECFF6FF9C
:10892800DDCFF7FF0800F550580AD8A441D04C50C5
:10893800D96EDA6ADECFF6FFDDCFF7FF0800F5CF94
:1089480058F04C50D96EDA6ADE2A000EDD224D50FE
:10895800D96EDA6ADF50DF2ADF2AD96EDA6ADECF0B
:108968004EF0DDCF4FF04EC050F04FC051F0526A7C
:10897800536A546A556A566A576A4BC025F050C004
:1089880026F051C027F052C028F053C029F054C037
:108998002AF055C02BF056C02CF057C02DF058C007
:1089A8002EF0D4EC39F025C04BF026C04CF0120064
:1089B8004C50D96EDA6ADECFF6FFDDCFF7FF08003C
:1089C800F550250AD8A413D04C50D96EDA6ADE2A9D
:1089D800000EDD22000E0E6E250E0D6E4BC00FF040
:1089E80045EC52F0000E4C6E010E4B6E12004C50CE
:1089F800D96EDA6ADE2A000EDD22000E4C6E000EF9
:108A08004B6E12004C50D96EDA6ADECFF6FFDDCF1E
:108A1800F7FF0800F5500D6E0E6A4BC00FF045ECDD
:108A280052F04C50D96EDA6ADE2A000EDD22DAD70F
:108A3800960E0001806FF70E816F6AC082F0836B1B
:108A48006BC084F0856B6CC086F0876B6BC0A9F136
:108A58000101AA6BAB6BAC6B040ED890A937AA378F
:108A6800AB37AC37E82EF9D76AC0ADF1AE6BAF6B58
:108A7800B06B040ED890AD37AE37AF37B037E82EAD
:108A8800F9D7D890AD35B16FAE35B26FAF35B36F9A
:108A9800B035B46FA951B125B56FAA51B221B66FDF
:108AA800AB51B321B76FAC51B421B86F6C50B52539
:108AB8000001886F000E0101B6210001896F000EC8
:108AC8000101B72100018A6F000E0101B8210001E0
:108AD8008B6FC9EC59F0000E0001F46F000EF36FB4
:108AE800000EF56F1CD019EC5AF00C500D10D8B4CC
:108AF80012D0F50E0C6E0D6AFDEC51F00001F16F0D
:108B0800000E7124D96EDA6A040EDA22F1C0DFFF92
:108B1800712AF34BF42B0001F5AB81AC05D0F4BFFF
:108B2800E2D7F405D8A0DFD7F3C0F6F0F4C0F7F029
:108B380082B411D0040EB16F020EB26F000EB36F83
:108B4800040EB46F010EB66F000EB56FF60EB76F58
:108B580012EC0FF0F26FF251D8B409D0BA0E806F50
:108B6800FD0E816FF2C082F0836BC9EC59F0F50EEF
:108B78000001806FFA0E816FF6C082F0F7C083F0B3
:108B8800C9EC59F071EC48F0000EA36F89901200FF
:108B98000600D9CF05F0DACF06F0F2A01CD081BCD0
:108BA80002D08994899281A802D089A20FD0939487
:108BB80025EE04F0010EDBBE08D0000EDE5C020ECE
:108BC800DE58D8A002D0939201D0938281B889B29E
:108BD80001D09384F290F2B281B083D081B889B287
:108BE80093928350FF0A096E8150FF0A086E04C5EC
:108BF8000AF005C50BF00BBE04D0020E0B5CD8B012
:108C08002CD00A4A0B2A0AC004F50BC005F502C588
:108C18000AF003C50BF0060E0A24D96E050E0B20C8
:108C2800DA6E09C0DFFF060E0A24D96E070E0B2084
:108C3800DA6E08C0DFFF0A4A0B2AFF0E016E010E2A
:108C4800026E0AC003F00BC004F001500316025074
:108C5800041603C002F504C003F581B889B29384F1
:108C6800938481A0FED781A802D089A202D09394D0
:108C780001D0938425EE04F0010EDBBE08D0000E6F
:108C8800DE5C020EDE58D8A002D0939201D0938207
:108C980008B80CD025D0898202D0898405D089945F
:108CA8001FD089A21DD0899489921AD00950016ECB
:108CB800026A0250000AD8A413D00150040AD8B49A
:108CC800F0D7100AD8B4EDD7340AD8B4E4D71F0ABD
:108CD800D8B4EAD77F0AD8B4E0D71F0AD8B4DFD708
:108CE800F29206C0DAFF05C0D9FF74921100000E97
:108CF800336E20EE04F02550D9262650DA22DF50B4
:108D0800D8B49FD020EE2AF02550D9262650DA2252
:108D1800DECF36F0DECF37F0DECF38F0DECF39F0F9
:108D28002E0E25241B6E000E26201C6E36C01DF04C
:108D380037C01EF038C01FF039C020F0000E226E78
:108D4800010E216E20EE01F02550D9262650DA2298
:108D5800DF5065EC4BF00009D8B403D0010E336E38
:108D680070D020EE04F02550D9262650DA22000EC5
:108D7800DF6E20EE16F02550D9262650DA2210EEA6
:108D88001EF02550E1262650E222E6CF2BF0E6CF52
:108D98002CF0E6CF2DF0E6CF2EF02B50365C2F6E60
:108DA8002C503758306E2D503858316E2E50395857
:108DB800326EDE502F5CDE503058DE503158DE50B7
:108DC8003258D8B03ED020EE03F02550D926265090
:108DD800DA22DF50276E2750346E356A355004E1A9
:108DE800020E345CD8A02DD020EE16F02550D926DE
:108DF8002650DA22DE503626DE503722DE50382260
:108E0800DD5039222E0E25241B6E000E26201C6EE6
:108E180036C01DF037C01EF038C01FF039C020F032
:108E2800000E226E010E216E20EE01F02550D9268B
:108E38002650DA22DF5065EC4BF03406D8A0350610
:108E4800CDD7335012004F0E0001806FF70E816F9F
:108E58006AC082F0836B6BC084F0856B6CC086F04F
:108E6800876B6BC0B4F0B56BB66BB76B040ED8905C
:108E7800B437B537B637B737E82EF9D76AC0B8F080
:108E8800B96BBA6BBB6B040ED890B837B937BA3721
:108E9800BB37E82EF9D7D890B835BC6FB935BD6F58
:108EA800BA35BE6FBB35BF6FB451BC25C06FB55165
:108EB800BD21C16FB651BE21C26FB751BF21C36F6B
:108EC8006C50C025886F000EC121896F000EC22129
:108ED8008A6F000EC3218B6FC9EC59F0000E000198
:108EE800C76F000EC86F000EC96F000ECA6F040E60
:108EF8008C6F020E8D6F340E8E6F0B0E8F6F010EFE
:108F0800916F000E906FCB0E926F936BA4EC15F0DF
:108F1800C66F600E806FF80E816FC6C082F0836BDB
:108F2800CBC084F0CCC085F0C9EC59F07250FD0B71
:108F3800726E010E0101A56FCBC049F0CCC04AF09A
:108F480044EC36F049C0C4F04AC0C5F0000E010137
:108F5800A56F0001C451C725C76FC551C821C86F87
:108F6800000EC921C96F000ECA21CA6FE20E806FB8
:108F7800FC0E816FC7C082F0C8C083F0C9C084F0FE
:108F8800CAC085F0C9EC59F0000E0101A36F8990A1
:108F980012000001A351A211A11104E1020EA05D6B
:108FA800D8A010D020EE12F09E51D9269F51DA2277
:108FB800DE50A05DDE50A159DE50A259DE50A35903
:108FC800D8A002D0020E30D0000EA46F74D09EC07C
:108FD80045F09FC046F0A0C047F0A1C048F0A2C02D
:108FE80049F0A3C04AF0E3EC21F045C0A5F046C023
:108FF800A6F047C0A7F048C0A8F00001A551A611E7
:10900800A711A811D8B467D0A505A611A711A81152
:10901800D8B4D8D7A5290AE1A62908E1A72906E1E5
:10902800A829D8A403D0010EA46F55D09EC045F03E
:109038009FC046F0A0C047F0A1C048F0A2C049F0C8
:10904800A3C04AF0000E4B6E000E4C6E000E4D6E23
:10905800000E4E6EF1EC1AF00001A46FA451D8A4D2
:109068003AD020EE0EF09E51D9269F51DA22DE2802
:1090780007E1DE2805E1DE2803E1DE28D8B413D0B5
:1090880020EE0EF09E51D9269F51DA22DE2A000EDC
:10909800DE22DE22DE2220EE05F09E51D9269F51E7
:1090A800DA22000EDB80A5C0A0F0A6C0A1F0A7C000
:1090B800A2F0A8C0A3F020EE12F09E51D9269F512D
:1090C800DA22DE50A05DDE50A159DE50A259DE50F2
:1090D800A359D8A07CD7A45112006C2A0F0E6C6437
:1090E80009D0000E6C6E6B2A010E6B6403D0000E63
:1090F8006B6E6A2A6CC0D8F00001D96BDA6BDB6B37
:10910800DAC0DBF0D9C0DAF0D8C0D9F0D86B6BC0C0
:10911800DCF0DD6BDE6BDF6BDEC0DFF0DDC0DEF0C8
:10912800DCC0DDF0DC6B040ED890DC37DD37DE37D1
:10913800DF37E82EF9D76AC0E0F0E16BE26BE36B4A
:10914800040ED890E037E137E237E337E82EF9D755
:10915800E2C0E3F0E1C0E2F0E0C0E1F0E06BD890FB
:10916800E035E46FE135E56FE235E66FE335E76F4B
:10917800DC51E425E86FDD51E521E96FDE51E62198
:10918800EA6FDF51E721EB6FD851E825EC6FD95131
:10919800E921ED6FDA51EA21EE6FDB51EB21EF6F38
:1091A800C20E806FFA0E816F69C082F0836B6AC04D
:1091B80084F0856B6BC086F0876B6CC088F0896B18
:1091C800C9EC59F0040E0001B16F020EB26FECC089
:1091D800B3F0EDC0B4F0EEC0B5F0EFC0B6F09FEC60
:1091E80012F0F06FF051D8B411D0560E806FFB0E0C
:1091F800816FECC082F0EDC083F0EEC084F0EFC068
:1092080085F0F0C086F0876BC9EC59F0000E0101BB
:10921800A36F12000CC016F00DC017F010501110FB
:10922800D8B4120016C0D9FF17C0DAFF0EC0DFFF8E
:1092380010501624126E11501720136EFF0E1224B0
:10924800D96EFF0E1320DA6E0EC0DFFF115004E155
:10925800030E105CD8A0120020EE01F01650D9269B
:109268001750DA220EC0DFFF20EE02F01650D92682
:109278001750DA220EC0DFFF10501624126E11505C
:109288001720136EFE0E1224D96EFF0E1320DA6E0D
:109298000EC0DFFF10501624126E11501720136EE7
:1092A800FD0E1224D96EFF0E1320DA6E0EC0DFFFFA
:1092B800115004E1070E105CD8A0120020EE03F054
:1092C8001650D9261750DA220EC0DFFF1050162488
:1092D800126E11501720136EFC0E1224D96EFF0E59
:1092E8001320DA6E0EC0DFFF115004E1090E105C86
:1092F800D8A0120016C012F017C013F0121E131EC9
:10930800124A132A030E1214146E156A14501626E4
:10931800155017221450105E1550115AFC0E1016D5
:10932800FF0E11160BD016C0D9FF17C0DAFF0EC0FA
:10933800DFFF1006D8A01106164A172A1050111080
:10934800D8B41200F0D7146815680C50D96EDA6AD0
:10935800DE50DE10D8B486D00C50D96EDA6ADECF73
:1093680018F0DDCF19F002D0184A192A18C0F6FFF4
:1093780019C0F7FF000EF86E0F0EF76403D008004F
:10938800F55005D0F6CFE9FFF7CFEAFFEF500E6EA4
:10939800200E0E6414D018C0F6FF19C0F7FF000E97
:1093A800F86E0F0EF76403D00800F55005D0F6CF1D
:1093B800E9FFF7CFEAFFEF503A0AD8A4D5D718C08B
:1093C800F6FF19C0F7FF000EF86E0F0EF76403D012
:1093D8000800F55005D0F6CFE9FFF7CFEAFFEF50C8
:1093E8003A0AD8A444D00C50D96EDA6ADECF12F00B
:1093F800DDCF13F012C0F6FF13C0F7FF000EF86EB2
:109408000F0EF76403D00800F55005D0F6CFE9FF3A
:10941800F7CFEAFFEF500E6ED00E0E24166E176AC5
:10942800FF0E1722124A132A17501CE10A0E165C67
:10943800D8B018D01850121815E119501318D8A41C
:1094480011D016501710D8A40DD016C014F017C09C
:1094580015F0184A192A0C50D96EDA6A18C0DEFFBE
:1094680019C0DDFF14C00CF015C00DF01200000E7D
:10947800156E000E146EF6D7000E216E000E206ECB
:10948800000E1A6E000E196E01D0132A010E1F6EFF
:109498001350D96EDA6A200EDE18D8B416D0F70E3B
:1094A800156EFF0E166E1350D96EDA6ADF50176EFE
:1094B800186A1550172616501822185004E1050E80
:1094C800175CD8A002D0000E1F6E1FC01BF01C6ACC
:1094D8001B501C10D8B407D0D8D7000E1A6E010E36
:1094E800196E132A2CD01350D96EDA6ADF50156E14
:1094F800166A1650000AD8A422D015502B0AD8B4E0
:10950800F0D7060AD8B4E9D71AD020C00CF021C089
:109518000DF0000E0F6E0A0E0E6E23EC59F013506C
:10952800D96EDA6ADF50156E15500C5E000E0D5AB2
:10953800300E0C24206E000E0D20216ED2D7D00ED6
:10954800156EFF0E166E1350D96EDA6ADF50176E5D
:10955800186A1550172616501822185006E10A0ED8
:10956800175CD8B002D0010E01D0000E1D6E1E6A25
:109578001D501E10D8A4C9D719501A10D8A40DD040
:1095880020C015F021C016F0151E161E154A162A01
:1095980015C013F016C014F0120020C013F021C03B
:1095A80014F012002F6C696664617461302E626970
:1095B8006E20002F6C696664617461312E62696E79
:1095C80020002F6C696664617461322E62696E20B6
:1095D800002F6C696664617461332E62696E2000C5
:1095E8002F6C696664617461342E62696E20002F85
:1095F8006C696664617461352E62696E20002F6C37
:10960800696664617461362E62696E20002F6C6928
:109618006664617461372E62696E20002F6C69661A
:1096280064617461382E62696E20002F6C6966640B
:10963800617461392E62696E20002F6C69666461FD
:109648007461612E62696E20002F6C6966646174B2
:1096580061622E62696E20002F6C696664617461B4
:10966800632E62696E20002F6C69666461746164A0
:109678002E62696E20002F6C696664617461652EC4
:1096880062696E20002F6C696664617461662E627F
:10969800696E2000000000000000000000000000CB
:1096A80000000000000000000000000000000000B2
:1096B80000000000000000000000000000000000A2
:0196C80000A1
:1096CA00246E2450D8A404D021502210D8A402D049
:1096DA00040E120073A002D0030E120073A402D06B
:1096EA00020E12006FB608D0090ED8901D361E362B
:1096FA001F362036E82EF9D721042210D8A41DD00F
:10970A001DC015F01EC016F01FC017F020C018F0BB
:10971A00180E3EEC57F00009D8A44FD01BC00EF02B
:10972A001CC00FF0FE0E106E4FEC55F00009D8B4B5
:10973A0044D0000E226E000E3FD06FC023F0060EFA
:10974A002316D8B409D021C015F022C016F0176A22
:10975A00186A970E3EEC57F01DC015F01EC016F0A1
:10976A001FC017F020C018F0190E3EEC57F0000980
:10977A00D8A423D01BC00EF01CC00FF0FC0E106E34
:10978A004FEC55F00009D8B409D0020E1C26210668
:10979A00D8A0220621502210D8A4ECD7000E0E6EB3
:1097AA00000E0F6EFD0E106E4FEC55F00009D8A496
:1097BA0004D0000E226E010E216E1EEC5AF02150CA
:1097CA002210D8B402D0010E1200000E1200AC0E04
:1097DA00F66E950EF76E000EF86E0DEE34F011EE81
:1097EA001DF00900F5CFEEFFE550E150FAE1E25035
:1097FA00F8E1FA0EF66EB20EF76E000EF86E03EE90
:10980A00C0F010EE20F00900F5CFEEFFE550E15070
:10981A00FAE1E00EF66EAC0EF76E000EF86E02EE8E
:10982A00A4F010EE46F00900F5CFEEFFE550E15046
:10983A00FAE15A0EF66EB40EF76E000EF86E0900D3
:10984A00F5CFDEF10900F5CFDFF10900F5CFE0F140
:10985A00620EF66EB40EF76E000EF86E0900F5CFC2
:10986A0073F005EE00F018EE34F0EE6AE550E150C0
:10987A00FCE1E250FAE104EE00F011EE00F0EE6ACB
:10988A00E550E150FCE1E250FAE103EE00F0C00ECF
:10989A00EE6AE806FDE102EE00F0A40EEE6AE806C2
:1098AA00FDE101EE00F0A90EEE6AE806FDE1000115
:1098BA00FD6BFC6B00EE69F0090EEE6AE806FDE14D
:1098CA0074907492000EF86E0001A1EF07F089807F
:1098DA00000E0C6E040E0D6E000E0F6EF60E0E6E5E
:1098EA00010E116E000E106E0EEC49F07C0E000196
:1098FA00806FFE0E816FC9EC59F0000E0001F66F01
:10990A00000EF56F2E0EDEEC59F082B412D0040E62
:10991A000001B16F020EB26F000EB36F040EB46F86
:10992A00010EB66F000EB56FF20EB76F12EC0FF0A4
:10993A00F46F0001F451D8B40AD0800E806FFF0E84
:10994A00816FF4C082F0836BC9EC59F0120019ECF4
:10995A005AF00C500D10D8B427D0F70E0C6E0D6AC1
:10996A00FDEC51F00001F16FF751100B496E000E3A
:10997A004A6EF15112EC24F049C0F8F04AC0F9F0ED
:10998A00040E0001F819F911D8B493EC56F0020E3E
:10999A000001F819F911D8B4BBEC54F00001F8052C
:1099AA00F911D8B403EC42F00001F54BF62BF6514D
:1099BA0004E1C80EF55DD8A0A5D7270E806FFF0E6B
:1099CA00816FC9EC59F089901200C4C065F0C5C016
:1099DA0066F0000E686E000E676EA8EC33F0CD6F6D
:1099EA00CD51D8A461D0000ECC6F000ECB6FC4C08D
:1099FA00D9FFC5C0DAFFDECF3AF0DDCF3BF020EE6B
:109A0A000EF0C451D926C551DA22DECF3CF0DECFA2
:109A1A003DF0DECF3EF0DECF3FF078EC50F00001B3
:109A2A00CD6FCD51D8A440D020EE12F0C451D92622
:109A3A00C551DA22DECFC8F0DDCFC9F0C8C0D9FFE0
:109A4A00C9C0DAFFE50EDE18D8B411D020EE12F044
:109A5A00C451D926C551DA22DECFC8F0DDCFC9F00C
:109A6A00C8C0D9FFC9C0DAFFDF50D8A40AD0CB4B8F
:109A7A00CC2BC651CB1909E1C751CC19D8B414D093
:109A8A0004D0000ECC6F000ECB6FC4C0B1F0C5C0BD
:109A9A00B2F0000EB46F010EB36F4FEC28F0000164
:109AAA00CD6FCD51D8B4A3D7040ECD19D8A402D006
:109ABA00070ECD6FCD511200C4C065F0C5C066F067
:109ACA00000E686E000E676EA8EC33F0C96FC951BC
:109ADA00D8B402D0C9511200C4C0D9FFC5C0DAFF38
:109AEA00DECF3AF0DDCF3BF020EE0EF0C451D9269E
:109AFA00C551DA22DECF3CF0DECF3DF0DECF3EF0BC
:109B0A00DECF3FF078EC50F00001C96FC951D8A4FC
:109B1A00E1D720EE12F0C451D926C551DA22DECFA0
:109B2A00C7F0DDCFC8F0C7C0D9FFC8C0DAFFDF5021
:109B3A00C66FC651D8A403D0040EC96FCBD720EE86
:109B4A000BF0C751D926C851DA22DFB618D0C7C0E0
:109B5A000CF0C8C00DF020EE14F0C451D926C5513E
:109B6A00DA22DECF0EF0DDCF0FF0000E116E0B0EF3
:109B7A00106E55EC54F00C500D10D8B4ABD7C4C0CD
:109B8A00B1F0C5C0B2F0000EB46F000EB36F4FEC67
:109B9A0028F00001C96FC951D8A49CD79DD76E502F
:109BAA00140D070EF324D96E010EF420DA6E000E9E
:109BBA00DE24D86F010EDE20D96F000EDE20DA6FA8
:109BCA00000EDE20DB6F6E50140D070EF324D96EE3
:109BDA00010EF420DA6ED8C0DEFFD9C0DEFFDAC08B
:109BEA00DEFFDBC0DEFF6E50140D070EF324D96EC4
:109BFA00010EF420DA6EDECFDDF0DDCFDEF04F0E9F
:109C0A00806FF60E816FCFCF82F0836BCECF84F058
:109C1A00856BDDC086F0DEC087F0DDC088F0DEC06F
:109C2A0089F0C9EC59F06E50200D040EF32400019E
:109C3A00B16F020EF420B26FDDC0B3F0DEC0B4F033
:109C4A00B56BB66B9FEC12F0DC6FDC51D8B410D058
:109C5A00560E806FFB0E816FDDC082F0DEC083F08E
:109C6A00DCC084F0856BC9EC59F0010E6D6E1200F0
:109C7A00000E6D6E1200CEC0C4F0CFC0C5F0000E4B
:109C8A00C76F010EC66FEAEC4CF0D06FD051D8A462
:109C9A0058D0CEC0D9FFCFC0DAFFDECF3AF0DDCF41
:109CAA003BF020EE0EF0CE51D926CF51DA22DECF8C
:109CBA003CF0DECF3DF0DECF3EF0DECF3FF078EC79
:109CCA0050F00001D06FD051D8A43BD020EE12F052
:109CDA00CE51D926CF51DA22DECF0CF0DDCF0DF0EE
:109CEA00000E0F6E000E0E6E000E116E200E106E1C
:109CFA00E6EC58F0000120EE12F0CE51D926CF51F1
:109D0A00DA22DECF0CF0DDCF0DF020EE14F0CE51CA
:109D1A00D926CF51DA22DECF0EF0DDCF0FF0000EBA
:109D2A00116E0B0E106E5FEC57F0CEC0D9FFCFC08C
:109D3A00DAFF10EE04F0DE50E126DD50E222010ED9
:109D4A00E76ED0511200236E2350D8A404D02150BC
:109D5A002210D8A402D0040E120073A002D0030E5F
:109D6A0012006FB608D0090ED8901D361E361F365F
:109D7A002036E82EF9D7225008E1020E215CD8B02D
:109D8A0004D0000E256E110E03D0000E256E120EA1
:109D9A00246E24C026F01DC015F01EC016F01FC088
:109DAA0017F020C018F026503EEC57F00009D8A44E
:109DBA0025D01BC00CF01CC00DF0020E0F6E000E59
:109DCA000E6EEDEC54F00009D8B409D0020E1C2630
:109DDA002106D8A0220621502210D8A4EAD7120EB2
:109DEA002618D8A40BD0000E156E000E166E000EA3
:109DFA00176E000E186E0C0E3EEC57F01EEC5AF061
:109E0A0021502210D8B402D0010E1200000E120006
:109E1A001A0E0E24106E000E0F20116E010E102461
:109E2A00D96E000E1120DA6EDF50126E1250146EC7
:109E3A00136A1A0E0E24D96E000E0F20DA6EDF5046
:109E4A00156E15501312000E141213C01AF014C016
:109E5A001BF01C6A1D6A0CC0D9FF0DC0DAFF030E85
:109E6A00DE18D8A42ED0140E0E24106E000E0F2069
:109E7A00116E010E1024D96E000E1120DA6EDF5019
:109E8A00126E1250146E136A140E0E24D96E000E3E
:109E9A000F20DA6EDF50156E15501310166E14501F
:109EAA00176E186A196A17C019F016C018F0176ADF
:109EBA00166A16501A1217501B1218501C121950F3
:109ECA001D121AC00CF01BC00DF01CC00EF01DC0F4
:109EDA000FF01200020E1A5E000E1B5A1C5A1D5A6F
:109EEA0020EE12F01850D9261950DA22FE0EDE247E
:109EFA001E6EFF0EDE201F6EFF0EDE20206EFF0E8E
:109F0A00DE20216E1E501A5C1F501B5820501C5810
:109F1A0021501D58D8A009D0000E186E000E196ED7
:109F2A00000E1A6E000E1B6E120020EE26F018505C
:109F3A00D9261950DA22DECF1EF0DECF1FF0DECF8F
:109F4A0020F0DECF21F020EE02F01850D926195069
:109F5A00DA22DF50226E22500C6E0D6A0E6A0F6AE8
:109F6A001AC010F01BC011F01CC012F01DC013F073
:109F7A00ACEC55F01E500C24186E1F500D20196EB3
:109F8A0020500E201A6E21500F201B6E120017EC63
:109F9A0058F0CC0EBBEC59F0660EBBEC59F06CECE9
:109FAA0059F04F6E4F50D8A409D0000E496E000EDA
:109FBA004A6E000E4B6E000E4C6E1200000E4E6E74
:109FCA00000E4D6E4D504F0FD96EDA6A6CEC59F097
:109FDA00DF6E4D4A4E2A4EBEF5D74E5004E1040EAE
:109FEA004D5CD8A0EFD7210E0001806FFC0E816F67
:109FFA004FC082F0836B50C084F0856B51C086F0ED
:10A00A00876B52C088F0896B4FC08AF050C08BF0C2
:10A01A0051C08CF052C08DF0C9EC59F05250511019
:10A02A00501004E10B0E4F5CD8A0BFD74FC049F0C7
:10A03A0050C04AF051C04BF052C04CF01200DAC086
:10A04A00E0F0DBC0E1F0E00E0C6EA7EC49F00CC0CA
:10A05A00E2F00DC0E3F00001E3AF02D00B0E1200F4
:10A06A00D890E235D96EE335DA6E820ED926010E22
:10A07A00DA22DECFDEF0DDCFDFF0DE51DF11D8B439
:10A08A0006D0DEC0D9FFDFC0DAFF000EDF6ED8517E
:10A09A00D911D8B406D0D8C0D9FFD9C0DAFF000E7A
:10A0AA00DF6ED890E235D96EE335DA6E820ED926A4
:10A0BA00010EDA22D8C0DEFFD9C0DDFFD851D9118E
:10A0CA00D8B403D0DC05D8B402D0000E1200D80EE2
:10A0DA00806F816BDA0E826F000E836F09EC00F0DD
:10A0EA00DD6FDD511200000E446E20EE2AF03A5068
:10A0FA00D9263B50DA223C50DE180AE13D50DE18E0
:10A10A0007E13E50DE1804E13F50DE18D8B43CD0D7
:10A11A003AC025F03BC026F07BEC46F0446E445032
:10A12A00D8A432D02E0E3A241B6E000E3B201C6E91
:10A13A003CC01DF03DC01EF03EC01FF03FC020F0E5
:10A14A00000E226E010E216E20EE01F03A50D92641
:10A15A003B50DA22DF50A8EC4EF00009D8B406D002
:10A16A003C683D683E683F68010E446E20EE2AF066
:10A17A003A50D9263B50DA223CC0DEFF3DC0DEFF12
:10A18A003EC0DEFF3FC0DEFF445012000CC014F098
:10A19A000DC015F00EC016F00FC017F01006D8A0AB
:10A1AA00110610280FE11128D8A40CD0000E0D6E4C
:10A1BA00000E0C6E1200144A152A164A172A1006A7
:10A1CA00D8A0110614C0F6FF15C0F7FF0800F55015
:10A1DA000009D8B418D016C0D9FF17C0DAFFDF506B
:10A1EA00D8B411D010501110D8B40DD016C0D9FF60
:10A1FA0017C0DAFF14C0F6FF15C0F7FFDE500900DA
:10A20A00F518D8B4D8D714C0F6FF15C0F7FF080060
:10A21A00F5CF12F016C0D9FF17C0DAFFDF50136E60
:10A22A001350125C0C6E0D6AD8A00D06120003D0F2
:10A23A000C4A0D2A0E2A0E50D96EDA6ADF500F6EBA
:10A24A000CC0F6FF0DC0F7FF000EF86E0F0EF76494
:10A25A0003D00800F55005D0F6CFE9FFF7CFEAFFA3
:10A26A00EF500F18D8A414D00CC0F6FF0DC0F7FF9A
:10A27A00000EF86E0F0EF76403D00800F55005D0F3
:10A28A00F6CFE9FFF7CFEAFFEF500009D8A4D0D7FD
:10A29A000CC0F6FF0DC0F7FF000EF86E0F0EF76444
:10A2AA0003D00800F55005D0F6CFE9FFF7CFEAFF53
:10A2BA00EF500F6E0E50D96EDA6ADF50106E1050E2
:10A2CA000F5C0C6E0D6AD8A00D0612000DC013F0BB
:10A2DA000EC014F013501410D8B43ED013C0D9FFD6
:10A2EA0014C0DAFFDE50DE10D8B436D013C0D9FF5E
:10A2FA0014C0DAFFDECF0FF0DDCF10F00FC0D9FFA8
:10A30A0010C0DAFFDF50D8B427D020EE02F0135085
:10A31A00D9261450DA2213C0E1FF14C0E2FF00EE7E
:10A32A0006F0E650E926E550EA22DE50EE1814E17E
:10A33A00DE50EE18D8A410D013C0D9FF14C0DAFF2B
:10A34A0010EE01F0DE50E126DD50E222E75003EC88
:10A35A005AF00F6E0FA002D0090E1200000E120062
:10A36A00EF0E0001806FF90E816FCFCF82F0836B01
:10A37A00CECF84F0856BC9EC59F07250FD0B726E2A
:10A38A00340E0C6E0B0E0D6EE50E0E6E020E0F6E77
:10A39A00000E116E050E106ED9EC56F0390E0C6EC9
:10A3AA000B0E0D6EC50E0E6E020E0F6E000E116EA6
:10A3BA00130E106ED9EC56F072500209726E4C0EE2
:10A3CA000C6E0B0E0D6ED80E0E6E020E0F6E000E78
:10A3DA00116E0D0E106ED9EC56F0000E4A6E250E57
:10A3EA00496E44EC36F07250FD0B726E8990120081
:10A3FA0025EE04F0DE50DE10D8B4FAD700C514F00A
:10A40A0001C515F0060E1424D96E050E1520DA6E54
:10A41A00DF50126E060E1424D96E070E1520DA6E5E
:10A42A00DF50136E144A152AFF0E0E6E010E0F6EC0
:10A43A0014C010F015C011F00E5010160F5011165E
:10A44A0010C000F511C001F5F29E25EE04F0DE06FB
:10A45A00000EDD5AF28E0CC0D9FF0DC0DAFF13C010
:10A46A00DFFF25EE04F0010EDBBE06D0000EDE5C37
:10A47A00020EDE58D8B002D089B29382125012006E
:10A48A000F50D8B403D00F50D8A404D00D50D4EC38
:10A49A0059F012000F50D96EDA6A040ED926DE502E
:10A4AA00DE10D8B414D00F50D96EDA6A040ED92649
:10A4BA000F50E16EE26A020EE126DE50E65CE650DB
:10A4CA00800A146EDE50800A1458D8B012000F5059
:10A4DA00D96EDA6A020ED926DECF10F0DDCF11F07E
:10A4EA000F50D96EDA6ADECF12F0DDCF13F01050BA
:10A4FA001224D96E11501320DA6E0DC0DFFF0F50EF
:10A50A00D96EDA6A020ED926DE2A000EDD22120080
:10A51A006EA108D01CC015F01DC016F01BC017F0A4
:10A52A0052EC58F01FBE05D01EC023F01FC024F005
:10A53A0004D0000E246E000E236E000E226E000E52
:10A54A00216E0AD0000E0E6E200E0D6E1BC00FF08B
:10A55A0045EC52F0214A222A2350215C2250800ADB
:10A56A00206E2450800A2058D8A0ECD701016EB181
:10A57A0008D01CC015F01DC016F01BC017F052EC15
:10A58A0058F01CC012F01DC013F0FBEC56F023501B
:10A59A0012241B6E245013201C6E1200000E8C6EA7
:10A5AA00000E8A6E95689368000E0101A56F000E71
:10A5BA00966F000E716E000E7F6F000E7E6F89928D
:10A5CA008994000E9C6F000E9B6F200E9E6F400EAA
:10A5DA009D6F000E7D6F000E7C6F0AD0000E7C25E9
:10A5EA00D96E040E7D21DA6E000EDF6E7C4B7D2B58
:10A5FA007DBFF4D77D05D8A0F1D7000E7D6F000E80
:10A60A007C6F0AD0340E7C25D96E0B0E7D21DA6E52
:10A61A00000EDF6E7C4B7D2B7DBFF4D77D05D8B055
:10A62A001200F0D724EC3FF0D8C0F5F0D9C0F6F00C
:10A63A00F551F611D8B405D0F5C0EFF0F6C0F0F038
:10A64A00120082B415D06E50200D040EF324B16F9F
:10A65A00020EF420B26F000EB36F040EB46F010E37
:10A66A00B66F000EB56FF30EB76F12EC0FF0F96FFD
:10A67A00F951D8B40ED0BA0E806FFD0E816FF9C0B1
:10A68A0082F0836BC9EC59F0F9C0EFF00001F06B6E
:10A69A001200D4EC4DF0010E0101A76F000E00016B
:10A6AA00F06F000EEF6F1200260E0001806FFB0E96
:10A6BA00816FCFCF82F0836BCECF84F0856BC9ECEC
:10A6CA0059F0000E4A6E000E496E6E50140D070EB8
:10A6DA00F324D96E010EF420DA6EDE6ADE6ADE6ACF
:10A6EA00DD6A6E50140D130EF324D96E010EF42098
:10A6FA00DA6E000EDF6E6E50140D0F0EF324D96E53
:10A70A00010EF420DA6EDE6ADE6ADE6ADD6A494A22
:10A71A004A2A4ABEDAD74A5004E1040E495CD8A054
:10A72A00D4D78990000E6D6E1200000E146E000EC2
:10A73A00156E000E166E000E176E105011101210C4
:10A74A001310D8B42AD0010E186E06D0D89010363D
:10A75A00113612361336182A13AEF8D7D890143693
:10A76A0015361636173610500C5C11500D5812500B
:10A77A000E5813500F58D8A009D010500C5E115023
:10A78A000D5A12500E5A13500F5A1480D890133281
:10A79A00123211321032182EE1D714C00CF015C043
:10A7AA000DF016C00EF017C00FF01200146E0C0E4A
:10A7BA001418D8B409D01EEC5AF0ACEC59F00009C0
:10A7CA00D8A402D0FF0E120014504009F1EC59F03F
:10A7DA001150F1EC59F01050F1EC59F00F50F1EC26
:10A7EA0059F00E50F1EC59F0010E136E1450D8A422
:10A7FA0002D0950E136E080E1418D8A402D0870E34
:10A80A00136E1350F1EC59F00C0E1418D8B412EC64
:10A81A005AF00A0E136E12EC5AF0126E12AE02D0F1
:10A82A00132EF9D71250120011D0030E0DD0050EB7
:10A83A000E6E000E0101736F000E726F2FD0010EA3
:10A84A0003D0020E01D0000E0E6E28D072C10CF099
:10A85A0073C10DF00D50000AD8B40AD0020AD8B458
:10A86A000FD00F0AD8B411D02A0AD8B413D0EBD714
:10A87A000C500A0AD8B4D9D71E0AD8B4D8D7E3D705
:10A88A000C50BC0AD8B4DDD7DED70C50AC0AD8B409
:10A89A00D6D7D9D70C500F0AD8A4D5D70E50120044
:10A8AA000CC014F00DC015F00EC016F00FC017F052
:10A8BA00000E196E000E186E1006D8A01106102888
:10A8CA0003E11128D8B41AD014C0D9FF15C0DAFF91
:10A8DA00144A152ADF50126E16C0D9FF17C0DAFFC4
:10A8EA00164A172ADF50136E1350125C186E196A33
:10A8FA00D8A0190618501910D8B4DED718C00CF011
:10A90A0019C00DF012001050111012101310D8B403
:10A91A0024D0010E146E06D0D89010361136123695
:10A92A001336142A13AEF8D710500C5C11500D5878
:10A93A0012500E5813500F58D8A008D010500C5E61
:10A94A0011500D5A12500E5A13500F5AD8901332F2
:10A95A00123211321032142EE7D70CC00CF00DC08F
:10A96A000DF00EC00EF00FC00FF01200490E0001DC
:10A97A00806FFD0E816FC9EC59F072500209726E38
:10A98A002BEE34F0A1C1DFFF000EE8CF35FB0D0E30
:10A99A00E8CF36FB000EE8CF37FB82A403D0600E67
:10A9AA00E8CF37FB82A406D036CB4FF0200E4F12E9
:10A9BA004FC036FB000E4A6E040E496E44EC36F068
:10A9CA007250FD0B726E000E0101A16F8990120088
:10A9DA00070E116ED00E106E0DD012EC5AF0126ED8
:10A9EA001228D8A40BD0A00E00D0E82EFDD710064E
:10A9FA00D8A0110610501110D8A4EFD7FE0E1218C5
:10AA0A00D8B402D0000E120012EC5AF00CC0D9FFD2
:10AA1A000DC0DAFFDF6E0C4A0D2A0E06D8A00F060B
:10AA2A000E500F10D8A4F0D712EC5AF012EC5AF0CC
:10AA3A00010E12004A6E850E4B6EF50E4C6E000E1C
:10AA4A00496E0CD04BC0F6FF4CC0F7FF4B4A4C2A5C
:10AA5A000800F5500009D8A4F5D7492A4A504918E0
:10AA6A00D8B409D04BC0F6FF4CC0F7FF0800F55028
:10AA7A000009D8A4E7D76E0E0001806FFE0E816F21
:10AA8A004AC082F0836B4BC084F04CC085F0C9EC9D
:10AA9A0059F0120035EC58F00009D8A402D0000E83
:10AAAA0012001050F1EC59F0FD0E1018D8B420D055
:10AABA00020E126E000E116E0EC0D9FF0FC0DAFF21
:10AACA00DF50F1EC59F00E4A0F2A1106D8A01206EF
:10AADA0011501210D8A4F0D712EC5AF012EC5AF016
:10AAEA0012EC5AF0136E13501F0B050AD8A4D7D7CD
:10AAFA00010E120012C017F013C018F012D015067A
:10AB0A00D8A01606142A1404D96EDA6A17C0E1FF0F
:10AB1A0018C0E2FF174A182ADFCFE7FFE750D8B478
:10AB2A000DD015501610D8B409D0E9D717C0D9FFDF
:10AB3A0018C0DAFF000EDF6E174A182A1506D8A0C9
:10AB4A0016061528F3E11628D8B41200EFD7000E1E
:10AB5A00146E000E156E000E166E000E176E0CA007
:10AB6A0008D01050142611501522125016221350D4
:10AB7A001722D8901036113612361336D8900F3263
:10AB8A000E320D320C320C500D100E100F10D8A4CC
:10AB9A00E6D714C00CF015C00DF016C00EF017C0A1
:10ABAA000FF0120015D00DC0F6FF0EC0F7FF000E11
:10ABBA00F86E0F0EF76403D00800F55005D0F6CFF3
:10ABCA00E9FFF7CFEAFFEF50DEEC59F00D4A0E2A03
:10ABDA000DC0F6FF0EC0F7FF000EF86E0F0EF764F9
:10ABEA0003D00800F55005D0F6CFE9FFF7CFEAFF0A
:10ABFA00EF500009D8B41200D6D75AC05DF05BC036
:10AC0A005EF0000E0101696F000E686F0DD059C029
:10AC1A004BF05D0E4C6E5CC04DF066EC44F04B5050
:10AC2A00010168274C5069235DC0F6FF5EC0F7FF3B
:10AC3A000800F5500009D8A4EAD768C159F069C1DB
:10AC4A005AF012009F0E146EFF0E156E12C016F007
:10AC5A0013C017F01450162615501722175006E184
:10AC6A001A0E165CD8B002D0010E01D0000E186E72
:10AC7A00196A18501910D8B405D05F0E1214126E42
:10AC8A00136A120012C012F013C013F0120002D09D
:10AC9A000C4A0D2A0CC0F6FF0DC0F7FF0800F5504C
:10ACAA000009D8B40FD00CC0F6FF0DC0F7FF08009A
:10ACBA00F550106E116A0E501018EAE10F50111873
:10ACCA00D8A4E6D70CC0F6FF0DC0F7FF0800F55070
:10ACDA000C6E0D6A120080004C4142454C31000056
:10ACEA000002800000000000000E00006870646925
:10ACFA00736B2E63666700010912200100010017B9
:10AD0A0000002D119420D00F000100000000000067
:10AD1A0000000000099F02800102E8054C0E0001B4
:10AD2A00806FFF0E816FC9EC59F0340E0C6E0B0E5A
:10AD3A000D6E000E0F6E000E0E6E010E116E000EDD
:10AD4A00106E0EEC49F02BEE34F0A3C1DFFF000EBB
:10AD5A004A6E010E496E44EC36F0000E0101A36FF3
:10AD6A001200630E0001826F5FC083F060C084F03E
:10AD7A00000E866F000E856F000E886F000E876FBB
:10AD8A00830E596E61C05AF062C05BF0820E5C6E2F
:10AD9A0002EC56F0000185515F24D96E865160207D
:10ADAA00DA6E000EDF6E12000EC015F00FC016F03C
:10ADBA000CC013F00DC014F010D015C0D9FF16C086
:10ADCA00DAFFDF50126E154A162A13C0D9FF14C0D3
:10ADDA00DAFF12C0DFFF134A142A1006D8A01106A0
:10ADEA001028EBE11128D8B41200E7D712C014F0EA
:10ADFA0013C015F002D0124A132A12C0F6FF13C06C
:10AE0A00F7FF000EF86E0F0EF76403D00800F55036
:10AE1A0005D0F6CFE9FFF7CFEAFFEF500009D8A433
:10AE2A00EAD71450125C126E15501358136E1200A2
:10AE3A0020EE1AF00C50D9260D50DA220EC0DFFF90
:10AE4A0020EE1BF00C50D9260D50DA220FC0DFFF7E
:10AE5A0020EE14F00C50D9260D50DA2210C0DFFF74
:10AE6A0020EE15F00C50D9260D50DA221150DF6E63
:10AE7A001200196E19AE12D0199E000E0E6E000E37
:10AE8A000F6E000E106E000E116E370EDBEC53F0D3
:10AE9A001A6E010E1A6402D01A50120015C00EF072
:10AEAA0016C00FF017C010F018C011F01950DBECE3
:10AEBA0053F012000CC012F00DC013F00EC014F0C3
:10AECA000FC015F00ED014C0D9FF15C0DAFF12C09A
:10AEDA00E1FF13C0E2FFDFCFE7FF144A152A124A47
:10AEEA00132A1006D8A011061028EDE11128D8B4AB
:10AEFA001200E9D7010E126E200E0C180D10D8B4EC
:10AF0A0014D0F70E0E6EFF0E0F6E0CC010F00DC0AF
:10AF1A0011F00E5010260F501122115004E1050EA7
:10AF2A00105CD8A002D0000E126E12C00CF00D6A8E
:10AF3A0012000C6E0C50D8B40ED023EC5AF0200E2E
:10AF4A00E82EFED726EC5AF0CC0E00D0E82EFDD71C
:10AF5A0000D000D0120023EC5AF0C00E00D0E82E28
:10AF6A00FDD726EC5AF0350EE82EFED700F0120077
:10AF7A00FB0E0001806FFE0E816FC9EC59F0340E92
:10AF8A000C6E0B0E0D6E000E0F6E000E0E6E010E85
:10AF9A00116E000E106E0EEC49F02BEE34F0A3C1C8
:10AFAA00DFFF8990000E0101A36F1200340E0C6EB0
:10AFBA000B0E0D6E000E0F6E000E0E6E010E116E50
:10AFCA00000E106E0EEC49F0010EE8CF34FB725001
:10AFDA000209726E000E4A6E010E496E44EC36F09A
:10AFEA007250FD0B726E12005CC04FF05DC050F0E3
:10AFFA0010EC3DF05E6E5E50D8A412D05CC00DF02D
:10B00A005DC00EF06BEC51F05E6E5E50D8A408D0B5
:10B01A005CC0D9FF5DC0DAFF000EDE6E000EDD6E89
:10B02A005E50120023EC5AF00A0E0D6EF80EE82E4E
:10B03A00FED70D2EFCD700D026EC5AF0E00E00D039
:10B04A00E82EFDD7FAEC59F00E6E090E0D6E840E3D
:10B05A00E82EFED70D2EFCD726EC5AF00E50120021
:10B06A00130E0D6E880E0C6E0CD012EC5AF0FF0AFD
:10B07A00D8B40BD0A00E00D0E82EFDD70C06D8A06D
:10B08A000D060C500D10D8A4F0D70C500D10D8B4E2
:10B09A0002D0010E1200000E1200000E1A6E000EEF
:10B0AA00196E09D018C00DF00E6A17C00FF045ECE2
:10B0BA0052F0194A1A2A19501524D96E1A50162014
:10B0CA00DA6EDF50186E1850D8B41200EBD79F0E04
:10B0DA000E6EFF0E0F6E200E0C10106E000E0D106D
:10B0EA00116E0E5010260F501122115006E11A0E41
:10B0FA00105CD8B002D0010E01D0000E0C6E0D6AA1
:10B10A001200B886AC84B898440EAF6E000EB06ECA
:10B11A00AC98AB8EAB88AB9A9D989D9AD08E9F8A3D
:10B12A00F28EAC90AB9CAC9AAC8A8B91000E8C6F71
:10B13A0012009F0E0E6EFF0E0F6E0CC010F00DC0A7
:10B14A0011F00E5010260F501122115006E11A0E5E
:10B15A00105CD8B002D0010E01D0000E0C6E0D6A40
:10B16A001200BF0E0E6EFF0E0F6E0CC010F00DC057
:10B17A0011F00E5010260F501122115006E11A0E2E
:10B18A00105CD8B002D0010E01D0000E0C6E0D6A10
:10B19A001200D00E0E6EFF0E0F6E0CC010F00DC016
:10B1AA0011F00E5010260F501122115006E10A0E0E
:10B1BA00105CD8B002D0010E01D0000E0C6E0D6AE0
:10B1CA0012000CC012F00DC013F008D012C0D9FF43
:10B1DA0013C0DAFF0EC0DFFF124A132A1006D8A0E6
:10B1EA0011061028F3E11128D8B41200EFD78450C1
:10B1FA00070B0C6E928A80AA03D00C50080F0C6EB3
:10B20A00020E01019119D8A404D00C50FF0A0F0BA9
:10B21A000C6E0C501200000EE8CF00F5000EE8CFBD
:10B22A0001F5000EE8CF02F5000EE8CF03F5000E97
:10B23A00E8CF04F5000EE8CF05F512000C500E0217
:10B24A00F3CF10F0F4CF11F00C500F02F350112687
:10B25A000D500E02F350112610C00CF011C00DF063
:10B26A00120023EC5AF0200EE82EFED726EC5AF0F4
:10B27A00300EE82EFED7FAEC59F00D6EB00E00D063
:10B28A00E82EFDD70D501200120E0001806FFF0E3E
:10B29A00816FC9EC59F0000E6C6E000E6B6E000ED9
:10B2AA006A6E8990000E0101A36F1200000E01015F
:10B2BA00A46F000E706E000E856F000E846F020E72
:10B2CA00A36F8990000EA26F000EA16F1200000EEC
:10B2DA000E6E000E0F6ED8900E3236EC59F0000941
:10B2EA00D8A40E8E0F2A070E0F64F5D70E5012003F
:10B2FA004D5946494C4531323334000100000001B2
:10B30A0000002000131012000000010000000000DD
:10B31A000C6E0C50D8B408D0000EC66E010EC66E64
:10B32A00400EC76EC68A1200000EC66E020EF7D70E
:10B33A00C2900F0EC16E070EB46E4F0EC86E000E8D
:10B34A00946E948894829482000E826E12002BEC82
:10B35A005AF012EC5AF035EC58F00009D8B402D081
:10B36A00010E12001EEC5AF0000E12000D6E000EB5
:10B37A000E6E0D50010B9EEC57F0D8900D320E2A2E
:10B38A00070E0E64F6D71200820E486E80C019F0BE
:10B39A0081C01AF0480E1B6EA6EC1FF012000C6E4C
:10B3AA0003D030EC5AF004009EA8FBD70CC0ADFFC6
:10B3BA0012000C6E03D030EC5AF004009EA8FBD7A2
:10B3CA000CC0ADFF12000C6E02D0898889980C0659
:10B3DA000C28D8B41200F9D70C6E0CC0C9FFC7B03C
:10B3EA00FED7C7A0FED7C9501200928880A802D003
:10B3FA00010E01D0000E0C6E0C5012000C6E0C5097
:10B40A00D8B402D0010E1200735012008980010EC6
:10B41A006D6E000E6D6E89901200C968C7B0FED7B6
:10B42A00C7A0FED7C950120004C50CF005C50DF01F
:10B43A00120029EC5AF012EC5AF0120089989298EC
:10B44A00120089989288120082801200829012005B
:03B45A00340BE7C9
:05B45E001200120001C4
:10F58400004F4B004449534B5F455252004E4F5479
:10F594005F5245414459004E4F5F46494C45004E29
:10F5A4004F545F4F50454E4544004E4F545F454EB7
:10F5B40041424C4544004E4F5F46494C455F5359C8
:10F5C4005354454D00000D0A202532582025325849
:10F5D400202532732025327320253273202532737F
:10F5E400202532732025327320253273202532736F
:10F5F4002025347320253473202534732025347357
:10F604002025347320253473202534732025347346
:10F6140020000D0A253032582530325820535338F3
:10F62400303A53657420537461747573206D61733B
:10F634006B2025582025582025582025582025584A
:10F6440020255820255820255820000D0A25303221
:10F65400582530325820535338303A20496E63725B
:10F66400656D656E743A205365656B696E672074C9
:10F674006F20256C642028256C582920000D0A4829
:10F68400504469736B204D6B20494920283138461A
:10F6940034363230292025732025732025732053D6
:10F6A40074617274696E672E2E2E0D0A000D0A2580
:10F6B400303258253032582053533830783A536515
:10F6C400656B3A205365656B696E6720746F2025FE
:10F6D4006C752028256C582920000D0A25303258D5
:10F6E4002530325820535338303A427566662077B5
:10F6F4007220256C6420627974657320727820000E
:10F704000D0A414D3A556E62756666207264206337
:10F714002F682F733A2025642F25642F25642073C6
:10F724003A256C6420000D0A547269656420746F74
:10F734002074616C6B207768696C7374206E6F74CD
:10F7440020616464726573736564000D0A414D3A07
:10F754004275666620726420632F682F733A2025F1
:10F76400642F25642F256420733A256C6420000DD2
:10F774000A253032582530325820313A52656164B6
:10F784002072746E2025582C2025642072656164D3
:10F7940020000D0A414D3A42756666207772206357
:10F7A4002F682F733A2025642F25642F2564207336
:10F7B4003A256C64000D0A25303258253032582021
:10F7C40053533830783A577269746520256C642035
:10F7D40028256C582920000D0A253032582530324E
:10F7E400582053533830783A5374617475732C200D
:10F7F400756E697420256420000D0A253032582561
:10F804003032582053533830783A52656164202599
:10F814006C752028256C582920000D0A2530325893
:10F824002530325820535338303A5365742061647C
:10F83400647265737320256C5820000D0A253032DC
:10F84400582530325820535338303A436820696E73
:10F854006420436C65617220256420000D0A5265A2
:10F8640061642072657475726E732025582C20258E
:10F87400642062797465732072656164000D0A4DB9
:10F88400617820566563746F72206469736B2025F8
:10F894006420256C642028256C582920000D0A2535
:10F8A400303258253032582053533830783A537414
:10F8B400617475735B25645D20255820000D0A254D
:10F8C4003032582530325820535338303A53657407
:10F8D400206C656E67746820256C5820000D0A251D
:10F8E4003032582530325820535338303A416D69FC
:10F8F400676F20436C65617220256420000D0A2522
:10F904003032582530325820535338303A536574C6
:10F9140020766F6C756D6520256420000D0A414DBD
:10F924003A205365656B3A202564202564202564BC
:10F934002025642C20733A256C64000D0A2530328E
:10F94400582530325820535338303A52707420516D
:10F954005354415420256420000D0A44736B73658D
:10F964006C2069732025642C206E756D626572208D
:10F97400697320256420003C6964656E743E20250B
:10F9840058202558206E7266643A2564206E64619E
:10F99400633A2564000D0A25303258253032582048
:10F9A400566563746F7220256C642028256C582971
:10F9B40020000D0A25303258253032582053533850
:10F9C400303A53657420756E697420256420000DE7
:10F9D4000A253032582530325820535338303A559E
:10F9E4006E6B6E6F776E20255820000D0A2530321D
:10F9F40058253032582053533830783A446573636D
:10FA04007269626520000D0A25303258253032585B
:10FA140020535338303A496E6974206469736B20FB
:10FA2400000D0A25303258253032582053533830CF
:10FA34003A52712073746174757320000D0A323A5E
:10FA4400526561642072746E2025582C2025642030
:10FA54007265616420000D0A253032582530325811
:10FA640020535338303A44657363726962652000E9
:10FA74000D0A253032582530325820256420627909
:10FA84007465732073656E742000466F756E642010
:10FA9400616E205254432066696C65206174202590
:10FAA400580D0A004C6F6F6B696E6720666F722089
:10FAB400616E205254432066696C650D0A000D0A7C
:10FAC400414D3A20496E63723A2025642025642012
:10FAD40025642025642C200046696E6446696C65A3
:10FAE400206661696C6564207365617263680D0AE0
:10FAF400000D0A414D3A42756666207772202564EE
:10FB0400206279746573207278000D0A4750494267
:10FB14002072633A25642025642062797465730D2C
:10FB24000A000D0A253032582530325820535338F4
:10FB340030783A436C65617220000D0A577269741B
:10FB4400655F736563746F7273206661696C2025E9
:10FB540064000D0A5365656B20746F20256C642066
:10FB64006661696C6564202564000D0A253032588D
:10FB74002530325820535338303A5772697465200F
:10FB8400000D0A4F70656E696E672065786973743D
:10FB9400696E6720257320005365656B696E672065
:10FBA400746F20736563746F722025580D0A0046C4
:10FBB400696E6446696C65206661696C656420726F
:10FBC4006561640D0A000D0A5365656B696E6720F3
:10FBD400746F20256C642028256C5829000D0A2593
:10FBE4003032582530325820535338303A526561F8
:10FBF4006420000D0A2530325825303258205353E2
:10FC040038303A44534A20000D0A25303258253002
:10FC1400325820535338303A4E4F50200025582044
:10FC2400255820255820255820256C752020200A89
:10FC3400000D0A566563746F7220256C64202825B4
:10FC44006C582920004469736B206368616E676592
:10FC54003A20256420200D0A000D0A4469736B20A4
:10FC64005374617475733A2025582C20000D0A577B
:10FC7400616974696E6720666F72206361726420C3
:10FC8400000D0A72632025582C20256420627974A3
:10FC940065730D0A000D0A46696C65202573206999
:10FCA40073206F70656E20000D0A526561642062D6
:10FCB40065796F6E6420656E64000D0A5365656B2B
:10FCC400206265796F6E6420656E64000D0A4F7062
:10FCD400656E696E67206E657720257320000D0AB6
:10FCE40020256C642062797465732073656E7400DA
:10FCF4000D0A545844415441206C656E20256420FB
:10FD0400000D0A46696C6520255820697320257307
:10FD140020000D0A4469736B20255820697320253F
:10FD24007320000D0A4469736B206E756D626572F1
:10FD3400202564004E6F742061204C49462064697C
:10FD4400736B0D0A000D0A414D3A53656E642073BE
:10FD54007461747573000D0A52656164696E67207D
:10FD64005254430D0A000D0A416D69676F20393101
:10FD74003231440D0A000D0A53532F3830203931E3
:10FD84003232440D0A000D0A44736B73656C2069AA
:10FD94007320256420000D0A5265616420256420C7
:10FDA4006279746573000D0A486F73742062797404
:10FDB4006532202564000D0A5772697465206661F6
:10FDC400696C202564000D0A486F7374206279748D
:10FDD4006573202564000D0A4F70656E696E672097
:10FDE40025732020000D0A4465627567206973201D
:10FDF400256420000D0A50726F746F2069732025EA
:10FE04006420000D0A5265616420636F6E66696741
:10FE140020000D0A46696C656E616D6520257320AE
:10FE240000566563746F722069732025580D0A00AB
:10FE34002041544E206173736572746564200022FE
:10FE44002A2B2C3A3B3C3D3E3F5B5D7C7F000D0AF8
:10FE540056616C75653A2025580D0A0020465320DA
:10FE6400747970652025640D0A0072633D25752040
:10FE740046525F25730D0A000D0A466F726D617458
:10FE840074696E6720000D0A4E6F206361726420EE
:10FE94002564002F6C6966646174612E62696E006A
:10FEA4000D0A25732025582025580D0A007B505033
:10FEB40025642025642025647D002A2A2056657245
:10FEC400696679202A2A000D0A4D6F756E74696E71
:10FED4006720004A616E2032352032303230000D06
:10FEE4000A4B3A257320563A2573000D0A7362793A
:10FEF400746573202564000D0A414D3A57616B65A2
:10FF040075700068706469736B2E636667000D0A10
:10FF1400414D3A436C656172005B535251206F66E8
:10FF2400665D00466D742065786974200031363A48
:10FF340032313A3532005B2532582025645D005B4E
:10FF4400535251206F6E5D000D0A414D3A44534A9D
:10FF5400005B25582025645D002D3E202558200097
:10FF64005458446174610044534B53454C004E4112
:10FF74004D452558004449534B25580072633D258F
:10FF84006420005B4D4C415D0044454255470050A0
:10FF9400524F544F002025303258007B4552527D39
:10FFA400004946432000454F49200052454E200059
:10FFB40041544E2000535251200044415620004EDB
:10FFC400444143004E52464400302E3900525443BB
:10FFD400002025580025325800207C2000443000A1
:10FFE4004431004432004433004434004435004476
:0BFFF40036004437002563002E00009B
:020000040020DA
:08000000FFFFFFFFFFFFFFFF00
:020000040030CA
:0E000000FF06191EFF8181FF0FC00FE00F40A9
:00000001FF
